:020000040000FA
:20000000303600102D53020031530200335302003553020037530200395302009AD6F1EFE6
:200020000000000000000000000000003B5302003D530200000000003F5302004153020074
:20004000435302000D56020043530200B19C0200435302004D89020043530200FD8B02002A
:200060004353020043530200435302004353020043530200435302004353020043530200C0
:200080004353020043530200435302004353020043530200435302004353020043530200A0
:2000A00099BB020043530200435302004353020043530200435302004353020043530200C2
:2000C00043530200435302004353020000F002F800F08CF80AA090E8000C82448344AAF1A4
:2000E0000107DA4501D100F081F8AFF2090EBAE80F0013F0010F18BFFB1A43F001031847A0
:20010000C4C1030004C203000A444FF0000C10F8013B13F0070408BF10F8014B1D1108BF93
:2001200010F8015B641E05D010F8016B641E01F8016BF9D113F0080F1EBF10F8014BAD1CCB
:200140000C1B09D16D1E58BF01F801CBFAD505E014F8016B01F8016B6D1EF9D59142D6D3D1
:20016000704700000023002400250026103A28BF78C1FBD8520728BF30C148BF0B6070479F
:20018000662900F03B8169292FF0E48064292FF0E18075292FF0DE806F292FF07581782999
:2001A0002FF09E810368DB0928BF41F0800163292FF08A8673292FF08F86E3292FF09A8643
:2001C000002070471FB530F087FF2FF005FF04000020002130F0BCFE401C6060002000212F
:2001E00030F0A0FEE0601FBD10B510BD2FF0F4FF1146FFF7E7FF00F019F930F012F803B46B
:20020000FFF7F2FF03BC30F053F8000010B5782119482FF0A3FB19494FF0FF30088010BD2C
:2002200016480188491C09B201800A290CD001EB41021149436841F8223001EB820183680E
:200240004B60C06888607047FEE70C4910B5B1F90000421C0ED0084A00EB4003401E52F81F
:20026000234002EB83024C6053688B609268CA60088010BDFEE700004002001004C00720BC
:2002800038B50546684604F044FE0D4C000611D49DF80000032809D087200A4920600020CB
:2002A0000860784608490860872038BD0AF059F9000601D5206838BD284607F0C9FA38BD01
:2002C00008C007200CC0072010C0072010B14FF0FF3070470248406D40F3C020401C704742
:2002E00000C0092091FBF2F302FB1311C0E90031704770477047704770470000FFFFFFFF1A
:200300007FB5054603A804F004FE244C00063CD49DF80C0001282ED00026022809D087209F
:2003200020601F48066078461E490860872004B070BD00200AF03BF9000626D42888ADF8B8
:2003400004006888ADF8060028798DF808008DF8096001A809F036F8000616D469462B2028
:2003600016F06EFB000610D49DF80000C00702D001208DF80C0003A804F0D2FD000604D4F8
:20038000284607F051F9000601D52068CFE703208DF80C0003A804F0B2FDC8E708C00720F4
:2003A0000CC0072010C0072038B50446684604F0B0FD01060A4801D5006838BD9DF800109C
:2003C000032909D087210160064900200860784605490860872038BD204607F00BFB38BDD0
:2003E00008C007200CC0072010C0072002F0FF0343EA032242EA02422FF090BA2FF008BC22
:20040000D874D498290C0A6802F8010B0A6070474F637420313720323031330000000000C2
:2004200031373A30333A3235000000009D4C86B00027208840F0020020809B4826F0F9FC68
:20044000994D288830F4805010D00127FFF7E8FE2E2014F0D3FF01200EF0BAFB10B108204D
:200460002AF0E4FEFFF7F1FE02F018FB2888000406D501270CF0D7FA000601D502F00EFB3B
:20048000002028808948007828B125F055F910B187A02AF0AAFE01F035F88B4DAE6801A8B0
:2004A00026F008FC00F0E6FF10B1012702F0F6FA01F065F8DFF81482C0B1FFF7B1FE01F0C0
:2004C000B3F9FFF7C2FED8F80000062802D000217FA004E0834902200870002182A02AF003
:2004E00008FD208840F0020020800CE001F061FA38B1FFF795FE01F097F9FFF7A6FE02F0C6
:20050000CDFA01F0D4FC7D48A968891B8142FBD302A826F0CFFB1FF0D5FE000601D502F00E
:20052000BDFADFF8E091764E99F8000006EB001000688047000601D502F0B0FA01F0DCFCF6
:20054000000601D502F0AAFA9DF80A009DF80610884201D0012000E0002001F00FFD00B175
:20056000012701F05BFD00F057FB6946532016F067FA000601D502F091FA9DF8000000F061
:2005800001008DF800006FB9B0B101200EF020FB000601D502F082FA0EF01EF9000601D5D7
:2005A00002F07CFA9DF8000030B101200EF010FB000601D502F072FA4F460DF10C093878A1
:2005C00006EB0010C0688047000601D502F066FA387806EB001040688047000601D502F00F
:2005E0005DFA387806EB001080688047000601D502F054FA00202AF0B1F9D8F800000C2840
:2006000005D004F075FA000601D502F047FA208840071ED501202AF0A1F9D0B903A804F0B4
:20062000F2FC50B909F1020004F0FEFC28B909F1040004F00AFD000601D502F02FFA32498D
:200640009DF81000087003A805F0EAFD08B906F067FB208810F0380F1DD001202AF07EF94F
:20066000000618D4A8682949AA68121A8A42FBD32088000701D50EF0EEF82088C00601D581
:2006800005F072FD2088800605D5012007F006FF01200EF09DFA01202DF02DFF2AF0ACFEED
:2006A0008DE7000002C0072000000010D1C10720C0E2F2EEEEF2F0E5E7F7E8EA20E2FBEA46
:2006C000EBFEF7E5ED0A0000000009400CC007208E9888818A80208F808C9F9288208F8442
:2006E0000A0A000000C00720878D208D852082828584858D0A0A0A0A0A000000E0C8100090
:200700006C0100106801001085C00720A08601002DE9F047FB4DFC4EFC4F9046C3B15C1E62
:200720000BD4DFF8EC93642200232EF0FDFC19F8023008F80430641EF5D5084310D089202D
:20074000286004203060784638608920BDE8F0878820286009203060784638608820F5E77F
:20076000002028603060784638600020EEE710B500220BE0835C03F00F04092C03D803F03C
:20078000F003902B01D9002010BD521C8A42F1D3012010BD2DE9FF4FDA4CDFF86C93DFF8C1
:2007A0006CA383B08346082A30D872B30020CDE90000012000214FF0860E00BF0BEB020528
:2007C00015F8018C08F00F05092D12DCA0FB056CEF1701FB05C500FB0755DDE900C71CEB8C
:2007E00006066F414FEA1818B8F1090FCDE9006715DD2020C4F800E07946C9F80000862002
:20080000CAF8001007B0BDE8F08FFFE7882009212060C9F800107946CAF80010F2E70A2688
:20082000A0FB065C01FB06C1002700FB0711A5FB080701FB08774FEAE87605FB0676DDE9BB
:2008400000C71CEB00007741CDE900070A26A5FB060C002701FB06C105FB0711521EADD183
:20086000D90001208840DDE90025401EC117801AA94108D2892004212060C9F80010794659
:20088000CAF80010BEE71A46694604982EF08BFF002020607946C9F80000CAF80010B1E704
:2008A00030B5401E83B240F2B554B3FBF4F0820604FB1030401C120E80B24FF4B773984237
:2008C0000BD9521CD2B2A0F5B77003E0521CD2B2A0F26D1080B29842F8D2202801D201238D
:2008E00019E01F3880B2930701D01C2300E01D23984201D802230EE0C01A854C002380B2E6
:20090000643403E0401B5B1CDBB280B2E55C8542F8D3DB1CDBB20A704B7088707949002065
:20092000086079490860784678490860002030BD10B5027840F26D135A430A80744C43789E
:200940006E3434F813301A440A8083781A4492B20A8003789C0705D14078022802D802EBDA
:20096000930003E0012000EB93001044088065490020086064490860784664490860002048
:2009800010BD10B581784FF0FF32C9B143780D2B18D2DFE803F017070D070A070A07070AE6
:2009A000070A07001F290BD80FE01E2908D80CE00078800702D01C2902D806E01D2904D9F9
:2009C000104610BD6FF0010010BD002010BD08B5C2788DF8022082788DF801200088A0F57F
:2009E000FA608DF800006846FFF7A2FF08BD2DE9F04F8A46434D0021DFF80CC1DFF80C8130
:200A000083464FF08609B3EB420F14D301201FE0A2EB000E1BF80E4004F00F04092C0ADC2B
:200A2000A3EB400606EB0A0730347C701BF80E402409092C08DDC5F80090CCF80010794608
:200A40008620C8F80010DEE630340AF80640401C9042DDD9012000EB4200302203E01E1A11
:200A6000401C0AF806209842F9D92960CCF8001079460020C8F80010C5E67CB50D4601A961
:200A8000FFF70EFF1F4C000601D520687CBD9DF8040000909DF805309DF806201DA1284671
:200AA0002EF0DEFB184900202060086078461749086000207CBD3C23B0FBF3F230B503FB25
:200AC0001203D4B20A20B4FBF0F202F1300500FB12420D7030324A703A228A70B3FBF0F2CA
:200AE00000FB123002F13004CC70303008710549002008600449086078460449086000205F
:200B000030BD000008C007200CC0072010C00720C6110300253032752D253032752D25308E
:200B20003275000010B53C24B0FBF4F304FB1300DAB2254B9A5C0A70185C48702349002021
:200B4000086023490860784622490860002010BD18B50C466946FFF7A3FE1C49000601D535
:200B6000086818BD9DF802201748825C22709DF80120825C62709DF80020805CA070002083
:200B8000086013490860784612490860002018BD70B5044611B92EF0E7FD014600222023CC
:200BA0000DE0A05CF02801DB103802E0C02802DB4038A05402E0802800DBA354521C8A4267
:200BC000EFDB002070BD0000C611030008C007200CC0072010C00720F8B504460D461646A5
:200BE00089480122694626F0E8FD000602D587480068F8BD9DF80000204000D00120287010
:200C0000022C06D08048401C0222314626F0D5FDF8BD7D48C01CF7E710B5AAB027A809F00E
:200C200091FC7A4C00064BD426AA28A90120FFF7D3FF000644D49DF8A00028B1BDF8980039
:200C4000BDF89C10884209D9714900202060086078467049086000202AB010BD022029F0E4
:200C60002CFF00062CD46C482AF0BFFA000627D4694814302AF0B9FA000621D426AA28A95D
:200C80000220FFF7A9FF00061AD49DF8A000C8B129A9BDF89800FFF703FE000610D49DF85D
:200CA000A4005D4900909DF8A5309DF8A620263101A82EF0D5FA01A82AF097FA000601D578
:200CC0002068C9E75548018841F00201018054490220087001200DF07BFFBDE7FEB501A832
:200CE00009F030FC494C000632D46A4602A90220FFF772FF00062BD49DF80800444D454E84
:200D000028B1BDF80000BDF80410884206D9002020602860784630600020FEBD022029F047
:200D2000CCFE000614D43C482AF05FFA00060FD4394814302AF059FA000609D437480188FE
:200D400041F00201018001200DF042FF000601D52068FEBD91202060BE202860784630607B
:200D60009120FEBD4FF0204301460422184626F024BD4FF0204301460422184626F028BD3B
:200D8000F7B50446204882B00E4605460122694626F013FD1D4F00060ED49DF800000EB184
:200DA000204300E0A0438DF8000001226946284626F00EFD000602D5386805B0F0BD022C1A
:200DC00006D01148401C022204A926F001FDF4E70D48C01CF7E738B50020012201460090B2
:200DE0001046FFF7CDFF094C000606D4012200210220FFF7C5FF000601D5206838BD68467F
:200E0000FFF7B7FF38BD0000040000A008C007200CC0072010C007204E12030002C0072068
:200E200000C007202DE9F04F841A99B071EB030404DA15461F460C46064603E00F4605466D
:200E400016461C4600208346059016E002220023284639462EF0DFF905460F46022200234F
:200E6000304621462EF0D7F90646012205981BEB020B40F100000C460590E80701D1F007B8
:200E8000E4D001200021CDE9220124AA0846A3C2681E67F10001CDE91601CDE91464CDE972
:200EA000126400BFDDE9260180468946C0072AD1DDE92201C20702D1249AD2070BD0321878
:200EC00044EB0100CDE92220DDE924012A1847EB0100CDE92420DDE92201022200232EF042
:200EE0009AF9CDE92201DDE92401022200232EF092F9CDE9240102220023404649462EF056
:200F00008AF9CDE92601DDE91201C20704D0DDE92632181A8A410BDA14A922A800F05CFA2E
:200F200016A924A800F058FA12A926A800F054FADDE9260110900D91C007B3D0DDE91401CD
:200F4000DDE916E2894600BFDDE922319A461B1A71EB090305DBDDE92483B8EB0E0C9341D1
:200F60000BDA16EB0A036141CDE92231DDE9241369187B41CDE92413E6E7BAEB000061EBEE
:200F80000901CDE922012598B8EB0E0160EB0200CDE92410DDE91201109B0D9A1B1A62EB1B
:200FA0000102CDE926320023181A73EB0102FFF679AF09E09B1BA24113D4CDE92232491B76
:200FC000B8410ED4CDE92410DDE92232981B72EB040006DBDDE92410B5EB010C77EB000C28
:200FE000E8DB4FF00008C4461DE000BFDDE922230C980799A0FB024601FB026100FB031082
:20100000CDE92240DDE926230C980799A0FB024601FB026100FB0310CDE92640012018EBD5
:2010200000084CF1000C0599B8EB0B007CEB0100DCDBDDE9261081F0010101430BD1DDE99F
:201040002410691A67EB00072898C0E90017002019B0BDE8F08F4FF0FF30F9E72DE9FF5F31
:201060009CB092462E990022CDE91122CDE9022213AA0A20CDE900029B460CAB0122491CE1
:2010800016F0D8F800287DD10CAF07AA395C0B0902F8103002EB400301F00F01401C59705F
:2010A0000828F3DB9DF82BC0DFF8408311460E2058F82C4000F10105235C645D801ECD5CD9
:2010C0000E5DCE540D55F3D5002002EB400312F810105B78914643EA01113954401C0828DD
:2010E000F3DB39460020139A0DE0141A0C440B5C14F8015D2E0146EA15150D541D0145EA63
:2011000013132370401CB0EB520FEED3082318A93846139AFFF73EFB0028B4D10CA90BF05A
:2011200025FE0028AFD10C210CA8FFF720FB00287DD0DDE90D01CDE90701082207A90020F1
:20114000141A0C440B5C14F8015D0D54401C2370B0EB520FF4D30020044607468046054665
:201160004FF00A0E19F800103A46303901EBC101B1FBFEF30EFB131101EB810103EB410CED
:20118000642300E0AAE0A2FB031704FB0373002602FB063411EB0C0774410A233246A8FBC9
:2011A000031605FB036308FB0232CDF84CC019F8003000F10100303B13EB010842EBE3757E
:2011C0000828CFDBDDE91821D01B61EB0401884A00232DF0A9FFCDE9182350EA01027DD0C5
:2011E0001AAA0692DDE90223CDE90423DDE91123CDE90232CDE90074DDE91C23FFF712FEB2
:2012000000286BD1DDE91A46A8FB040105FB0411DDE91C2308FB06112DF086FF1546DDE9A5
:2012200018129846A1FB040302FB043200E070E001FB0621DDE91C232DF076FF9146039379
:2012400055EA080202D1012000211DE0DDE92A01012414E0DDE92A23A0FB026701FB0271A3
:2012600000FB03113046BAEB00037BEB010205D252465B462DF058FF10461946641CE21726
:20128000661B72EB0802E5DBCDE91A0188460399044659EA010002D10120002121E0DDE901
:2012A0002C01012515E000BFDDE92C23A0FB026701FB027100FB03113046BAEB00037BEB0C
:2012C000010205D252465B462DF02EFF104619466D1CEE17039BB5EB090200E01CE09E416A
:2012E000E2DBA0FB045201FB042100FB081152465B4628462DF018FF10461946DDE91C2376
:201300002DF012FFDDE9180150405940084303D1012020B0BDE8F09F0020FAE7F0B5411E4E
:2013200085B01E2932D2012404FA00F111F0520F2CD0304FBE68401E2C4D8440083D696865
:201340000C4229D1C1B204912B49002301EBC001D1E90021CDE902212749284A303901EB0E
:20136000C001D1E90001CDE9000143F6E1001946FFF774FE0028286801D0204300E0A043AA
:201380002860B8681E49801B884202D3002005B0F0BD68682043686028682040F7E7411E5A
:2013A0001E290ED2012101FA00F212F0520F08D0401E81400D48083842688A4342600120CE
:2013C00070470020704700B501231846FFF7E7FF5B1C1E2BF9DD00BD30B5D0E90023D1E99E
:2013E0000045C0E90045C1E9002330BD0C00001000E1F50500000940C0120300BBF81A031B
:20140000404B4C0038B50446684603F061FD9DF80000204038BD38B50446684603F058FDA8
:20142000000602D5FA48006838BD9DF8000020438DF80000684603F042FD38BD38B50446A7
:20144000684603F045FD000602D5F148006838BD9DF80000A0438DF80000684603F02FFD6C
:2014600038BD01B5FEF7DCFE684603F048FDFEF7ECFE08BD7CB5684603F04BFDE44C000618
:2014800038D49DF800000025082809D009280DD0E048256005607846DF49086000207CBDB6
:2014A000684603F047FD000624D40BE001A804F0E9F900061ED49DF8040001281CD0132006
:2014C0008DF80000684603F01AFD000612D48DF8045001A804F0CCF900060BD48DF80450EA
:2014E00001A803F053FD000604D43E2013F086FF000603D520687CBD0220E1E701200DF095
:2015000067FB7CBD2DE9F0410024022029F0B9FEC24DAE68C24F4FF4FA7811E0A868801B4C
:20152000B8420DD3012024F0FBFEC821404624F02FF8012024F0FFFEAE68641C042C04DC21
:201540000020FEF7C3FE0028E8D1012C06D0022C07D0032C09D0042C0CD109E001F06CF879
:2015600008E0022020F04CFF04E002F0F1FA01E024F098FABDE8F041012029F082BE0EB5AB
:2015800068460BF06EFB50B1932803D1A1480068062801D00E2000E01120FFF762FF9C48DF
:2015A00000680EBD2DE9F34F002789B088460F703E4608A9384609F093FE954C000639D4C2
:2015C0009DF82000DFF84C92DFF84CA2400607D407A803F08DFC00062CD49DF81C0068B3BE
:2015E000694609980AF008FC000623D40125EB4605A9284603F070FF00061BD405EB850160
:201600005944491F052205A82EF05EF800B101276D1CEDB2042DEBD9C7B18249099808801B
:20162000402013F0EBFE000604D401200DF0D0FA00060BD520680BB0BDE8F08F2660794606
:20164000C9F800600020CAF80010F4E788F80070F4E72DE9F34F85B00320002408700E4631
:201660002746214601200BF04CFB0106684802D5006807B0E0E70168DFF89891DFF898A146
:201680000025052913D08046EB46694601200BF012FB0006D8F80000EBD405280DD005227F
:2016A0000BF1040005992EF00FF818B103E0357005600DE0671C641CE7E737B1BC4201D13B
:2016C000022000E00120307000E03570C8F800507946C9F800500020CAF80010C9E730B55B
:2016E000044685B00020208002200BF020FB484D05280BD0694602200BF0DDFA00061ED43B
:20170000BDF800002188884200D9208001200BF00EFB052802D06946012006E000200BF033
:2017200006FB05280BD0694600200BF0C4FA000605D4BDF800002188884200D92080286808
:2017400005B030BD2DE9F04387B00646694600200BF00CFB2E4D000649D403A90B2009F0DC
:20176000BFFD000643D40C2203A968462DF0ACFF0227DFF8A080DFF8A090002408B1377095
:201780003EE003A9102009F0ABFD00062FD4694604200BF0EBFA000629D4BDF80000BDF885
:2017A0000C108842EBD16946062009F099FD00061DD4BDF80000BDF80C10401E8142DED1D6
:2017C00069460E2009F08CFD000610D403A8FFF786FF00060BD4BDF80000BDF80C10884265
:2017E000CDD36946002009F07BFD000603D5286807B0BDE8F0839DF800004007BFD53470B8
:201800002C607946C8F800400020C9F80010EFE708C007200CC0072010C007200000094094
:20182000C0C62D0030C00720FEB502A803F071FBFC4C00063BD49DF808000025FA4EFB4F71
:201840001D2812D003F0FBFA08B103F08BFA01A803F0A6FB00062AD49DF8040028B101286C
:2018600009D002280BD0032811D025607846356038600020FEBD012006F010FE15E007F022
:2018800065FA000613D403202CF0E9FA11E08DF80050684603F0ECFF000608D43E2013F045
:2018A000ADFD000603D409F0E5FA000601D52068FEBD01200DF08CF9FEBD2DE9F0418AB0CB
:2018C000002606A80BF0CDF9DFF86083D54CD64D932804D12868082869D0062833D000219A
:2018E00008460BF00EFA000661D405A900200BF0D2FC00065BD4CE4F387858B10021012078
:201900000BF0FFF9000652D405A901200BF0C3FC00064CD409A804F0BDFA000647D49DF8E7
:20192000240028B3002101200BF0EBF900063ED4694601200BF0BFF905280DD00120397810
:2019400061B160B114E00020206079462860C8F800100AB0BDE8F0810020F0E740B193204E
:2019600020600820794628609320C8F80010F0E702200BF0DCF9000619D4694602200BF06D
:201980009AF9000613D4002102200BF0BAF900060DD405A902200BF07EFC2068932806D190
:2019A0002868082803D1761CB6B2032EF1D32068CFE72DE9F04F97B011A803F099FA994CA6
:2019C000000673D413A804F065FA0006F9D4DFF860A21026DFF854829AF80000924D4FF06D
:2019E00000094FF0160B9227C0B10AA809F0CFFB40F3C010401C8DF81C0011D09DF8390030
:201A0000010633D59DF84C1079B38DF8206008A803F075FA032027602860AEE18DF81C9091
:201A20009DF84C00D0B19AF80000B8B12868032811D004280FD08DF820B000BF9DF82000D9
:201A4000FFF70FFD2868092830D9412013F0D6FC30202760E0E78DF82060EFE7FFF7E4FE33
:201A600091E100BF8DF8200051E1FFE7C00603D509F000FA0006A4D4FFF71FFF4FF0020A0A
:201A8000932814D09DF8390000077AD50AF00CFB000696D4674828F0C0FF000691D407A971
:201AA0000DA8FFF7D6FD00286AD119E06AE1FFF7BBFE000685D40E208DF8200008A803F07D
:201AC0001EFA0006D7D400215BA029F012FA5F495F4881F800A0018841F002010180B4E1C1
:201AE0009DF81C00022804D0012872D0002871D0D4E19DF8390040076DD5684609F0D9FADD
:201B0000002869D103E000BFFFF7ABFCC4E109A904200BF02BF90006F8D4BDF82400BDF82A
:201B20000010401C81427CD19DF83900800609D5FFF77AFE0AF0B8FA0006E7D43D4828F07F
:201B40006CFF0FE015A803F02BFA0006DED49DF85400012816D0FFF767FE0006D6D411A8E2
:201B600003F0C6F90006D1D4BDF8000014A9FFF719FD20688228C9D092286DD093286CD1D0
:201B800024E166E10FA803F03EFA0006BED40FAEB01C03F049FA0006B8D4301D03F055FA9F
:201BA0000006B3D42B499DF84000087008A803F0B0F90006AAD49DF8200004280DD005281C
:201BC00054D01D282AD0FFF72FFE08A803F0A1F9C8E7ACE0B4E09FE0F5E003F030F930B122
:201BE00003F0C0F80FA804F01BFB00068ED40126002712A9304603F033FB000686D4129867
:201C0000761CF6B20744102EF3D93FB11D208DF8200008A803F073F900068ED40C4801880F
:201C20001CE028E008C007200CC0072010C00720FA020000F0CD07208E9888818A80208FFF
:201C4000808C9F9288208F840A0A000000C0072002C0072085C0072041E043E041F00401C2
:201C600001800FA804F0DCFA00068FD405F058F800068BD4A9E7FFF7D7FD000686D49DF800
:201C80003900400609D49DF8440030B1BDF82410BDF80000891C88420FD009F0EBF8000660
:201CA00070D414208DF8200008A803F028F9000668D4482013F0A2FBB4E0401E80B214A918
:201CC000FFF770FC206882285CD0922802D0932803D17BE02868082876D11320C2E628685C
:201CE000082871D19DF8500008B11520BAE608A803F00FF9000645D49DF820001D287DD0EE
:201D00009DF8440008B10120ACE68DF820A008A803F0F5F817B08FE48DF8206008A803F0C7
:201D2000EEF800062ED42F2013F068FBF2E78DF8206008A803F0E3F8000623D43C209CE0CF
:201D4000FFF772FD00061DD49DF839004FF0310610F0600F1DD09DF84C00A0B18DF820B000
:201D600008A803F0CCF800060CD43D2013F046FB01200CF02DFF27602E6079469220C8F8E6
:201D80000010C7E77FE09DF844000028BBD1022068E6684609F08DF9A8B914A8FFF7D2FC1B
:201DA000822879D092280FD093280FD09DF8500070B1022839D0882020607946C5F800A080
:201DC000C8F80010A6E7FFE70F209DE60E209BE60CF0D5FD01200CF0FBFE582013F00EFBF7
:201DE00009F0E1FD000657D4F74D0121F6480CF057FF00060CD5FEF713FA00E04EE009F0F5
:201E000039F8000648D4FEF720FA2068000643D409F0FBFD00063FD495F840000028E4D107
:201E200018200CE0000637D40FE09DF84C00002894D19DF8440008B1012000E002208DF8D6
:201E4000200008A803F05BF8ECE701200CF0C0FE60E7FFF7E9FC9DF84C0000289DF84400BA
:201E60000ED008B10C2000E00D208DF8200008A803F045F800060FD43B2013F0BFFAE4E742
:201E800010B1012001E007E002208DF8200008A803F035F8000601D520683BE7C4F800902F
:201EA0007946C5F800900020C8F8001032E7C74810B5007820B10420FFF730FA40B111E0CA
:201EC0000620FFF72BFA68B90420FFF727FA48B90120FFF723FA28B9322013F08FFA012050
:201EE0000CF076FEBA4900200860BA4908607846B9490860002010BD38B5684603F009F8D8
:201F0000B34C000629D4B54D2878752827D00220FFF778FA70B17B202870684603F000F812
:201F200000061AD41C208DF80000684602F0E7FF000612D40120FFF765FA80B151202870CA
:201F4000684602F0EDFF000607D417208DF80000684602F0D4FF000601D5206838BD9DF8F7
:201F600000000F2801D17E2028709A49002020600860784698490860002038BD2DE9FC41C8
:201F80008046032024F05AFE924E934F904C002530B9B8F1000F03D00420FFF733FA78B343
:201FA00001200CF015FE382013F028FA01200CF00FFE8A4975200870684602F0AAFF00061B
:201FC0001BD4684602F0BDFF000616D401A802F08FFF000611D49DF8040008B1192000E047
:201FE0001A208DF80000684602F089FF000604D40420FFF710FA000603D52068BDE8FC8170
:2020000006E0822020607846356038608220F5E725607846356038600020EFE72DE9F043A0
:202020008BB000273E4606A802F073FF684C00067ED49DF81800DFF89C81DFF89C910025D2
:20204000022803D0192801D01A2872D103A9352014F0F6FC00066BD49DF80E0000F00F010D
:20206000000900EB800001EB400000F5FA60ADF814009DF80D0000F00F01000900EB8000A2
:2020800001EB40008DF816009DF80C0000F00F01000900EB800001EB40008DF8170008A9EB
:2020A00005A8FEF794FC03A9362014F0C9FC00063ED49DF80E0000F00F01000900EB8000F4
:2020C00001EB400000F5FA60ADF814009DF80D0000F00F01000900EB800001EB40008DF805
:2020E00016009DF80C0000F00F01000900EB800001EB40008DF8170007A905A8FEF767FC38
:20210000684608F01FFA00065AD404A824F0D2FD000655D4BDF82000A0B1BDF80010814260
:2021200010D39DF8100017280CD2012703AB01E046E055E0352239460220039515F0C0F89B
:2021400000063DD4BDF81C0088B1BDF8001081420DD39DF8100050B1012603AB36223146AC
:202160000220039515F0ACF8000629D4C7BB56EA070041D009A9342014F062FC00061FD4BE
:202180009DF82400012816D0022804D0032833D112497D20087001200CF01AFD00060FD4BD
:2021A0000EB1432000E0422013F028F901200CF00FFD000604D404A824F07CFD000610D56C
:2021C00020680BB0BDE8F083B8020010FA02000008C007200CC0072010C0072084C007209A
:2021E0000AE09DF810000EB1401E00E0401C8DF8100004A824F0C7FD25607946C8F800508A
:202200000020C9F80010DCE738B50546684602F080FE2C4C000618D49DF80010062916D090
:2022200008DC012913D0032911D004290FD0052906D10CE007290AD0132908D0152906D071
:20224000284602F055FE000603D5206838BD012028701D4900202060086078461B490860BF
:20226000002038BD38B50546684602F063FE154C000619D49DF80010072917D007DC0729ED
:202280000DD2DFE801F00C130C13131313000E290CD013290AD0152908D01B2906D0284669
:2022A00002F026FE000603D5206838BD01202870054900202060086078460449086000200B
:2022C00038BD000008C007200CC0072010C007201FB5684628F0CCFEAE4C00062FD40220A7
:2022E000ADF80A00ADF80200ADF804000120ADF800000A20ADF806000021684628F0D9FC88
:2023000000061CD40021A4A028F0F3FD000616D40021A4A028F0EDFD000610D401210846A9
:2023200028F05FFC00060AD400219FA028F0E1FD000604D4012028F0C0FB000602D52068B9
:2023400004B010BD28F030FFFAE72DE9F0438146A5B00D46084628F0DCFB8E4C00066DD4BE
:20236000484628F074FC000668D4012028F002FC000663D42B464A4692A168462CF070FF24
:202380000021684628F0B5FD000657D493482A22C58968462946FEF729F80A200DF8050097
:2023A0000DF101014FF0000805F801804146684628F09FFD000641D428F0FFFF884F06461B
:2023C000BD680021874828F094FD000636D40021844828F08EFD000630D4002171A028F04B
:2023E00088FD28F0EAFF861BB8684FF47A71401BB0FBF1F506EB4600C0EBC61005EBC00014
:20240000401EB0FBF5F7A9F1010028F0D9FF4FF47A714E436843B6FBF0F2FF1DFB0872A10D
:2024200068462CF01DFF684628F0DFFE000605D4002175A028F05DFD000603D5206825B051
:20244000BDE8F0837149C4F800807846C1F800806F4908600020F2E770B50646012028F0B4
:202460002CFB4C4D00061BD4304628F0F0FB000616D40121084628F0B4FB000610D40820F5
:2024800028F078FB00060BD40424032E02D10D2C00D10E2421463046FFF757FF000601D55F
:2024A000286870BDE41C0F2CEFD35849002028600860784656490860002070BD10B50020BA
:2024C00028F0C5FB334C000635D400213CA028F010FD00062FD40121084628F082FB000660
:2024E00029D400214BA028F004FD000623D40221012028F076FB00061DD4002145A028F0DB
:20250000F8FC000617D40121022028F06AFB000611D400213FA028F0ECFC00060BD4022122
:20252000084628F05EFB000605D4002139A028F0E0FC000601D5206810BD344900202060C1
:202540000860784632490860002010BD10B5012028F0B3FA0F4C000614D40121084628F009
:2025600040FB00060ED41F4B1822A5336421002028F093FC000605D4002129A028F0B9FCDA
:20258000000601D5206810BDBDE81040012028F000BC000008C00720465072696E742D327F
:2025A000320000000A00000084A5ACAEADE1E2E0A0E6A8AEADADA0EF20AFA5E7A0E2EC0A74
:2025C000200A0000200A98908894922025752C209F908A8E91929C2025750A00F0CD07201D
:2025E0000000094090130300D1EAEEF0EEF1F2FC3A20257520D1D2D02FD12028257520CC31
:20260000CC2FD1290A0000000A200A000CC0072010C0072031323520544543540A000000AB
:20262000203420363032323432203030313733370A200A200A00000070B5B8B0022028F07F
:202640003CFAAD4D00067CD40221084628F0C9FA0006F8D4A9A2ACA102A82CF001FE002158
:2026600002A828F046FC0121084628F0BAFA0006E9D4A6A028F0B9FD012028F01EFA9FA2B1
:20268000A1A102A82CF0ECFD002102A828F031FC02A800F0D6FF02A800F012FD002102A856
:2026A00000F0D5FC002102A800F0C0FE02A800F0DDFF02A801F048F9202228A9984825F086
:2026C0007CF802AA95A197A000F073FC02A828F08CFD97A130A8289A2CF0C2FD02AA30A991
:2026E00095A000F066FC02A828F07FFD90A130A8299A2CF0B5FD02AA30A994A000F059FC7D
:2027000002A828F072FD8AA130A82A9A2CF0A8FD02AA30A992A000F04CFC02A828F065FDED
:2027200083A130A82C9A2CF09BFD02AA30A990A000F03FFC02A828F058FD7DA130A82D9A6F
:2027400000E0D0E02CF08CFD02AA30A98DA000F030FC02A828F049FD75A130A82E9A2CF09C
:202760007FFD02AA30A98CA000F023FC02A828F03CFD684627F001FE8BA130A8009A2CF0A4
:202780006FFD02AA30A98AA000F013FC02A828F02CFD02A800F0DFFC8AA028F026FD34A87E
:2027A00026F0BFF8349801282ED004282ED088A102AA89A000F0FDFB02A828F016FD8A4C9E
:2027C000202202A8E189FDF711FE0E2287A102A82DF070F836A90120CDE90001014627AB49
:2027E0000222092014F026FD00067CD49DF89C3001A80A22411E0A2B4FD2DFE803F04E0913
:202800000D4E14181C24284A7CA1D1E77DA1CFE7E18908447CA102E0E18908447CA10968DD
:20282000016002711DE0E18908447BA1F7E7E08908447BA102E0E08908447BA10A680260BF
:20284000898881800DE0E089084479A1F6E7E1890DF10200084478A10B6803608988818016
:20286000827102A828F0C1FC02AA75A176A000F0A0FB02A828F0B9FC27A81DF060FD9DF83E
:202880009C0070B101280FD0022802AA2ED023A10CE0E089084471A1D0E7E189084471A1A9
:2028A000BDE702AA71A101E002AA72A173A000F080FB02A828F099FC25F02BFF012028F0C9
:2028C00068FA4F2012F09AFD35A802F07AFB000609D435A802F0DFF8000604D435A802F014
:2028E00066FB000604D5286838B070BD68A1DDE701200CF06DF9F7E708C007204650726965
:202900006E742D323200000025730A00C8CDD4CED0CCC0D6C8DF20CE20CFC40A00000000E7
:2029200008000040CDC0D0C0C1CED2CAC00000002531306C7500000020C02DCED2D0C5C7D7
:20294000D72E2CC2D1C5C3CE0000000020C4C2C8C3C0D2C5CBDC2CC2D1C5C3CE0000000019
:2029600020C3CECBCEC2CAC02CC2D1C5C3CE000020C02DCED2D0C5C7D72E2CD1C1D0CED171
:202980000000000020C4C2C8C3C0D2C5CBDC2CD1C1D0CED10000000020C3CECBCEC2CAC045
:2029A0002CD1C1D0CED1000025326C7543000000D2C5CCCFC5D0C0D2D3D0C020C3CECBCE69
:2029C000C2CAC800D1C2DFC7DC20D120CFCA0A00556E6B6E6F776E0020CAC0CDC0CB20CEFA
:2029E000C1CCC5CDC0000000F0CD072020D1CACED0CED1D2DC20C1DBCBC0000052532D3223
:202A00003332000055534200313230300A000000323430300A000000393630300A000000F1
:202A200031343430300A000033383430300A000035373630300A00003131353230300A004B
:202A4000343830300000000020D1CACED0CED1D2DC20C2D0C5CCC5CDCDCE000031393230C8
:202A6000300A0000343830300A000000C0D2CECB00000000D8D2D0C8D500000020CFD0CE77
:202A8000D2CECACECB20CEC1CCC5CDC000000000C0D2CECB20CDCEC2DBC900002DE9F04FC5
:202AA00095B04FF0000ADFF88893DFF888B3CDF848A0E14FD9F80030CBF800303868DF49EB
:202AC000DFF88083CBF804007F25DD4C0988D8F800205646882B73D014DC052B08D008DC99
:202AE000002BFBD0012BF9D0032BF7D0042B67D129E1812BFCD0822B73D0862BF8D0872BF2
:202B0000F5D120E1912BF3D008DC892BF0D08A2BEED08F2B66D0902BE9D114E1922B34D089
:202B2000932B04D0962B7BD0A02BE0D1EDE00A2817D008DC052814D00628D9D0082810D0B9
:202B4000092806D10DE00B280BD0802810D081280ED00090BC4901A82CF082FB002101A8C2
:202B600042E011B90021B9A005E00426257005E00029FAD1BDA028F0BCF9F6E7C54902203B
:202B80000870462012F03AFCA8E0FDF749FB13A803F080F9FDF759FB9DF84C0000286ED0A9
:202BA0003868082826D00CDC082818D2DFE800F01722222222222222C9F80000386078E0E0
:202BC000AFE02A2813D006DC092813D020280ED0282804D10BE0302823D0312821D000214F
:202BE00001E024E073E0ACA028F083F9BEE70BF026FE19E00BF023FEA649CBF800A0022070
:202C0000CBF804A00870AB485446018841F00201018001200BF0DCFFC9F800403C6048E04E
:202C200097E00A2028F002FB7E202070A6E7BC46232876D2DFE800F08F1C1C2A2A248F12F7
:202C4000288F3531358F358F8F358F8F8F8F8F8F1C2A33338F358F8F3544440031B98D49A6
:202C600002200870002179A028F043F9042634E019B9002190A028F03CF902262DE02AE03F
:202C8000002196A028F035F9012626E019B900219BA028F02EF903261FE00A261DE0092679
:202CA0001BE0CBF800A0CBF804A0C9F800A0CCF800A07846C8F80000002015B0BDE8F08F03
:202CC00019B9002196A028F014F9082605E0032801D0072801D150466EE725709A4C9B4D48
:202CE000760012A9304600F071F800F03EF8287804EB001040688047287804EB0010806819
:202D0000804700202BF0F7FBEBE72BF02EF98007E1D5684602F049FA000603D5D9F80000DC
:202D2000CBE718E09DF800000028D4D1002188A028F0DFF85F48018841F002010180012049
:202D40000BF046FFC7E7CBF800A05046CBF804A032E70428BFD000903B4901A82CF080FAFE
:202D6000002101A828F0C5F8B7E738B56946012023F0B0FA2E4C000615D400982E49C3075A
:202D8000304A4FF0000010D02C4B1B889D0502D50121084603E01B0607D50121002007F07E
:202DA000FDFE000607D5206838BD2060086078461060002038BD4FF4FA74FA21204622F04A
:202DC000E7FB2146002022F0E3FBF6E770B5040008680D4605D0611E884210D14FF4FA6134
:202DE00011E01949184A36396C3A31F9101032F9100022F07EFB002818D11B240CE0C007F6
:202E000003D04FF4FA71002002E0C8214FF4167022F06FFB002809D1012023F097FA2868AA
:202E2000401C2860A04201D10020286070BD000008C0072014C007200CC007200000001038
:202E400084C0072010C00720BC1403008EE8A8A1AAA020AFA0ACEFE2A8208F84200A0A0A2F
:202E60000A0A0A0A0A0A0A0A0A0A000091A1AEA920AEA1ACA5ADA020E120AFA0ACEFE2EC7F
:202E8000EE208F84200A0A0A0A0A0A0A0A0A0A0A0A0A000000C007208EE8A8A1AAA0209DC2
:202EA0008A8B870A0A0A0A0A0A0A0A0A0A0A0A0A0000000002C0072091A1AEA920AEA1AC67
:202EC000A5ADA020E120454550524F4D0A0A0A0A0A0A0A0A0A0A0A0A0A0000008220E7A06C
:202EE000E1A0E520ADA5A2A5E0ADAEA520A2E0A5ACEF0A0A0A0A0A0A0A0A0A0A0A0A0A006F
:202F000091A1AEA920AEA1ACA5ADA020E1204652414D0A0A0A0A0A0A0A0A0A0A0A0A0A0052
:202F200091A1AEA920AEA1ACA5ADA020E12044415441464C4153480A0A0A0A0A0A0A0A0AF8
:202F40000A0A0A0A000000006C010010680100108EE8A8A1AAA02053440A00002DE9F04142
:202F6000804628F042F9002821D0FC4CFC4D4FF496764FF4FA77012023F0E8F93146384681
:202F800022F006FB012023F0E1F9A068A168091AA942FBD328F008F90028ECD10021F1A073
:202FA00027F0A7FF4046BDE8F04128F01EB9BDE8F0812DE9F05F8B46144682462CF0D4FBB0
:202FC000814658462CF0D0FBE74D064609EB0600E9890A274FF00008884217D220222046E6
:202FE000FDF704FA4A46514620462CF0DCFBE8893246801B204459462CF0D5FBE889275400
:20300000E989641C01F80480BDE8F09F012000EB410120222046FDF7E9F94A4651462046B4
:203020002CF0C1FBE889324659462754E889C6EB40002044401C2CF0B6FBE88904EB400026
:203040004770E98904EB410181F80280DCE730B585B005460C4604A822F03CFBFDF7E0F8E0
:203060000499642091FBF0F200FB12100A2190FBF1F3BEA168462CF0F3F82A466946BEA079
:20308000FFF797FF2846FFF769FFFDF7DEF83CB1C0A1684622682CF0E3F82A46694607E08B
:2030A000BF482A460068000601D5BEA100E0BFA1B0A0FFF77EFF2846FFF750FF05B030BD9E
:2030C00070B5044688B0012027F0F7FCA64E01252846FEF764F9002838D02A46B5A12046E8
:2030E0002CF0BEF82046FFF739FFF18920222046FDF77CF907A91420CDE9000102AB012274
:2031000029460A2014F096F82846FEF707F950B1079A611C530002A8FDF769FCF189201FF3
:203120000844A8A109E0079858224100601CFDF75DF9F189A01F0844A4A12CF091F8F28907
:20314000601C002111542046FFF708FF6D1C1E2DBEDB08B070BD10B5044686B0012027F03B
:20316000ACFC9CA0FFF7FAFE9D489EA1028868462CF076F8224669469CA0FFF71AFF2046CF
:20318000FFF7ECFE03A904A80AF060F8BDF80C2094A168462CF064F82246694694A0FFF728
:2031A00008FF2046FFF7DAFE06B010BD70B5064686B00C46032023F041FDA8B100218DF8E5
:2031C00000108DF801108DF8021040F2DA70ADF8140001208DF816008DF8170005A823F065
:2031E000F4FD684623F0CFFD684623F063FD5B499DF8025088687F4A8B681B1A9342FBD321
:20320000684623F057FD9DF8020064B1A84202D12068401C20605FA101A822682CF020F865
:20322000324601A905E0A842324601D05FA100E05CA171A0FFF7BDFE3046FFF78FFE06B006
:2032400070BD30B50C006FA187B00546D1E90001CDE900010DD023F0E3FD10B12068401CD7
:2032600020604CA102A822682BF0FAFF2A4602A906E023F0D5FD2A4608B14AA100E04BA1D3
:203280006846FFF796FE2846FFF768FE07B030BD30B55EA305460C460FCB89B08DE80F006E
:2032A00008A9084609F0D2FF5C480068C8B105282A461ED05AA16846FFF77BFE64B1206880
:2032C000401C206033A104A822682BF0C9FF2A4604A96846FFF76DFE2846FFF73FFE09B09F
:2032E00030BD2A4631A16846FFF763FE002CE9D1F2E72CA16846FFF75CFE002CECD021689F
:20330000491C2160DEE77FB505460C4614F030F878B142482A460068012808D021A141A0D6
:20332000FFF747FEACB12068401C206007E03CA1F5E72A461DA13BA0FFF73BFE4CB115A106
:20334000684622682BF08CFF2A46694635A0FFF730FE2846FFF702FE7FBD0000000009408E
:2033600020A107000A000000F0CD072025752E25303175C200000000C1C0D2C0D0C5DF206B
:20338000D7C0D1CEC228322E32202D20332E3329000000002530346420CED8C8C1CECA007D
:2033A00008C00720CDC5CDCED0CC0000CDCED0CC00000000CACEC420C7C0D9C8D2DB202588
:2033C000750A0000CDCED0CC0A000000CDC5CDCED0CC0A00494420D1C5D0C8C83A0A000073
:2033E0000404000025303475000000002031000020320000E0C81000D5CEC420D7C0D1CEAF
:20340000C2000000CFCE20CFC4000000CFCE20CFC0CCDFD2C820CFC4000000000CC0072063
:20342000CDC5D200454550524F4D00007FB505460C4608F020FFA0B1F748016822290CD058
:2034400021290AD02A46AFF2A401F4A0FFF7B1FDCCB12068401C20600AE02A46AFF240013D
:20346000F3E72A46AFF2BC01ECA0FFF7A2FD54B1AFF2E001684622682BF0F2FE2A4669469A
:20348000E6A0FFF796FD2846FFF768FD64E77FB505460C4602F058FC000607D42A46AFF200
:2034A000F401E1A0FFF785FD74B918E0DA482A460068192817D0AFF29801DBA0FFF779FDB6
:2034C0006CB12068401C2060AFF23811684622682BF0C6FE2A466946D3A0FFF76AFD28460D
:2034E000FFF73CFD38E7AFF24411E6E72DE9F0438146CFA00C46D0E9001289B080680026D8
:20350000CDE902200191012027F0D7FA0021084609F0F7FB0027C04D12E02868082815D112
:2035200017B9C6A0FFF71AFDBDF80020CAA1521C48462BF095FE4846FFF710FD7F1C01260B
:203540006946002009F0A7FE0028E6D1DFF81083D8F80000932800D101260021012009F0F7
:20356000D0FB002712E02868082815D117B9BDA0FFF7F4FCBDF80020B7A1521C48462BF06A
:203580006FFE4846FFF7EAFC7F1C01266946012009F081FE0028E6D1D8F80000932800D10F
:2035A00001260021022009F0ACFB002712E02868082815D117B9B2A0FFF7D0FCBDF8002089
:2035C000A5A1521C48462BF04BFE4846FFF7C6FC7F1C01266946022009F05DFE0028E6D139
:2035E000D8F8000093280BD09EB14A46AFF24C2101A8FFF7DEFCF4B12068401C20600FE007
:203600002868802801D08128EFD14A46AFF2F011EEE74A46AFF26C2101A8FFF7CAFC54B109
:20362000AFF2902104A822682BF01AFE4A4604A901A8FFF7BEFC4846FFF790FC09B0BDE8CB
:20364000F0833EB5044623F00EFD00F00F03C0F3031291A168462BF003FE2246694690A08F
:20366000FFF7A7FC2046FFF779FC3EBD10B58CB0044618228FA105A82CF01CF90BA802F0AD
:2036800009FC9DF82C0008B190A101E0AFF27021224605A8FFF78DFC2046FFF75FFC9DF887
:2036A0002C00002879D06946002009F0A2FA002873D1BDF8002086A1521E01A82BF0D0FDA0
:2036C000224601A984A0FFF774FC2046FFF746FCBDF800007EA1C0F1190201A82BF0C0FD8F
:2036E000224601A981A0FFF764FC2046FFF736FC6946022009F07DFA00284ED1BDF8002056
:20370000AFF2203101A82BF0ABFD224601A97AA0FFF74FFC2046FFF721FC04A9022009F09D
:2037200039FA002839D1BDF81000BDF80010421AAFF2503101A82BF093FD224601A96BA0AB
:20374000FFF737FC2046FFF709FC6D480078002823D06946012009F04CFA00281DD1BDF8BD
:2037600000205BA101A82BF07BFD224601A965A0FFF71FFC2046FFF7F1FBBDF8000054A1D7
:20378000C0F1400201A82BF06BFD224601A957A0FFF70FFC2046FFF7E1FB0CB010BDF0B59A
:2037A000074693B00C460025032007F031FE2C4E000602D5306813B0F0BD07F03EFE000621
:2037C00005D411A9052007F08BFD00060AD514B12068401C206001253F220A216846FCF751
:2037E00005FE05E00A230522694611A8FDF7FFF800208DF80A006A4647A104A82BF030FDFF
:2038000044B1AFF270410DA822682BF029FD3A460DA98EE086E000000CC0072044415441CA
:20382000464C4153480000004652414D00000000CFE0ECFFF2FC20CFC4000000CFCEC2D08A
:20384000C5C6C4C5CDCDDBC520D4C8D1CAC0CBC8C7C0D6C8C83A0A0023253034750A000014
:2038600008C00720CFCEC2D0C5C6C4C5CDCDDBC520C0CAD2C8C2C8C7C0D6C8C83A0A0000DD
:20388000CFCEC2D0C5C6C4C5CDCDDBC520D1CCC5CDDB3A0A0000000025752E2575000000DB
:2038A000DDCBC5CAD2D0CECDCDDBC920C1CBCECA00000000CFC0CCDFD2DC20CFC420C0CA9A
:2038C000D2C8C2C8C7C8D02E00000000C4C00000253032750000000020CFC5D0C5D0C5C316
:2038E000C8D1D2D0C0D6C8C9000000002020D1C2CEC1CEC4CDCE000020D1CCC5CD00000088
:20390000FA02000020C0CAD2C8C2C8C7C0D6C8C920DDCACBC7000000DDCACBC7202825737D
:203920002900000015B1AFF2845101E0AFF284513A4604A8FFF73DFBFCF772FC3846FFF79C
:203940000DFBFCF782FC35E770B5064688B0032007F05EFDFD4C000660D407F06EFD68B1B6
:20396000FCF75EFC3246AFF24851F9A0FFF721FB3046FFF7F3FAFCF768FC4FE005A90520EB
:2039800007F0AEFC000649D40A230522694605A8FDF72DF800258DF80A5032466946ECA0E3
:2039A000FFF707FB3046FFF7D9FA04A9002007F097FC9DF81000000702D5AFF2F00101E083
:2039C000AFF2A4513246E4A0FFF7F3FA3046FFF7C5FA9DF81000400702D5AFF2101101E0E1
:2039E000AFF2C4513246E0A0FFF7E3FA3046FFF7B5FA9DF81000000602D5AFF2301101E0E6
:203A0000AFF2E4513246DCA0FFF7D3FA3046FFF7A5FA684608F02AFB000602D5206808B026
:203A200070BD32466946DAA0FFF7C3FA3046FFF795FAD948256005607846D8490860002098
:203A4000EDE770B5D64C0546B222E189FCF7CEFCE1890A2068540321D2A027F094FC002454
:203A60000021284627F045FA641C0A2CF8D327F09BFBBDE87040082027F07CB81FB504464D
:203A80002AF0E8F8C84B99684EF660209A68521A8242FBD32AF08FF9002851D02AF0A6F9B0
:203AA0000028224650D0AFF2FC61C0A0FFF781FA2046FFF753FA68462BF0A7FA224669465D
:203AC000BDA0FFF776FA2046FFF748FA68462BF0B3FA22466946BAA0FFF76BFA2046FFF7E7
:203AE0003DFA68462BF0CCFA22466946B7A0FFF760FA2046FFF732FA68462BF0F3F922469D
:203B00006946B4A0FFF755FA2046FFF727FA082027F08CFB2246B3A18EA000BFFFF749FA38
:203B20002046FFF71BFA2AF0D9F88849002008609949086078469949086004B0002010BDDD
:203B40002246AFF2247101E0AFF2A87197A0E5E72DE9F043C3B0002439943A943B943C940F
:203B60003D943E943F94409434A8419427F080FA764D000618D43020ADF8DE000220ADF86A
:203B8000DA000120ADF8D200ADF8D400ADF8D0000820ADF8D600A046ADF8DC40002134A87E
:203BA00027F087F8000602D5286843B047E5022027F067FB8DA0FFF7D1F9012026F07DFFA8
:203BC00091A0FFF7CBF9DFF85C9299F8000018B195A0FFF7C3F915E0082027F027FB00247A
:203BE000002194A027F085F930B9012027F0E8FA10B927F0D9FA08B1FEF750FF641CA4B252
:203C00000A2CEDD3012026F058FF8BA0FFF7A6F9082027F00BFB904F00260020FCF756FBB2
:203C200010F0FF0F37D0022026F047FF7EA0FFF795F9012026F041FF27F057FB3888002887
:203C4000FAD1594CA068854DA168091AA942FBD383A0FFF783F9012026F02FFF28A809F072
:203C600000F820B13F220C2128A8FCF7BFFB8DF8AC802022052128A8FCF7B8FB03AA28A963
:203C80007CA0FFF796F903A8FFF768F931A823F046F870B909E027F028FB38880643B6B29A
:203CA0007007BAD5B007B8D5C6E732A823F002F820B171A103A82BF033FD12E0BDF8C420C2
:203CC0009DF8C9009DF8C810A2F5FA620092CDE901109DF8C6309DF8C7206CA103A82BF0F3
:203CE000BFFA032026F0E9FE03A8FFF737F9012026F0E3FE03A8FFF7E3F96BA26DA103A8BF
:203D00002BF0AEFA002103A827F0F3F803A8FFF798FC69A0FFF722F927F0E7FA388899F87A
:203D2000001000F01000084303AA0DD0AFF68C1164A0FFF73EF903A8FFF710F9B00703AA1D
:203D400003D5AFF69811CCE0C6E0C8E008C00720DDCACBC70000000020C0CAD2C8C2C8C786
:203D6000C8D0CEC2C0CDC00020C0D0D5C8C220CED2CAD0DBD200000020CDC5C8D1CFD0C00E
:203D8000C2C8CCC0DF20CED8C8C1CAC00000000020C2C5D0D1C8DF000CC0072010C007207C
:203DA000F0CD07201B3300000000094053442DCAC0D0D2C00000000020CEC1DAC5CC0000BE
:203DC00020D1C2CEC1CEC4CDCE00000020C7C0CDDFD2CE0020CACECB2DC2CE20D4C0C9CBF9
:203DE000CEC20000CFD0CEC9C4C5CD003D20D2C5D5CDCECBCEC3C8D7C5D1CAC8C920CFD098
:203E0000CEC3CECD203D0A00D2C5D1D220CDCEC6C020C0C2D2CECED2D0C5C7D7C8CAC00A23
:203E200000000000D1C10720CFD0CECFD3D9C5CD0A0000000A0A0A00D2C5D1D220C4C0D277
:203E4000D7C8CACEC220CAD0DBD8CAC820C820C1D3CCC0C3C80A00002802001020A10700AB
:203E60003D3D3D2020CFD0CEC3CECD203120203D3D3D0A00CFC4000058582D58582D585831
:203E800058582058583A58580A000000253032752D253032752D2530327520253032753A0A
:203EA000253032750A000000465072696E742D323200000025730A00C4C0D2D7C8CAC80AE5
:203EC0000000000020CDCEC620C0C2D2CECED2D0C5C7D7C8CAC00000AFF6303128E7AFF640
:203EE0003C31FAA0FFF765F803A8FFF737F8700703AA02D5AFF64C3101E0AFF65831F5A0D7
:203F0000FFF757F803A8FFF729F8F4A0FFF726F8002024F080FD012024F07DFD38B902207F
:203F200024F079FD18B103AAAFF6803102E003AAAFF69031EDA0FFF73CF803A8FFF70EF8D8
:203F4000EDA0FFF70BF8082027F070F90020FCF7BDF9C7B2012024F05EFD28B1022024F052
:203F60005AFD08B1012600E000263743EED0032026F0A3FD0EB1E3A000E0E5A0FEF7EEFF6A
:203F8000012026F09AFD032024F045FD0020FCF79DF90028FAD1E1A0FEF7E0FF002024F0B5
:203FA00092FE012024F08FFE38B9022024F08BFE18B103AAAFF60C4102E003AAAFF61C4106
:203FC000CAA0FEF7F6FF03A8FEF7C8FFCAA0FEF7C5FF082027F02AF90020FCF777F9C7B2A5
:203FE000012024F070FE28B1022024F06CFE08B1012600E000263743EED0032026F05DFDF4
:204000000EB1C0A000E0C2A0FEF7A8FF012026F054FD032024F057FEA068A168091AA94270
:20402000FBD30020FCF752F90028FAD1002103A8FFF7BCF8002103A8FFF709F8002103A85C
:20404000FFF7FFF8002103A8FFF722F9002103A8FFF71DFA002103A8FFF755F9002103A8E1
:20406000FFF7E4F9002103A8FFF740FA03A8FFF7FDFA002103A8FFF792FB47462FA91320F2
:20408000CDF8BC8012F0A7FD08B164202F90A7A128A82F9A2BF0E4F803AA28A9A4A0FEF7EE
:2040A00088FF03A8FEF75AFF03A8FFF7CAFC012026F003FDA1A0FEF751FF082027F0B6F86F
:2040C000A6680020FCF702F900B1A668A068801BA842F6D303AAAFF62C519AA0FEF769FF49
:2040E00003A8FEF73BFF9AA0FEF738FF082027F09DF8A6680020FCF7E9F800B9A668A068DB
:20410000801BA842F6D3032026F0D7FCAFF64C50FEF724FF012026F0D0FC0020FCF7D6F808
:204120000028FAD18DA0FEF719FF082027F07EF88D4E07E0032022F009F9A068A168091A70
:20414000B142FBD30020FCF7C1F80028F2D003AAAFF2703164A0FEF72CFF03A8FEF7FEFE39
:20416000032022F0E8F8022022F0DAF87FA0FEF7F5FE082027F05AF84FF4FA76C82130467A
:2041800021F006FAA168A268521AAA42FBD30020FCF79CF80028F1D003AAAFF2B83152A01C
:2041A000FEF707FF03A8FEF7D9FE0020FCF78EF80028FAD1012026F080FC6FA0FEF7CEFE7E
:2041C000032026F07AFC27F090F8714D2888400702D4AFF6106001E0AFF61060FEF7BEFE4A
:2041E000012026F06AFC6BA0FEF7B8FE082027F01DF86B4E26F0A3FBA068A168091AB14284
:20420000FBD30020FCF762F80028F3D0022026F054FC64A0FEF7A2FE012026F04EFC64A0D2
:20422000FEF79CFE082027F001F827F05EF8032026F043FC2888400702D5AFF6786001E0A6
:20424000AFF67860FEF78AFE03A8FFF717FC03A8FEF781FF26F0A8FFB8463D46ADF8CC7071
:2042600033A9392012F0B7FCADF8B4502DA93A2012F0B1FCBDF8B420AFF6986128A82AF0BB
:20428000EFFF03AA28A94DA0FEF793FE03A8FEF765FEBDF8CC204DA128A82AF0E1FF03AA36
:2042A00028A94DA0FEF785FE03A8FEF757FE4E2011F0A4F838A800F084FE38A800F0EBFBC0
:2042C00038A800F074FE0126464D22E120CAD0DBD8CAC80020C1D3CCC0C3C800525332330B
:2042E000322D310A200A200A0000000020D0C0C7CCDBCAC0CDC8C50020C7C0CCDBCAC0CD29
:20430000C8C5000020CDCED0CC0A0A0A0000000020CDC5CDCED0CC0A0A0A0000525332338A
:20432000322D320A200A200A0000000025750000DFD0CACED1D2DC20D7CB0000CACDCECF38
:20434000CAC00A00D0C0C7CCDBCAC0CDC8C50000C7C0CCDBCAC0CDC8C50A0A00C8CDC4C8A0
:20436000CAC0D2CED0DB0000400D0300C4C8CDC0CCC8CA0A00000000C4C5CDC5C6CDDBC945
:2043800020DFD9C8CA0A20C7C0CAD0DBD20A000026020010D2C5D1D220C7C0CCCAC00A0038
:2043A00000350C00CFD0CEC9C4C5CD0A0000000020CED2CAD0DBD20A00000000D7C8D1CBDA
:2043C000CE20D6C8CACBCEC2000000002530347520D1C5CA00000000C7C0C4C5D0C6CAC07E
:2043E0000000000002C00720288840F00200288001200AF0EDFB012026F05FFBBDF8B4301D
:20440000324658A103A82AF02BFF03A8FEF7A6FD31A822F084FC18B932A822F04BFC28B1B1
:20442000AFF2AC5103A82BF07BF913E0BDF8C4209DF8C9009DF8C810A2F5FA620092CDE912
:2044400001109DF8C6309DF8C720AFF2C05103A82AF006FF032026F030FB03A8FEF77EFD49
:20446000012026F02AFB4448B222C78903A83946FBF7BCFF03A90A20C855491C07F8018081
:204480000321AFF2E06026F07EFFCDF8BC80002103A826F02EFD2F98401C2F900A28F6D399
:2044A000082026F067FB39A903A8FEF77FFE3AA903A8FEF7CCFD3BA903A8FEF7C2FE3CA9E8
:2044C00003A8FEF7E5FE3EA903A8FEF7E0FF3FA903A8FEF718FF40A903A8FEF7A7FF3DA93F
:2044E00003A8FFF703F841A903A8FFF758F9A76803E00020FBF7EAFE80B9A06843F6095283
:20450000C11BBDF8CC005043B1EB801FF1D3761CB6B2BDF8B40086427FF666AF4F2010F088
:204520006DFF38A800F04DFD38A800F0B4FA38A800F03DFD288840F00200288001200AF0C8
:2045400047FB0EA0FEF70AFD032026F0B6FA14A0FEF704FD288840F00200288001200AF037
:2045600037FBFEE7D6C8CACB202530347520C8C720253034750A0000F0CD07203DD2C5D56F
:20458000CDCECBCEC3C8D7C5D1CAC8C920D2C5D1D220C7C0C2C5D0D8C5CD3D0A0A0A0A006D
:2045A00028CFCEC4CFC8D1DC290A0A00F0B50479002364F3070302680C68A21843F100017E
:2045C000FD4C0B0AFD4EFE4F04D1FE4DE823AD1A8B4107D28920206001203060784638601E
:2045E0008920F0BD02600171002020603060784638600020F0BDF0B50C68002309791A4620
:2046000061F3070201680579611865F307035A41E94CEA4EEA4F130A04D1EA4DE8236D1A7F
:20462000934107D28920206001203060784638608920F0BD01600271002020603060784685
:2046400038600020F0BDF0B502680C680023A218D94CDA4DDA4F53EB030104D1D94EE823D7
:20466000B61A8B4107D28920206001202860784638608920F0BD02600020206028607846FF
:2046800038600020F0BDF0B502680C680023A218C94CCA4DCA4F53EB030104D1CA4E0223BC
:2046A000B61A8B4107D28920206001202860784638608920F0BD02600020206028607846BF
:2046C00038600020F0BD30B502680D68BA49BB4BBB4CAA4207D28920086002201860784673
:2046E0002060892030BD521B026000200860186078462060002030BDF0B502680C680023E4
:20470000A218AD4CAD4DAE4F53EB030104D1AE4E0223B61A8B4107D2892020600120286070
:20472000784638608920F0BD0260002020602860784638600020F0BD30B502680D689E4975
:204740009E4B9F4CAA4207D2892008600220186078462060892030BD521B026000200860EA
:20476000186078462060002030BD10B502880988924B1144904A924CB1F5803F07D38920C4
:2047800010600120186078462060892010BD018000201060186078462060002010BD002187
:2047A0000160017184480160844801607846844908600020704700210160818081717E48C7
:2047C00001607E48016078467D490860002070477CB50023CDE90033036800938388ADF8A3
:2047E000043080798DF8060000231360DDE900450868041B73EB050101D2581E06E0DDE978
:204800000051281A71F1000101D2012010606A4803606A48036078466949086000207CBDE3
:204820002DE9FC410022CDE90022026800928288ADF8042082798DF80620DDE900340A684A
:20484000D21844F10001CDE900210C0E5A495B4A5B4B06D1DDE900565C4F5D4C7D1BB44185
:2048600008D28920086001201060784618608920BDE8FC81009C0460BDF8044084809DF829
:2048800006408471002008601060784618600020EEE72DE9FC410022CDE900220268009271
:2048A0008288ADF8042082798DF80620DDE900620968414B414C424F761A72F1000207D26E
:2048C0008920186001202060784638608920CFE7DDE90062711A62F10002CDE90012016030
:2048E000BDF8041081809DF806108171002018602060784638600020BAE72DE9FC410022AD
:20490000CDE900220B68097961F30702016800918188ADF8041081798DF80610DDE9001442
:204920005B186241CDE90032140E2349234A244B06D1DDE90056254F254C7D1BB44107D2D1
:2049400089200860012010607846186089208FE7009C0460BDF8044084809DF80640847193
:2049600000200860106078461860002080E72DE9F0410446006809680022A1FB005602FB07
:20498000006001FB02014FF4FA70281841F100014FF47A7200232AF0C7FB074B074D084F6D
:2049A00021B9094E0222361A8A4117D2892018600320286078460DE008C007200CC0072045
:2049C00010C00720FF0FA5D4FFE30B54FFFF63A7B3B6E00D38608920BDE8F08120600020C3
:2049E00018602860784638600020F5E72DE9F0410446006809880022A1FB005602FB00606A
:204A000001FB020141F28830281841F1000142F2107200232AF088FB304B314D314F21B970
:204A2000314E0222361A8A4107D28920186003202860784638608920CEE720600020186047
:204A40002860784638600020C6E7018842F20F73491C8AB2002102809A4200D901801F488B
:204A600001601F48016078461E49086000207047018842F20F72491E89B20180914200D99C
:204A8000028016490020086015490860784615490860002070470268144B521C00210260D2
:204AA0009A4200D901600D4801600D48016078460C4908600020704701680C4A491E01609B
:204AC000914200D902600549002008600449086078460449086000207047000008C0072004
:204AE0000CC0072010C00720FFE30B54FFE0F5052DE9FC4111F0E4FB454C00067DD401F0A6
:204B0000A5FD444E444F454D4FF0000868B1012820D0872873D0684600F0B4FE00066CD43B
:204B20009DF800000E285FD067E0684600F0AAFE000662D401A800F0CCFE00065DD49DF883
:204B400000000E285BD1BDF80400402857D17120287054E0684600F095FE00064DD49DF860
:204B600000001B282CD2DFE800F02B0E2727272713131313131313130E11111111110E2936
:204B80002929292B11001DF0C7FD03E0202000E06020287001F0DAFD00062ED49DF800000D
:204BA0000E2816D001200AF013F8000625D49DF80000172810D022E05020EAE73020E8E79E
:204BC0008820206009203060784638608820BDE8FC810AF0A1F8E8E71148007878B11DF06B
:204BE000FFFD000609D40AE0FBF71AFB1DF094FDFBF72BFB01F0AAFD00062068E7E7C4F87F
:204C000000807846C6F8008038600020DFE7000008C007200CC0072010C0072084C0072056
:204C200024C007202DE9F843904D8F48904E2978904F914C4FF088084FF00A0959B90122D3
:204C4000694622F0BAFD000602D52068BDE8F8839DF8000038B1C4F800807846C6F8009091
:204C600038608820F2E70120287040F6CA506860002020603060784638600020E6E738B5EA
:204C8000002479488DF800400122694622F0A0FD0106794801D5006838BD74490C70046051
:204CA00073480460784673490860002038BD2DE9F74F6E4A6E4E6F4F13786F4D92B04FF088
:204CC000880CA3B15368149C4FF0000A03EB040808F10508B8F5005F0ED3C5F800C0C6F810
:204CE00000A078463860882015B0BDE8F08F0A20C5F800C03060F4E7ADF8400080B293462B
:204D00005B1CADF8000043F080482246E9460DF102002AF048FD09EB0400D146847080F80B
:204D200003A0221D6946404622F052FD00060AD4DBF804005C4640F08040012214A922F0BC
:204D400047FD000601D52868CEE7606814990844001D6060C5F800907846C6F8009038605F
:204D60000020C1E72DE9F04F434D414F3E4CD5F80080DFF800A1D7F8009097B000264FF498
:204D8000005B012201A9204622F017FD00064BD49DF80400F0B30444241D24F06041594522
:204DA00001D2402809D988202860012038607846CAF80000882017B097E7761CE1E7641EA4
:204DC000012201A9204622F0F8FC00062CD49DF804000222241AA41E15A9204622F0EDFCB8
:204DE000000621D4A41C9DF8042002A9204622F0E4FC000618D4BDF854009DF8042040F058
:204E0000804002A922F0E4FC00060DD49DF80400211800E002E00C1AE41E761E002ECED131
:204E2000FFF72DFF000601D52868C4E7C5F800807946C7F800904046CAF80010BBE738B507
:204E40000A4C0948217809B1012038BD0122694622F0B3FC08B1002038BD9DF8000008B193
:204E600001202070207838BDCA0D00401CC007200CC0072010C0072008C007202DE9F041BA
:204E80008046FC4815460F4600781E4680B11A46404622F092FCF84C000606D432463946AA
:204EA0004046FFF704FF000602D52068BDE8F081324629464046BDE8F04122F089BC38B571
:204EC000EE4C0246012369462046FFF7D7FF38BDEA4B01460122184622F06FBC38B5E74CFC
:204EE0000246641C012369462046FFF7C7FF38BDE24B01465B1C0122184622F05EBC38B57B
:204F0000DE4C0246A41C012369462046FFF7B6FF38BDDA4B01469B1C0122184622F04DBCC7
:204F200038B5D64C0246E41C012369462046FFF7A5FF38BDD14B0146DB1C0122184622F065
:204F40003CBC38B5CD4C0246241D012369462046FFF794FF38BDC94B01461B1D01221846FF
:204F600022F02BBC1CB5C0EBC00026300A4640F0804007236946FFF781FF1CBDC0EBC000D3
:204F8000263040F08040072222F017BC38B5BB4C02464B34012369462046FFF76FFF38BD70
:204FA000B64B01464B330122184622F006BC38B5B24C02464C34042369462046FFF75EFF94
:204FC00038BDAE4B01464C330422184622F0F5BB38B5AA4C02465034022369462046FFF7F8
:204FE0004DFF38BDA54B014650330222184622F0E4BB38B5A14C02465234022369462046A1
:20500000FFF73CFF38BD9D4B014652330222184622F0D3BB38B5994C02465434022369461E
:205020002046FFF72BFF38BD944B014654330222184622F0C2BB38B5904C02465634012378
:2050400069462046FFF71AFF38BD8C4B014656330122184622F0B1BB38B5884C02465734FD
:20506000042369462046FFF709FF38BD834B014657330422184622F0A0BB7F2208B502EB26
:2050800080000A4640F0804004236946FFF7F6FE08BD7F2202EB800040F08040042222F095
:2050A0008CBB38B5754C02468334042369462046FFF7E4FE38BD714B0146833304221846B6
:2050C00022F07BBB38B56D4C02468734022369462046FFF7D3FE38BD684B01468733022211
:2050E000184622F06ABB38B5644C02468934042369462046FFF7C2FE38BD604B01468933E4
:205100000422184622F059BB38B55C4C02468D34022369462046FFF7B1FE38BD574B01468A
:205120008D330222184622F048BB38B5534C02468F34012369462046FFF7A0FE38BD4F4B25
:2051400001468F330122184622F037BB38B54B4C02469034042369462046FFF78FFE38BD7D
:2051600038B5464C02469434042369462046FFF785FE38BD38B5414C024698340423694692
:205180002046FFF77BFE38BD3C4B014698330422184622F012BB38B5384C02469C3401239C
:2051A00069462046FFF76AFE38BD344B01469C330122184622F001BB38B5304C02469D3421
:2051C000042369462046FFF759FE38BD2B4B01469D330422184622F0F0BA38B5274C0246DC
:2051E000A134022369462046FFF748FE38BD234B0146A1330222184622F0DFBA38B51F4C61
:205200000246A334022369462046FFF737FE38BD1A4B0146A3330222184622F0CEBAC9228C
:2052200008B502EB80000A4640F0804004236946FFF724FE08BDC92202EB800040F0804009
:20524000042222F0BABA40F2091208B502EB80000A4640F0804004236946FFF70FFE08BD4D
:2052600040F2091202EB800040F08040042222F0A4BA00001CC0072008C007202800004094
:2052800038B5F94C0246042369462046FFF7F6FD38BDF54B01460422184622F08EBA38B528
:2052A000F14C0246241D042369462046FFF7E6FD38BDED4B01461B1D0422184622F07DBA9A
:2052C00038B5E94C02460834012369462046FFF7D5FD38BDE44B014608330122184622F0EE
:2052E0006CBA38B5E04C02460934042369462046FFF7C4FD38BDDC4B0146093304221846D4
:2053000022F05BBA38B5D84C02460D34042369462046FFF7B3FD38BDD34B01460D3304222A
:20532000184622F04ABA38B5CF4C02461134042369462046FFF7A2FD38BDCB4B01461133FD
:205340000422184622F039BA38B5C74C02461534012369462046FFF791FD38BDC24B01462D
:2053600015330122184622F028BA38B5BE4C02461634022369462046FFF780FD38BDBA4B40
:20538000014616330222184622F017BA38B5B64C02461834042369462046FFF76FFD38BD02
:2053A000B14B014618330422184622F006BA38B5AD4C02461C34012369462046FFF75EFD01
:2053C00038BDA94B01461C330122184622F0F5B938B5A54C02461D34012369462046FFF767
:2053E0004DFD38BDA04B01461D330122184622F0E4B938B59C4C02461E3402236946204613
:20540000FFF73CFD38BD984B01461E330222184622F0D3B938B5944C02462034042369468E
:205420002046FFF72BFD38BD8F4B014620330422184622F0C2B938B58B4C024624340423E3
:2054400069462046FFF71AFD38BD874B014624330422184622F0B1B938B5834C0246283465
:20546000042369462046FFF709FD38BD7E4B014628330422184622F0A0B938B57A4C0246AA
:205480002C34042369462046FFF7F8FC38BD764B01462C330422184622F08FB938B5724CA1
:2054A00002463034012369462046FFF7E7FC38BD6D4B014630330122184622F07EB91CB53C
:2054C00000EB800000F279100A4640F0804005236946FFF7D3FC1CBD00EB800000F279104B
:2054E00040F08040052222F068B94FF4C87208B502EB40000A4640F0804002236946FFF7F1
:20550000BDFC08BD4FF4C87202EB400040F08040022222F052B94FF4CC7208B502EB4000C7
:205520000A4640F0804002236946FFF7A7FC08BD4FF4CC7202EB400040F08040022222F025
:205540003CB91CB500EB800001EB810100EB810000F2891040F0804005236946FFF78EFC6E
:205560001CBD0B46114600EB800003EB830200EB820000F2891040F08040052222F01DB9D5
:20558000090108B501EB800000F2CE2040F0804004236946FFF772FC08BD0B4611461A0146
:2055A00002EB800000F2CE2040F08040042222F004B91CB500EB800000F2DD300A4640F0FE
:2055C000804005236946FFF759FC1CBD00EB800000F2DD3040F08040052222F0EEB81CB506
:2055E00000EB800000F2F1300A4640F0804005236946FFF743FC1CBD00EB800000F2F1308A
:2056000040F08040052222F0D8B81CB500EB800001EB810100EB810000F2F13040F08040B8
:2056200005236946FFF72AFC1CBD0B46114600EB800003EB830200EB820000F2F13040F068
:205640008040052222F0B9B81CB500EB800001EB810100EB810000F2B94040F080400523C7
:205660006946FFF70BFC1CBD4D0100400B46114600EB800003EB830200EB820000F2B94039
:2056800040F08040052222F098B81CB500EB800001EB810100EB810000F2996040F08040A0
:2056A00005236946FFF7EAFBDDE70B46114600EB800003EB830200EB820000F2996040F066
:2056C0008040052222F079B81CB500EB800000F605100A4640F0804005236946FFF7CEFB83
:2056E000C1E700EB800000F6051040F08040052222F063B840F6121208B502EB40000A46B4
:2057000040F0804002236946FFF7B8FB08BD40F6121202EB400040F08040022222F04DB8A5
:205720001CB500EB800001EB810100EB410000F6091040F0804005236946FFF79FFB92E7B4
:205740000B46114600EB800003EB830200EB420000F6091040F08040052222F02EB840F642
:205760007A1208B502EB40000A4640F0804002236946FFF783FB08BD40F67A1202EB400077
:2057800040F08040022222F018B840F6821208B502EB40000A4640F0804002236946FFF755
:2057A0006DFB08BD40F6821202EB400040F08040022222F002B838B5F74C02460223694699
:2057C0002046FFF75BFB38BDF34B01460222184621F0F3BF38B5F04C0246A41C0223694653
:2057E0002046FFF74BFB38BDEB4B01469B1C0222184621F0E2BF38B5E74C0246241D0123DD
:2058000069462046FFF73AFB38BD38B5E24C0246641D022369462046FFF730FB38BDDE4BF6
:2058200001465B1D0222184621F0C7BF38B5DA4C0246E41D022369462046FFF71FFB38BDF5
:20584000D54B0146DB1D0222184621F0B6BF38B5D14C02460934012369462046FFF70EFB1A
:2058600038BDCD4B014609330122184621F0A5BF38B5C94C02460A34012369462046FFF7EB
:20588000FDFA38BDC44B01460A330122184621F094BF40F6951208B502EB40000A4640F05D
:2058A000804002236946FFF7E9FA08BD40F6951202EB400040F08040022221F07EBF38B55D
:2058C000B54C02463F34022369462046FFF7D6FA38BDB14B01463F330222184621F06DBFA3
:2058E00038B5AD4C02464134022369462046FFF7C5FA38BDA84B014641330222184621F0E0
:205900005CBF38B5A44C02464334042369462046FFF7B4FA38BDA04B0146433304221846CF
:2059200021F04BBF38B59C4C02464734042369462046FFF7A3FA38BD974B01464733042227
:20594000184621F03ABF38B5934C02464B34042369462046FFF792FA38BD8F4B01464B33FA
:205960000422184621F029BF1CB500EB800000F6D6100A4640F0804005236946FFF77EFA0D
:2059800071E600EB800000F6D61040F08040052221F013BF38B5804C024663340423694601
:2059A0002046FFF76BFA38BD7B4B014663330422184621F002BF38B5774C02466734012381
:2059C00069462046FFF75AFA38BD734B014667330122184621F0F1BE4FF41F6208B502EB25
:2059E00080000A4640F0804004236946FFF746FA08BD4FF41F6202EB800040F080400422CF
:205A000021F0DBBE1CB500EB800001EB810100EB810000F6EF1040F0804005236946FFF714
:205A20002DFA20E60B46114600EB800003EB830200EB820000F6EF1040F08040052221F029
:205A4000BCBE1CB500EB800001EB810100EB810000F6532040F0804005236946FFF70EFA88
:205A600001E60B46114600EB800003EB830200EB820000F6532040F08040052221F09DBE60
:205A800040F6A83208B502EB80000A4640F0804004236946FFF7F2F908BD40F6A83202EB13
:205AA000800040F08040042221F087BE38B53B4C0246012369462046FFF7E0F938BD374BBF
:205AC00001460122184621F078BE38B5334C0246641C042369462046FFF7D0F938BD2F4B19
:205AE00001465B1C0422184621F067BE38B52B4C0246641D042369462046FFF7BFF938BD22
:205B0000264B01465B1D0422184621F056BE38B5224C02460934022369462046FFF7AEF9F5
:205B200038BD1E4B014609330222184621F045BE38B51A4C02460B34022369462046FFF7E4
:205B40009DF938BD154B01460B330222184621F034BE38B5114C02460D3404236946204641
:205B6000FFF78CF938BD0D4B01460D330422184621F023BE38B5094C0246113401236946BE
:205B80002046FFF77BF938BD044B014611330122184621F012BE00008C090040EC0B0040F8
:205BA00038B5CF4C0246012369462046FFF766F938BDCB4B01460122184621F0FEBDC9009F
:205BC00008B501EB400000F6F63040F0804002236946FFF753F908BD0B461146DA0002EB86
:205BE000400000F6F63040F08040022221F0E5BD40F67E4208B502EB40000A4640F0804062
:205C000002236946FFF73AF908BD40F67E4202EB400040F08040022221F0CFBD40F6B242C4
:205C200008B502EB40000A4640F0804002236946FFF724F908BD40F6B24202EB400040F007
:205C40008040022221F0B9BD1CB500EB800001EB810100EB810000F6CF4040F080400523A6
:205C60006946FFF70BF9FEE40B46114600EB800003EB830200EB820000F6CF4040F08040B1
:205C8000052221F09ABD1CB500EB800001EB810100EB810000F61F5040F080400523694633
:205CA000FFF7ECF8DFE40B46114600EB800003EB830200EB820000F61F5040F080400522D8
:205CC00021F07BBD40F6865208B502EB40000A4640F0804002236946FFF7D0F808BD40F6B6
:205CE000865202EB400040F08040022221F065BD40F6885208B502EB80000A4640F08040DE
:205D000004236946FFF7BAF808BD40F6885202EB800040F08040042221F04FBD40F6925276
:205D200008B502EB40000A4640F0804002236946FFF7A4F808BD40F6925202EB400040F097
:205D40008040022221F039BD2DE9F84304226946002021F0E5F9634C00060FD46249009848
:205D60008227624D624E4FF0190888420DD104226946104621F0D4F9000602D52068BDE800
:205D8000F8835C490098884206D027607846C5F8008030608220F2E7002020602860784638
:205DA00030600020EBE72DE9F0434E4EDFF83C81DFF83C9191B000254FF4005700246119A6
:205DC000684600F083F820226946204621F070FA00060ED42034BC42F1D30024611968468E
:205DE00000F074F8202208A9204621F099F9000603D5306811B0BDE8F083202208A968465B
:205E000029F062FC40B1822019213060C8F800107946C9F80010EDE72034BC42DED3ED1C6E
:205E2000FF2DCBD9002030607946C8F80000C9F80010DFE770B58CB000208DF824002A4830
:205E40000A9024226946042021F06AF9254D000617D4FFF7A8FF000613D400244FF4005671
:205E6000012209A9204621F023FA000609D4641CB442F5D324226946042021F019FA000655
:205E800002D528680CB070BD04220AA9002021F00FFAF7E738B504466946002006F0A9FE1E
:205EA0000106104801D5006838BDBDF8001001B101212170002101600C48016078460C49DC
:205EC0000860002038BDFF2006F0CCBF00220B46491C521C00F8013B202AF8D3704700005F
:205EE000FE0B004008C007204CC9E44B0CC0072010C00720CEFAADDE38B504466846FFF70E
:205F000008F801060A4801D5006838BD9DF80010032909D0872101600649002008607846AD
:205F200005490860872038BD204601F041FE38BD08C007200CC0072010C0072038B5044674
:205F40006846FEF7E6FF01060A4801D5006838BD9DF80010032909D087210160064900200B
:205F60000860784605490860872038BD204601F0ABFE38BD08C007200CC0072010C00720DB
:205F800038B504466846FEF7C4FF01060A4801D5006838BD9DF80010032909D08721016025
:205FA000064900200860784605490860872038BD204601F025FF38BD08C007200CC00720A8
:205FC00010C0072038B504466846FEF7A2FF01060A4801D5006838BD9DF80010032909D019
:205FE00087210160064900200860784605490860872038BD204601F08FFF38BD08C00720E8
:206000000CC0072010C0072038B504466846FEF780FF01060A4801D5006838BD9DF800100C
:20602000032909D087210160064900200860784605490860872038BD204602F007F838BD1F
:2060400008C007200CC0072010C0072038B504466846FEF75EFF01060A4801D5006838BDA4
:206060009DF80010032909D087210160064900200860784605490860872038BD204602F02E
:206080005FF838BD08C007200CC0072010C0072038B504466846FEF73CFF01060A4801D597
:2060A000006838BD9DF80010032909D087210160064900200860784605490860872038BDE9
:2060C000204602F0C3F838BD08C007200CC0072010C0072038B504466846FEF71AFF0106E5
:2060E0000A4801D5006838BD9DF80010032909D0872101600649002008607846054908601D
:20610000872038BD204602F01BF938BD08C007200CC0072010C0072038B56846FEF7F9FE22
:206120000E4C000611D49DF80000032809D087200B4920600020086078460A49086087205E
:2061400038BD02F083F9000601D5206838BD04208DF800006846FEF7D2FE38BD08C0072083
:206160000CC0072010C007202DE9FE43284C2068822800D001276846FEF7CBFE00063AD4C0
:206180009DF800001D280DD101A800F049F8000631D42048018821F00201018000F0C0FD2F
:2061A000000628D49DF8000000251B4EDFF86C8003280DD004280BD00E2809D01B2807D0BF
:2061C0008720206079463560C8F80010BDE8FE83002002F063F900060DD49DF800001B2821
:2061E0000BD06846FEF7A6FE000604D46846FEF786FE000601D52068E8E717B1012008F064
:20620000E7FC2560794635600020C8F80010DDE708C0072002C007200CC0072010C007204C
:206220002DE9F04389B081466846FEF772FE344C000651D49DF8000000250526314FDFF81B
:20624000C88004280AD01D2831D08720206079463D60C8F8001009B0BDE8F08306A9484649
:2062600002F0DEF920B1922813D0932834D10CE09DF8180090B32548007878B31D208DF879
:2062800000006846FEF73BFE24E0F9F7C9FF0E2005E0386831281FD1F9F7C2FF16208DF8FE
:2062A00000006846FEF72BFEF9F7CFFF14E001A804F06DFF00060FD407A9039805F0B9F97C
:2062C000000609D403A8FFF7C7F8000604D407A8FFF7D3F8000602D52068BCE709E008F044
:2062E00022FB30B1256079463D600020C8F80010B1E78DF800606846FEF701FEABE700001E
:2063000008C007200CC0072010C00720FA02000030B587B0054603A8FEF7FBFD2A4C00062D
:2063200049D49DF80C001D280DD104A8FFF778FF000640D42548018821F00201018000F0CE
:20634000EFFC000637D49DF80C10012929D00020022909D0872121601D49086078461D492E
:206360000860872007B030BD2988ADF804106988ADF8061029798DF808108DF8090001A8DE
:2063800003F020F8000616D469462B2010F058FB000610D49DF80000C00702D001208DF8F7
:2063A0000C0003A8FEF7BCFD000604D4284602F04FFC000601D52068D4E706208DF80C0019
:2063C00003A8FEF79CFDCDE708C0072002C007200CC0072010C0072038B56846FEF799FDE8
:2063E0000F4C000616D49DF80000062809D087200C4920600020086078460B490860872091
:2064000038BD02F0A3FC000604D46846FEF792FD000601D5206838BD6846FEF770FD38BD88
:2064200008C007200CC0072010C0072038B505466846FEF76EFD0F4C000612D49DF8000061
:20644000062809D087200C4920600020086078460A490860872038BD284602F0AFFC00060B
:2064600001D5206838BD07208DF800006846FEF746FD38BD08C007200CC0072010C0072069
:2064800038B504466846FEF744FD01060B4801D5006838BD9DF8001004290BD0062909D09F
:2064A00087210160064900200860784605490860872038BD204602F0A5FD38BD08C007200E
:2064C0000CC0072010C0072038B504466846FEF720FD01060B4801D5006838BD9DF80010A9
:2064E00004290BD0062909D087210160064900200860784605490860872038BD204602F044
:206500002BFE38BD08C007200CC0072010C0072038B504466846FEF7FCFC01060B4801D582
:20652000006838BD9DF8001004290BD0062909D087210160064900200860784605490860F5
:20654000872038BD204602F09FFE38BD08C007200CC0072010C0072038B505466846FEF701
:20656000D8FC124C000617D49DF80000022809D087200F4920600020086078460D490860DD
:20658000872038BD002004F012F8000604D4284602F018FF000601D5206838BD01208DF8ED
:2065A00000006846FEF7ABFC38BD000008C007200CC0072010C0072038B505466846FEF7E8
:2065C000A8FC1F4C000632D49DF8000010281FD00CDC0C281CD004DC012819D002280DD1E2
:2065E00016E00D2814D00E2808D111E013280FD014280DD015280BD0182809D08720114927
:2066000020600020086078460F490860872038BD6846FEF785FC000609D46846FEF791FC21
:20662000000604D4284606F0B1FE000601D5206838BD08208DF800006846FEF760FC38BD6F
:2066400008C007200CC0072010C007202DE9FE4301A8FEF75EFC3A4C00066FD49DF80400AA
:206660000127384E0025082806D0092804D00A2857D08720BDE8FE8306F032FF00903168C6
:206680004FF00A080291062824D2DFE800F003052317190300953CE06846FFF732F9000657
:2066A0004CD402A8FFF73EF9000647D48DF8048001A8FEF724FC000640D42AE0082000E0CF
:2066C00009208DF8040001A8FEF719FC0090306802901EE008F0BFF80098822801D0922821
:2066E00001D104F0C7FB6846FFF70BF9000625D402A8FFF717F9000620D49DF804000928F7
:2067000007D08DF8048001A8FEF7F9FB14E000970295009820600299316079460A4A11601D
:20672000A8E78120009002956846FFF7EAF8000604D402A8FFF7F6F80006E8D5206899E745
:2067400008C007200CC0072010C007202DE9F04186B003A8FFF796F8364C000660D402A84E
:20676000FEF7D7FB00065BD401A8FFF7D4F8000656D404A8FFF7E0F8000651D49DF8080040
:2067800087272D4D2D4E4FF000080A2801D0092835D107F0A1FC000642D4019801286846B5
:2067A00008D0FEF7C7FB00063AD49DF80800092805D013E0FEF7CFFB000631D414E0019849
:2067C000922801D0822802D113208DF800009DF80C00142802D10C208DF800000198932844
:2067E00002D10E208DF800006846FEF788FB000616D49DF80800092814D00A2808D02760BA
:206800007846C5F800803060872006B0BDE8F0819DF80C000E2805D1FBF700FC000601D503
:206820002068F2E7019820600499296079463160EBE7000008C007200CC0072010C00720BD
:2068400038B505466846FEF764FB164C00061FD49DF800000C2809D087201349206000205E
:206860000860784611490860872038BD6846FEF757FB00060CD40D208DF800006846FEF764
:2068800060FB000604D4284602F042FF000601D5206838BD08208DF800006846FEF72FFB4B
:2068A00038BD000008C007200CC0072010C00720FEB56846FEF72DFB2B4C00064CD49DF85A
:2068C00000002A4D2A4E0D2809D0182807D08720206000202860784630608720FEBD02A87B
:2068E000FEF706FB000637D49DF8080038B1912020609C202860784630609120FEBD0120BB
:2069000003F055FE000627D401A803F01DFB00064FF0020722D59DF80400E8B1012809D003
:20692000022810D08820206009202860784630608820FEBDF9F774FC18208DF8000006E0C0
:20694000F9F783FC08E0F9F76BFC8DF800706846FEF7D5FA0006F3D52068FEBD8DF800701C
:206960006846FEF7CCFAFEBD08C007200CC0072010C007202DE9FC4781466846FEF7C9FA94
:206980001F4C000632D49DF80000002587261D4FDFF87480022804D00D2815D018280BD1AE
:2069A00012E001A8FFF776FA00061FD49DF8040050B11648007838B1266079463D608720FB
:2069C000C8F80010BDE8FC8701A9484603F06CF870B19DF8040048B1F9F722FC18208DF8B2
:2069E00000006846FEF78BFAF9F72FFC2068E9E702208DF800006846FEF781FAE2E700006E
:206A000008C007200CC0072010C00720FA020000F8B507463148002505706846FEF779FA7E
:206A20002F4C00064FD49DF800002E4E132811D004DC01280ED00E2804D10BE0152809D092
:206A40001B2807D08720206078462749356008608720F8BDFAF731FF93281ED06846FEF701
:206A60005FFA00062FD49DF800001B2819D002208DF800006846FEF764FA000623D401202D
:206A800003F095FD00061ED4384607F073FB50B18F280FD0922816D117E0F9F7C1FB0E208D
:206AA00016E01020E4E708208DF800006846FEF726FAF8BDF9F7B4FB3068072801D1142054
:206AC00006E0F9F7C2FB2068F8BDF9F7A9FB16208DF800006846FEF712FAF2E724C0072004
:206AE00008C007200CC0072010C00720F8B505460E466846FEF70DFA1C4C00062DD49DF8C3
:206B00000020132A19D008DC012A16D0022A14D00E2A12D0102A06D10FE0142A0DD0152AB6
:206B20000BD0182A09D0872011492060002008607846104908608720F8BD6846FEF7F0F9EF
:206B400000060AD46846FEF7FCF9000605D43146284607F0DBFC000601D52068F8BD0820E6
:206B60008DF800006846FEF7CAF9F8BD08C007200CC0072010C00720F8B505460E466846A2
:206B8000FEF7C7F91D4C000627D49DF800101C4A1C48102911D004DC02290ED00D2904D159
:206BA0000BE0112922D0142907D08721216000211160794601608720F8BD6846FEF7B0F927
:206BC00000060AD46846FEF7BCF9000605D43146284607F057FD000601D52068F8BD082029
:206BE0008DF800006846FEF78AF9F8BD91212160A9211160794601609120F8BD08C0072052
:206C00000CC0072010C007203EB501A8FEF770F9214C00063ED46846FEF77BF9000639D4E1
:206C200002A901201FF056FB000633D49DF800001A4D022806D00E2804D0102802D0029871
:206C4000C00705D003F0EAFA80B1922822D114E09DF804208721124821600AB1042100E0F3
:206C6000002129607946016087203EBD10208DF800006846FEF743F93EBD2868312809D156
:206C8000F9F7CEFA16208DF800006846FEF737F9F9F7DBFA20683EBD08C007200CC0072084
:206CA00010C0072038B505466846FEF732F9184C00061DD49DF80000112809D087201549D0
:206CC000206000200860784613490860872038BD12482968016069684160A968816030208E
:206CE0000EF08CFB000603D424F05EFA000601D5206838BD284606F0E0FA10B107F0ABFDCF
:206D0000F6E702208DF800006846FEF7F8F838BD08C007200CC0072010C007206DC2072038
:206D2000F8B56846FEF7F5F8144D00061BD49DF800000024124E134F052808D01D2816D015
:206D4000872028607846346038608720F8BD03F027FB000607D401208DF800006846FEF77F
:206D6000CEF8000601D52868F8BD07F0BCFD2C607846346038600020F8BD000008C0072042
:206D80000CC0072010C0072038B56846FEF7C1F80E4C000611D49DF80000072809D0872037
:206DA0000B4920600020086078460A490860872038BD03F01BFB000601D5206838BD0120DF
:206DC0008DF800006846FEF79AF838BD08C007200CC0072010C0072038B504466846FEF751
:206DE00098F801060A4801D5006838BD9DF80010032909D08721016006490020086078462F
:206E000005490860872038BD204603F065FC38BD08C007200CC0072010C0072038B5044661
:206E20006846FEF776F801060A4801D5006838BD9DF80010032909D0872101600649002093
:206E40000860784605490860872038BD204603F097FC38BD08C007200CC0072010C0072000
:206E600038B504466846FEF754F801060A4801D5006838BD9DF80010032909D087210160AD
:206E8000064900200860784605490860872038BD204603F0C9FC38BD08C007200CC0072016
:206EA00010C0072038B504466846FEF732F801060B4801D5006838BD9DF8001001290BD0A0
:206EC000022909D087210160064900200860784605490860872038BD204603F0DDFD38BD96
:206EE00008C007200CC0072010C007202DE9F8438046694601201FF0EDF9104C00060CD49B
:206F000000980F4E0F4FC0074FF0000508D00021404603F043FE000609D52068BDE8F883D4
:206F2000872020607846356038608720F6E725607846356038600020F0E7000008C0072065
:206F40000CC0072010C0072038B50446FDF76AFE000602D51648006838BD2046FEF749F880
:206F600000061FD4A01CFEF755F800061AD4201DFEF761F8000615D407F0C1FE000602D519
:206F800007F069FC0EE06846FEF71BF8000609D46846FDF780FD000604D46846FEF707F86F
:206FA000000602D5FDF7DEFE38BDFDF768FE38BD08C007202DE9F04188B001A8FDF798FF3E
:206FC000384C00065ED49DF80400374F374E48B1912020609C20306078463860912008B01C
:206FE000BDE8F08106A901201FF074F9000649D406984FF00005C00746D06846FDF789FF23
:2070000000063FD46846FDF78BFF00063AD46846FDF797FF000635D408208DF80000684675
:20702000FDF76DFF00062DD44FF001088DF8088002A8FEF71DFC000624D403208DF80C002A
:2070400003A8FDF7A3FF00061CD419490220087014482560FEF755FC000613D413483560F9
:20706000FEF760FC00060DD4ADF8108004A8FEF726FC000606D4ADF8145005A8FEF730FC29
:20708000000608D52068AAE7872020607846356038608720A3E72560784635603860002021
:2070A0009DE7000008C0072010C007200CC0072000C007202DE9FF470646684603F042FA07
:2070C000924C000662D4BDF800004FF4B46148433178C1EB011100EB81007178451802A83B
:2070E000FEF7D8FE000651D49DF80800DFF82092DFF820A286274FF01708D0B18648007809
:20710000B8B16946022004F0EBF800063ED401A9032004F0E5F8000638D4BDF80000BDF82C
:207120000410C0EB001000EB400001EB401085421DD303A8FBF768F8000627D49DF80C00C3
:20714000F8B16846FEF740FB00061FD401A8FEF74BFB00061AD4BDF80000BDF80410C0EBAE
:20716000001000EB400001EB4010854209D227607946C9F800808620CAF8001004B0BDE89E
:20718000F08730461FF0FFFD000601D52068F5E703F078FAF2E72DE9FE4F8146694653202D
:2071A0000FF04EFC594C000629D49DF8000000F004008DF8000001A8FDF7ABFE00061ED492
:2071C0009DF80410524D534E0027DFF85081102918D009DC022915D00D291AD091200E29D9
:2071E0007CD00F2906D17CE011290BD0192916D01A2914D002A8FBF707F8000678D52068FE
:20720000BDE8FE8F4846FFF755FF05E088F800700FE048461FF0B7FD0006F0D4F6E748461A
:20722000FFF748FF0028EAD198F80000C246022805D0276078462F6030600020E0E79DF8B7
:20724000000020B147200EF0D9F80006D7D448461FF030FD0006D2D4314999F80280886883
:20726000304A8B681B1A9342FBD348461FF022FD0006C4D499F80210414507D1822020604C
:2072800005202860784630608220B9E703218AF8001025494FF0010801A881F80080FDF7AF
:2072A0005AFE0006ABD401A8FDF729FE0006A6D40420FAF7C3F80006A1D49DF8000020B1FC
:2072C000012007F085FC000699D4C4F8008078462F603060012093E700E009E02060A020E5
:2072E00001E02060D220286078463060912087E79DF808108720206011B10420286000E024
:207300002F607846306087207AE7000008C007200CC0072010C00720FA02000026C00720A6
:2073200000000940E0C81000340000102DE9FE43054601A8FEF7AEFDB14C00062BD49DF886
:207340000400B04EB04F4FF086084FF01A09A8B1AE48007848B16946022003F0C1FF0006B3
:2073600019D4BDF8000085421CD36846FAF7B7F9000610D4BDF80000854213D302A8FAF77F
:2073800043FF000607D49DF8080098B16846FEF71BFA000602D52068BDE8FE83BDF80000EC
:2073A000854207D2C4F800807846C6F8009038608620F1E700202060306078463860002029
:2073C000EAE72DE9F14F88B003A90898F9F7FFFABDF80C008B4D8C4E894C4FF086094FF0C4
:2073E000140B012803D948F26A01884204D3C4F80090C5F800B06DE002A953200FF020FBE5
:2074000000067DD49DF8080000F004008DF808006846FDF77EFD0006F3D49DF80000002751
:207420004FF087084FF0040A102824D009DC022821D00D281FD091210E2877D00F2808D1A2
:20744000A0E0112817D019280CD01A2813D01C2811D006A8FAF7D8FE000651D49DF81800D8
:2074600098B996E007A901201EF034FF000647D40798C00709D0BDF80C00FFF757FFDFF8EF
:20748000908168B386283BD104E0C4F80080C5F800A081E088F800709DF800001C2810D07F
:2074A0001A282DD019282BD06846FDF739FD000626D41C208DF800006846FDF720FD0006F3
:2074C0001ED40220F9F7A7FF000619D41A20C4F80090286078463060862009B0BDE8F08F30
:2074E00001A81FF01CFC00064FF0010A07D54FF4FA60ADF804008DF806A08DF807A000E013
:207500006EE005A901A8F9F762FABDF80C10BDF8140098F80020814240460ED9012A06D0FF
:20752000418088F800A0C4F800A063E027E042888A4204D088F8007059E7012AF7D0089898
:207540001FF043FC00064BD44FF0020988F800909DF8080048B135200DF050FF00063FD40E
:20756000012007F035FB00063AD40220F9F766FF000635D49DF800001C2811D01AE0A020B5
:20758000216001E0D22021602860784630609120A3E7C4F800802F607846306087209CE7C2
:2075A0006846FDF7C7FC00061AD46846FDF7A7FC000615D403F066F89DF80000192807D040
:2075C0001A2805D0276078462F603060002084E79DF8080050B139200DF010FF000601D5C6
:2075E00020687AE700210BA023F083FC88F80090C4F800A078462F60306001206DE7000086
:2076000008C007200CC0072010C00720FA02000026C00720200A200A200A200A200A200A8C
:20762000200A200A00000000F0B505464179844C844F854E91B0862009B1042902D92060AD
:20764000062005E0297909B11E2907D920600520386078463060862011B0F0BD698828885C
:2076600002F006FF00067DD468796946FDF760FF0006F8D4BDF800100020A1F57F42FF3A92
:2076800006D18B2121603860784630600846E3E7064600906846FDF78FFD000662D46846F4
:2076A000FEF751F900065DD4012769463846FDF7B6FD00067ED47F1CFFB2112FF5D36846FE
:2076C000FDF7DEFD000675D46846FDF7E8FD000670D4012769463846FDF7CFFC000669D464
:2076E0007F1CFFB20B2FF5D3012769463846FEF7C7F900065ED47F1CFFB2112FF5D36846F8
:20770000FDF7CFFC000655D46846FDF7ECFC000650D46846FDF7A0FC00064BD401270096A6
:2077200069463846FEF758F9000643D47F1CFFB2052FF5D9ADF800606846FDF74EFD000673
:2077400038D46846FDF75AFD000633D46846FDF7B9FC00062ED46846FDF7D6FC000629D441
:20776000009600E026E0012669463046FDF76BFD00061FD4761CF6B2112EF5D32846FDF749
:2077800038FC000616D4A81CFDF744FC000611D4281DFDF750FC00060CD426F0B6FF0006A6
:2077A00008D4012007F014FA000603D4FDF73AFA000601D520684FE701248DF80040684690
:2077C000FDF7E4FB000624D420480470681DFDF7E2FC00061DD46846FDF7F3FB000618D42C
:2077E0006846FDF758F9000613D46846FDF7DFFB00060ED46846FDF7F5FB000609D4684622
:20780000FDF723F9000604D46846FDF7E1FB000602D5FDF7A7FA1FE707F058F8000609D45A
:207820008DF8014068798DF80200684604F06EFE000602D507F00FF8EBE7FDF720FA0BE75F
:2078400008C007200CC0072010C0072000C0072070B5057A624E98B00446102D0AD98620BC
:20786000604930600320086078465F490860862018B070BD05B9012560681190214611A86E
:20788000FDF775F8000603D4FDF7CCF9000601D53068EDE716A8FDF799FC000652D411A97C
:2078A00016A8FCF7F0FE00064CD416A8FDF784FC000647D416A8FDF79AFC000642D4BDF897
:2078C0005800401CADF8580016A8FDF786FC000638D416A92846FDF7AEFC000632D411A920
:2078E00016A8FCF7D0FE00062CD416A92846FDF796FC000626D416A92846FDF7B1FC00067C
:2079000020D4214616A8FCF7F7FE00061AD416A92846FDF798FC000614D404F10800FDF7DE
:20792000CFFC00060ED42046FDF7DBFC000609D4201DFDF7E7FC000604D411A8FDF7F3FCF2
:20794000000602D5FDF70EFA92E707F0E9F800063DD4012005F086FA000638D416A8FEF78B
:2079600099FA000633D49DF8580090B11F48007878B112A8FDF719FC000628D48DF8545043
:20798000206813901198149012A804F07CF800061DD40C208DF80100207A8DF80F006068AE
:2079A000CDF803002068CDF807001198CDF80B000F4904A827F0B4FE0DF10200FDF7F5FB81
:2079C000000604D4684604F0A1FD000602D506F042FFB7E7064900200870FDF750F947E785
:2079E00008C007200CC0072010C00720FA020000BBC2072070B5057A684E98B00446102DE5
:207A00000AD986206649306003200860784665490860862018B070BD05B901256068119057
:207A2000214611A8FCF7A3FF000603D4FDF7FAF8000601D53068EDE716A8FDF7C7FB00060C
:207A400062D411A916A8FCF73EFE00065CD416A8FDF7B2FB000657D416A8FDF7D9FB0006F7
:207A600052D4BDF85800401CADF8580016A8FDF7C5FB000648D416A8FDF76FFF000643D4A9
:207A800011A916A8FCF7FFFD00063DD416A8FDF75AFF000638D416A92846FDF7CCFB00065D
:207AA00032D411A916A8FCF70EFE00062CD416A92846FDF7B4FB000626D416A92846FDF752
:207AC000CFFB000620D4214616A8FCF735FE00061AD416A92846FDF7B6FB000614D404F1EE
:207AE0000800FDF7EDFB00060ED42046FDF7F9FB000609D4201DFDF705FC000604D411A8C0
:207B0000FDF711FC000602D5FDF72CF982E706F0FAFF000638D416A8FEF7BCF9000633D48F
:207B20009DF8580090B12048007878B112A8FDF73CFB000628D48DF854502068139011982A
:207B4000149012A803F0FCFF00061DD40D208DF80100207A8DF80F006068CDF803002068E9
:207B6000CDF807001198CDF80B00104904A827F0D7FD0DF10200FDF718FB000604D468463D
:207B800004F0C4FC000602D506F065FEBCE7074900200870FDF773F83CE7000008C00720FF
:207BA0000CC0072010C00720FA020000BBC2072030B504460079404D93B008B110280AD9EF
:207BC00086203E4928600320086078463C490860862013B030BDFDF725F8000601D52868E7
:207BE000F7E76846FDF7F2FA000626D421466846FCF769FD000620D46846FDF7DDFA000632
:207C00001BD420796946FDF716FB000615D421466846FCF758FD00060FD420796946FDF7B7
:207C2000FEFA000609D4201DFDF7C1FB000604D42046FDF7ABFB000602D5FDF793F8C8E793
:207C400006F054FF000630D46846FEF723F900062BD49DF8000048B11A48007830B120683C
:207C6000129012A803F0BDFF00061ED408208DF805000025CDF806500DF10B00FDF76EFBA9
:207C8000000612D46846FDF77AFB00060DD4BDF80000ADF80C008DF80A502068CDF80E005A
:207CA00001A804F033FC000602D506F0D4FDC4E7FCF7E5FF8DE7000008C007200CC007207C
:207CC00010C00720FA02000030B504460079484D95B008B110280AD986204649286003207B
:207CE0000860784644490860862015B030BDFCF799FF000601D52868F7E76846FDF766FA3A
:207D0000000640D421466846FCF7BDFC00063AD46846FDF751FA000635D420796946FDF73C
:207D20008AFA00062FD421466846FCF7ACFC000629D420796946FDF772FA000623D412A8A4
:207D4000FDF7BDFE00061ED49DF8480088B16946FDF7A3FE000616D421466846FCF7B3FC7B
:207D6000000610D469469DF84800FDF789FE000609D4201DFDF71BFB000604D42046FDF7B0
:207D800005FB000602D5FCF7EDFFAEE706F0A1FE000626D46846FEF77DF8000621D49DF855
:207DA000000048B11548007830B12068139013A803F041FF000614D469464C200EF040FEB6
:207DC00000060ED49DF80000800702D49DF8480050B904208DF8050001A804F097FB000600
:207DE00002D506F038FDCEE7FCF749FF7DE7000008C007200CC0072010C00720FA02000058
:207E000070B504460079404D94B008B110280AD986203E4928600320086078463C490860EA
:207E2000862014B070BDFCF7FDFE000655D46846FDF7CCF9000626D421466846FCF723FC00
:207E4000000620D46846FDF7B7F900061BD420796946FDF7F0F9000615D421466846FCF7C5
:207E600012FC00060FD420796946FDF7D8F9000609D4201DFDF79BFA000604D42046FDF71D
:207E800085FA000602D5FCF76DFFCAE706F014FE000632D46846FDF7FDFF00062DD49DF828
:207EA000000048B11B48007830B12068129012A803F0EEFE000620D407208DF80500002679
:207EC000CDF806600DF10B00FDF748FA000604D46846FDF754FA000601D52868A1E7BDF8C1
:207EE0000000ADF80C008DF80A602068CDF80E0001A804F00BFB000602D506F0ACFCC2E7C0
:207F0000FCF7BDFE8DE7000008C007200CC0072010C00720FA02000070B504460079474DEE
:207F200094B0032608B1102809D98620286044480660784643490860862014B070BDFCF7A5
:207F400071FE000601D52868F7E76846FDF73EF9000640D421466846FCF7B5FB00063AD4A9
:207F60006846FDF729F9000635D420796946FDF762F900062FD421466846FCF7A4FB0006E1
:207F800029D420796946FDF74AF9000623D412A8FDF795FD00061ED49DF8480088B169466B
:207FA000FDF77BFD000616D421466846FCF78BFB000610D469469DF84800FDF761FD000609
:207FC00009D4201DFDF7F3F9000604D42046FDF7DDF9000602D5FCF7C5FEAEE706F05FFD1F
:207FE000000625D46846FDF755FF000620D49DF8000048B11448007830B12068139013A869
:2080000003F070FE000613D469464C200EF018FD00060DD49DF80000800702D49DF848002E
:2080200048B98DF8056001A804F070FA000602D506F011FCCFE7FCF722FE7EE708C0072051
:208040000CC0072010C00720FA02000010B594B00446FCF7E7FD000603D53748006814B087
:2080600010BD12A8FDF7B2F8000626D412A8FDF7E2F9000621D412981190214611A8FCF7F9
:2080800022FB000619D411A8FDF796F8000614D411A8FDF7FEF800060FD4214611A8FCF708
:2080A000F2FA000609D411A8FDF7EAF8000604D42046FDF7AFF9000602D5FCF753FECEE7AC
:2080C00006F0E0FC000631D411A8FDF7E3FE00062CD49DF8440048B11848007830B120681C
:2080E000139013A803F07DFD00061FD408208DF801001298CDF802000DF10700FDF772F939
:20810000000613D411A8FDF77EF900060ED4BDF84400ADF8080000208DF806002068CDF8C8
:208120000A00684604F0F2F9000602D506F093FBC3E7FCF7A4FD92E708C00720FA020000A5
:2081400030B595B00446FCF76DFD3E4D000619D46846FDF73BF8000631D46846FDF76BF9EA
:2081600000062CD421466846FCF78DFA000626D46846FDF721F8000621D412A8FDF79FFC6B
:20818000000602D5286815B030BD9DF84800C8B16946FDF782FC000611D421466846FCF756
:2081A00092FA00060BD469469DF84800FDF768FC000604D42046FDF72DF9000611D5FCF72D
:2081C000D1FDE0E76846FDF764F80006F7D421466846FCF778FA0006F1D46846FDF750F80C
:2081E000E6E706F042FC000626D46846FDF752FE000621D49DF8000048B11348007830B14F
:208200002068139013A803F016FD000614D469464C200EF015FC00060ED49DF80000800756
:2082200002D49DF8480050B904208DF8050001A804F06CF9000602D506F00DFBBFE7FCF75E
:208240001EFDA0E708C00720FA02000030B595B00446FCF7E7FC384D000656D412A8FCF7E5
:20826000B5FF000626D412A8FDF7E5F8000621D412981190214611A8FCF705FA000619D474
:2082800011A8FCF799FF000614D411A8FDF711F800060FD4214611A8FCF7F5F9000609D429
:2082A00011A8FCF7FCFF000604D42046FDF7B2F8000603D5FCF756FD15B030BD06F0AEFBC0
:2082C000000633D411A8FDF7E5FD00062ED49DF8440048B11948007830B12068139013A888
:2082E00003F0D6FC000621D407208DF801001298CDF802000DF10700FDF774F8000604D45D
:2083000011A8FDF780F8000601D52868D4E7BDF84400ADF8080000208DF806002068CDF873
:208320000A00684604F0F2F8000602D506F093FAC0E7FCF7A4FCBFE708C00720FA0200007C
:2083400010B594B00446FCF76DFC000603D53D48006814B010BD6846FCF738FF00062ED432
:208360006846FDF768F8000629D421466846FCF7AAF9000623D46846FCF71EFF00061ED49A
:2083800012A8FDF79CFB000619D49DF84800C8B16946FDF782FB000611D421466846FCF73C
:2083A00092F900060BD469469DF84800FDF768FB000604D42046FDF72DF8000611D5FCF72E
:2083C000D1FCC6E76846FCF774FF0006F7D421466846FCF778F90006F1D46846FCF75FFFFB
:2083E000E6E706F00EFB000626D46846FDF752FD000621D49DF8000048B11348007830B183
:208400002068139013A803F06DFC000614D469464C200EF015FB00060ED49DF800008007FF
:2084200002D49DF8480050B903208DF8050001A804F06CF8000602D506F00DFABFE7FCF75F
:208440001EFC86E708C00720FA02000000B593B0FCF7E8FB000603D50F48006813B000BDBF
:2084600006F0C2FA00060FD40F208DF8010011A8FCF7ACFE000607D41198CDF80200684657
:2084800004F044F8000604D506F0E5F9FCF76AFCE4E7FCF7F4FBE1E708C00720F0B55B4DEF
:2084A000070093B0288802D040F0200001E040F010002880FCF7B6FB554E00067ED412A87E
:2084C000FCF773FE000655D469469DF84800FDF72FF800064ED4BDF800006946401CADF8D5
:2084E00000009DF84800FDF716F8000642D46846FCF767FD00063DD46846FCF7DDFA0006E7
:2085000038D46846FCF753FD000633D46846FCF769FD00062ED46846FCF7AAFA000629D4FA
:208520006846FCF755FD000624D4002468460094FCF742FE00065BD46846FDF7ABFC00062D
:2085400003D500BF06F087F914E03800314F0DD09DF8000028B1387818B102F08BFC00061F
:2085600008D406F00CFA000604D410E006F007FA000603D5FCF7F6FB13B0F0BD9DF8000097
:2085800028B1387818B102F075FC0006DAD48DF800406846FCF7FFFD0006D3D48DF800409E
:2085A0006846FCF7F3FC0006CCD46846FCF7C2FC0006C7D49DF80000022800E018E001D01D
:2085C000032007E08DF800406846FCF787FC0006B8D4082025F043FC02208DF8050001A845
:2085E00003F094FF0006ADD4FCF749FB000601D53068C1E7288820F03000288006483460A1
:2086000004607846054908600020B5E702C0072008C00720FA0200000CC0072010C0072008
:208620002DE9F04F9FB04FF00009054681F800900079FF4FFF4E8A46CB464FF08608FE4CEE
:2086400008B11E2803D90520C4F800800FE0288848F6AD61884203D91420C4F8008006E0F7
:208660006888B0F5B46F09D31720C4F8008030607846386086201FB0BDE8F08F13A8FCF7C6
:20868000C2FC000633D42888BDF84C108842E3D309D113A8FCF7C8FC000628D46888BDF8DB
:2086A0004C108842E0D36846FCF7E0FC00061ED413A8FCF78BFD000619D400991398884235
:2086C00007D08C2020607846C6F800B038608C20D1E7022004F0C6FB000608D4012002F0A3
:2086E00097FE000603D4FCF79DFA000601D52068C1E711A8FCF759FD00067DD413A8FCF76B
:2087000065FD0006F9D4139898B169469DF84400FCF7E2FE0006F0D413A96846FBF746FF6A
:208720000006EAD469469DF84400FCF7C8FE0006E3D413A8FDF711F90006DED4139898B112
:2087400069469DF84400FDF71CF90006D5D413A96846FBF72BFF0006CFD469469DF8440022
:20876000FDF702F90006C8D469469DF84400FCF7C9FE0006C1D4BDF800006946401CADF826
:2087800000009DF84400FCF7B0FE0006B5D413A8FCF72DFD0006B0D4BDF84C0098B1694675
:2087A0009DF84400FCF7E8FF0006A6D413A96846FBF7DBFF0006A0D469469DF84400FCF75B
:2087C000CEFF000699D413A8FCF722FD000694D4BDF84C00A8B169469DF84400FCF7E2FF68
:2087E00000068AD413A96846FBF7BFFF000684D469469DF8440000E066E1FCF7C6FF000630
:2088000089D44FF0010840468DF84880C0B213A9FCF711FD000684D41398B8B19DF8481052
:208820006A469DF84400FCF79CFE000685D413A96846FBF7BBFE000688D49DF848106A46AF
:208840009DF84400FCF77DFE000685D49DF8480013A9FCF705FD000685D41398B8B19DF8DC
:2088600048106A469DF84400FCF797FE00068DD413A96846FBF7E7FE000687D49DF8481099
:208880006A469DF84400FCF77BFE00068DD49DF84800401CC0B28DF848001028B6D913A882
:2088A000FCF7F7FC000686D4139898B169469DF84400FCF78BFE000684D413A96846FBF7C0
:2088C00075FE00068DD469469DF84400FCF771FE000686D413A8FCF7ECFC000687D41398D2
:2088E00098B169469DF84400FCF786FE000687D413A96846FBF75AFE00068CD469469DF871
:208900004400FCF76CFE000685D440468DF84880C0B213A9FDF7C1F8000687D41398B8B134
:208920009DF848106A469DF84400FDF79AF800068BD413A96846FBF739FE000685D49DF84F
:2089400048106A469DF84400FDF77BF800068ED49DF84800401CC0B28DF848001128D7D30C
:2089600040468DF84880C0B213A9FCF792FB00068CD41398B8B19DF848106A469DF8440086
:20898000FCF753FE00068ED413A96846FBF70EFE000688D49DF848106A469DF84400FCF7F8
:2089A00034FE000688D49DF84800401CC0B28DF848000B28D7D313A8FCF708FC000688D4BA
:2089C000139898B369883C20B1FBF0F0401CC1B28DF848106A469DF84400FCF747FE000655
:2089E00072D413A96846FBF7E1FD00066CD49DF848106A469DF84400FCF726FE000663D4E7
:208A000029796A469DF84400FCF74FFE00065BD413A96846FBF7CAFD000655D429796A4612
:208A20009DF84400FCF731FE00064DD4404605E010C007200CC0072008C007208DF8488083
:208A4000C0B213A9FCF7D5FF00063DD49DF848106A469DF84400FCF7E5FF000634D413A9F3
:208A60006846FBF7A3FD00062ED49DF848106A469DF84400FCF7C6FF000625D49DF84800A4
:208A8000401CC0B28DF848000528D9D969460120FCF774FA000617D413A90120FCF7F9FA77
:208AA000000611D49DF84400012813D002280CD003280AD004280DD08820206002203060F8
:208AC000784638608820D6E550E013A96846FBF7E0FE03E013A96846FBF7A2FE00066FD44B
:208AE00069460120FCF73EFA000669D4012004F0B9F9000664D412A8FDF7CCF900065FD487
:208B00009DF848004FF0920B88B35048007870B31BA9032004F02AF9000651D41DA905201A
:208B200002F0DEFB00064BD405221BA91DA826F0CBFD58B1FCF716F93D200CF05FFC0820D0
:208B400022F074FB3120C4F800B077E01AA9002002F0C6FB000633D49DF8680080062AD55B
:208B600005F000FF000603D505F075FE28E02CE02888ADF860006888ADF8620028798DF8D5
:208B8000640015A918A803F0DAF8306828280FD020680006E8D415A8FCF75EFC0006E3D456
:208BA00016A8FCF76AFC0006DED48AF8008010E04FF00109EFE713A8FCF708FB000602D547
:208BC000FCF7D0F857E5139818B905F0CBFE0006CAD48DF8488012A8FCF780F90006C3D4B0
:208BE0000B208DF8010013A8FCF7FCF90006BBD4BDF84C00ADF80A0013A8FCF7E2F900064D
:208C0000B2D41398CDF8060028798DF80C002888ADF802006888ADF804001598CDF80D00B7
:208C20001698CDF81100684603F070FC00069BD4B9F1000F07D02820C4F800B0306078469C
:208C40003860922017E5FCF71AF814E5FA020000F8B505464379394C39493A4A86200BB133
:208C6000022B02D92060072005E02B790BB11E2B06D9206005200860784610608620F8BD42
:208C80006988288801F0F4FB00063FD400270126009769463046FCF7F0F9000636D4761CB2
:208CA000F6B20B2EF5D36846FCF7FBF900062DD46846FCF718FA000628D46846FCF7CCF954
:208CC000000623D4ADF800706846FCF7FBF900061CD46846FCF718FA000617D42846FCF7F2
:208CE00088F9000612D4A81CFCF794F900060DD4281DFCF7A0F9000608D4012005F068FFAC
:208D0000000603D4FBF78EFF000601D52068F8BD02208DF800006846FCF738F9000607D484
:208D2000094901200870681DFCF7B8FB000602D5FCF718F8F8BDFBF7A2FFF8BD08C0072051
:208D40000CC0072010C0072000C007201CB5FBF769FF000602D5184800681CBD06F05AF851
:208D600000061ED400248DF800406846FCF70EF9000616D48DF8044001A8FCF78FFB000685
:208D80000FD46846FCF7D6F800060AD49DF8000002280ED18DF800406846FCF79FF80006FC
:208DA00004D505F058FDFBF7DDFF1CBD082025F056F8FBF764FF1CBD08C007202DE9F04FEC
:208DC000054600798B4C8C4E8C4F97B04FF086084FF0050B08B11E2804D9C4F80080C6F80A
:208DE00000B017E0288848F6AD614FF01409884205D900BFC4F80080C6F800900AE06888A9
:208E00004FF0170AB0F5B46F0AD300BFC4F80080C6F800A078463860862017B0BDE8F08F0D
:208E200002A8FCF7F0F8000613D42888BDF808108842DFD309D102A8FCF7F6F8000608D480
:208E40006888BDF808108842E0D3FBF7EBFE000601D52068E1E76846FCF72AFB00067CD4B5
:208E600002A8FCF703F9000677D4029898B103A99DF80000FCF735FC00066ED402A903A822
:208E8000FBF794FB000668D403A99DF80000FCF71BFC000661D403A99DF80000FCF737FC22
:208EA00000065AD4BDF80C0003A9401CADF80C009DF80000FCF71EFC00064ED40120804653
:208EC00002A9FCF7E6F8000647D40298A8B103AA41469DF80000FCF733FC00063DD402A955
:208EE00003A8FBF763FB000637D403AA41469DF80000FCF715FC00062FD408F10100C0B224
:208F000080460A28DCD903A90120FCF737F8000623D402A90120FCF7BCF800061DD49DF8B9
:208F200000004FF0880801280BD0022803D00220C4F800801DE002A903A8FBF7AAFC04E034
:208F40000BE002A903A8FBF76BFC000605D403A90120FCF707F8000602D5FBF703FF5CE7C5
:208F60009DF80000012809D002280AD00920C4F8008030607846386088204EE78DF815B0E4
:208F800002E006208DF8150002A8FCF72BF8000627D4BDF80800401CADF81E0002A8FCF7F5
:208FA00010F800061DD40298401CCDF81A0002A8FCF7EAF8000614D40298089010490DF1E7
:208FC000250026F0ADFB28798DF824002888ADF816006888ADF8180005A803F097FA000615
:208FE00002D505F038FCB8E7054900200870FBF746FE12E708C007200CC0072010C00720E4
:20900000BBC2072030B504460078504D95B008B10A280AD986204E49286004200860784646
:209020004C490860862015B030BDA0681190211D11A8FBF79CFC000603D4FBF7F3FD0006EC
:2090400001D52868EFE712A8FCF735F8000650D411A912A8FBF717FB00064AD412A8FCF787
:2090600020F8000645D412A8FCF736F8000640D4BDF84800401CADF8480012A8FCF722F8B7
:20908000000636D4207812A9FCF703F8000630D411A912A8FBF7F7FA00062AD4207812A9C7
:2090A000FBF7EBFF000624D412A8FBF7DFFF00061FD411A912A8FBF7E6FA000619D412A860
:2090C000FBF7CAFF000614D42046FCF72EF800060FD4201DFCF73AF800060AD404F108003C
:2090E000FCF73EF8000604D411A8FCF743F8000602D5FBF737FE96E705F01FFD00061ED4F8
:2091000013A8FBF74DFF000619D49DF84C00022803D105F093FE000611D49DF84C00012809
:2091200010D109208DF8010020788DF802001198CDF80300684603F0E9F9000602D505F0BA
:209140008AFBD6E7FBF79BFD6DE7000008C007200CC0072010C0072030B504460078474DDB
:2091600093B008B10A280AD986204549286004200860784643490860862013B030BDA06886
:209180001190211D11A8FBF7F2FB000603D4FBF749FD000601D52868EFE712A8FBF78BFFCB
:2091A000000650D411A912A8FBF78DFA00064AD412A8FBF776FF000645D412A8FBF78CFFFD
:2091C000000640D4BDF84800401CADF8480012A8FBF778FF000636D4207812A9FBF759FF5F
:2091E000000630D411A912A8FBF76DFA00062AD4207812A9FBF741FF000624D412A8FBF765
:2092000035FF00061FD411A912A8FBF75CFA000619D412A8FBF720FF000614D42046FBF761
:2092200084FF00060FD4201DFBF790FF00060AD404F10800FBF794FF000604D411A8FBF715
:2092400099FF000602D5FBF78DFD96E705F082FC00060DD40A208DF8010020788DF8020077
:209260001198CDF80300684603F050F9000602D505F0F1FAE7E7FBF702FD7EE708C00720C3
:209280000CC0072010C0072030B5044600784A4D93B008B10A280AD98620484928600420B2
:2092A0000860784646490860862013B030BDA0681190211D11A8FBF75AFB000603D4FBF785
:2092C000B1FC000601D52868EFE712A8FBF715FF000650D411A912A8FBF7D5F900064AD45D
:2092E00012A8FBF700FF000645D412A8FBF716FF000640D4BDF84800401CADF8480012A8C9
:20930000FBF702FF000636D4207812A9FBF7C1FE000630D411A912A8FBF7D5F900062AD404
:20932000207812A9FBF7A9FE000624D412A8FBF79DFE00061FD411A912A8FBF7C4F90006DA
:2093400019D412A8FBF788FE000614D42046FBF7ECFE00060FD4201DFBF7F8FE00060AD4CC
:2093600004F10800FBF7FCFE000604D411A8FBF701FF000602D5FBF7F5FC96E705F0F7FB57
:20938000000612D410208DF8010012A8FBF793FE00060AD41298CDF802001198CDF8060025
:2093A000684603F0B3F8000602D505F054FAE2E7FBF765FC79E7000008C007200CC00720E3
:2093C00010C00720F0B599B0044616A816F0B7FF2179CB4DCB4ECC4F862009B11E2902D97C
:2093E000286005200DE0218848F6AD62914202D92860142005E06188B1F5B46F07D328607A
:209400001720306078463860862019B0F0BD18A9022003F0FBFE00061FD4BDF8600058B12D
:2094200025F0FFF8000618D402F0BFFF000614D49DF8580040B10CE0912028608A20306053
:20944000784638609120E0E7012005F0C1FB000603D4FBF7E7FB000601D52868D5E701256D
:20946000ADF8545015A91A20FCF713FA00067CD402A8FBF794F90006F9D400201790ADF8ED
:2094800054002846C0B2064602A9FCF718F80006EDD402A93046FCF767FA0006E7D415A9E3
:2094A0003046FCF722F80006E1D415A93046FCF732F80006DBD415A93046FCF750F90006F2
:2094C000D5D415A93046FCF760F90006CFD48DF8045000BF9DF8041002AA3046FCF731F83B
:2094E0000006C4D49DF8041017AA3046FCF748F800063AD49DF80400401CC0B28DF80400B7
:209500001028E7D902A93046FCF753F800062CD402A93046FCF763F8000626D48DF80450A6
:209520009DF8041002AA3046FCF76FF800061CD49DF80400401CC0B28DF804000A28EFD926
:209540008DF804509DF8041002AA3046FCF77CF800060AD49DF80400401CC0B28DF804002C
:209560001828EFD98DF8045000E081E09DF8041002AA3046FCF789F8000679D49DF804009E
:20958000401CC0B28DF804001E28EDD98DF804509DF8041002AA3046FCF734FA000667D462
:2095A0009DF80400401CC0B28DF804000528EFD98DF804509DF8041002AA3046FCF741FAF4
:2095C000000655D49DF80400401CC0B28DF804001028EFD9761CF0B204287FF653AF2E4621
:2095E000F0B2064602A9FCF76FF8000640D415A93046FCF77FF800063AD48DF8045000BF14
:209600009DF8041002AA3046FCF78AF800062FD49DF80400401CC0B28DF804000A28EFD917
:20962000761CF6B2022EDBD901F02CF800061FD42046FCF7C0F800061AD4A01CFCF7CAF888
:20964000000615D4201DFCF7D6F8000610D48DF8045001A8FBF742FC000609D49DF85800B1
:2096600001284AD001A92B200DF0EAF9000602D5FBF778FBC9E69DF80400C00701D16079D6
:2096800090B101A8FBF79DFC000633D401A8FBF702FA00062ED401A8FBF789FC000629D486
:2096A00005F0C0F8000625D418490220087011208DF8110001A9042003F058FB000619D435
:2096C000BDF80400401CADF8120020798DF81C002088ADF814006088ADF8160001A8FBF7E5
:2096E00070FC000606D40198069004A802F00EFF000602D505F0AFF8BAE7FBF7C0FA84E614
:2097000008C007200CC0072010C0072000C00720F8B505460379384C3849394A86200BB12B
:209720001E2B02D9206005200EE02B8848F6AD671426BB4202D920600E6006E06B88B3F5EC
:20974000B46F06D3206017200860784610608620F8BD2C490120FBF7BFFE000640D42A4993
:209760000220FBF7B9FE00063AD42846FBF741FC000635D4A81CFBF74DFC000630D4281D10
:20978000FBF759FC00062BD4002568460095FCF7B8F8000624D468460095FCF7C3F800067D
:2097A0001ED48DF800606846FCF762F8000617D40120ADF800006846FCF781F800060FD41D
:2097C00069461C200DF03CF9000609D49DF8000040B1ADF800506846FBF7FAFB000601D59D
:2097E0002068F8BD032009498DF80000022008706846FBF7CBFBF8BD08C007200CC007209B
:2098000010C00720460000104B00001000C007207CB5FBF707FA000602D51C4800687CBDB3
:209820006846FAF7C8FF000624D401263446E0B205466946FBF796FB00061BD46D1CECB2F8
:209840000B2CF4D3002468460094FBF7B0FB000610D4ADF800406846FBF7BAFB000609D400
:20986000ADF800600220C0B204466946FCF711F8000604D504F0EFFFFBF774FA7CBD641C80
:20988000E0B21A28EFD9FBF7FAF97CBD08C00720FEB56846FAF783FF284C000640D4002796
:2098A0000125ADF808702E46F0B206466946FBF706FE000634D402A93046FBF716FE000623
:2098C0002ED402A93046FBF726FE000628D402A93046FBF744FF000622D402A93046FBF7E8
:2098E00054FF00061CD469463046FBF762FE000616D469463046FBF772FE000610D4761CB5
:20990000F6B2042ED0D9E8B205466946FBF7DCFE000605D402A92846FBF7ECFE000601D5B4
:209920002068FEBD6D1CEDB2022DECD90448276007607846034908600020FEBD08C0072052
:209940000CC0072010C007207CB506466846FAF726FF0D4D000607D401246A4631462046EF
:20996000FBF772FE000601D528687CBD641CE4B2052CF2D30549002028600860784604496B
:20998000086000207CBD000008C007200CC0072010C007207CB506466846FAF700FF0D4DB8
:2099A000000607D401246A4631462046FBF76DFE000601D528687CBD641CE4B2052CF2D306
:2099C000054900202860086078460449086000207CBD000008C007200CC0072010C0072084
:2099E000FEB507466846FAF7DAFE114D000610D40026012402966A4639462046FBF7A1FDA0
:209A0000000606D402AA39462046FBF7B9FD000601D52868FEBD641CE4B2052CEBD30548B4
:209A20002E6006607846044908600020FEBD000008C007200CC0072010C007202DE9FC41B8
:209A400007466846FAF7ABFE144E000615D401252C46E0B204466A463946FBF7D6FD0006B2
:209A60000BD4641CE4B2052CF3D3E8B204466A463946FBF755FE000602D53068BDE8FC810B
:209A8000641CE5B2032DF0D305490020306008607846044908600020F0E7000008C00720FD
:209AA0000CC0072010C007202DE9F04F97B007464FF000098A4681F80090052001F0A8FCF8
:209AC000FE4C00067ED4FF2003F0CCF90006F9D415A8FCF7DFF90006F4D46946002003F022
:209AE00088F80006EED4BDF80000F54DF54E4FF09008192803D30120C4F80080E0E0F2489F
:209B00000DF12C0B0078002874D06946012003F070F80006D6D4BDF80000402803D303203B
:209B2000C4F80080CCE014A9002001F0D9FB0006C8D49DF85000410903D00420C4F8008097
:209B4000BEE001070BD5410709D4872020607846C5F800903060872017B0BDE8F08FC00640
:209B600003D501F087F90006ACD403A9052001F0B7FB0006A6D46946032003F0F7F8000668
:209B8000A0D42068052805D0052203A9684625F09BFDD8B19DF8500000077DD56946002003
:209BA00003F0E4F800068DD403A90B2001F098FB000687D40C2203A9684625F085FD48B19B
:209BC000052000E0ABE0C4F8008079E00720C4F8008075E003A90C2001F082FB000699D4EF
:209BE0000622B91D03A825F06FFD20B10620C4F8008065E07CE003A9112001F071FB000627
:209C000088D40622394603A825F05EFD18B10820C4F8008054E069460E2001F061FB000695
:209C20007DD403A800F08EFC000678D4BDF80000BDF80C10884208D95D200BF0DFFB0006D3
:209C40006DD40920C4F800803AE003A9F6F728FE9DF80C00694600F5FA60ADF82C009DF880
:209C60000D008DF82E009DF80E008DF82F000F2001F036FB000652D4BDF800103C22B1FB81
:209C8000F2F08DF8300002FB10108DF831008DF8329003A9102000E025E001F021FB00063F
:209CA0003DD46946042003F061F800067ED4BDF80000BDF80C10884207D00A20C4F800808F
:209CC000286078463060902046E76946062001F007FB00066AD4BDF80C00BDF80010401CE3
:209CE0008142EAD10FE001F0A8FB00287FF46EAF0BF104001CF0DEFF000657D40BA81DF0D1
:209D00000EF8000652D402F067FB00064ED40BF10701002003F02AF8000647D400E045E036
:209D2000D7F80600CDF83F007889ADF843003868CDF84500B888ADF8490013A9042003F0B6
:209D400015F8000632D4D7F8060007907889ADF820003868CDF82200B888ADF82600F868C6
:209D60000A9006A90BA8F6F732FEBDF84C00ADF81A0006A8FBF73DF9000617D49DF830106E
:209D80009DF83100C1EB011100EB8100ADF800006846FBF73FF9000608D44C48FBF74BF9AA
:209DA000000603D4FAF73EFF000601D52068D3E604F033FF00066CD406A804F043FF000625
:209DC00067D49DF85000000707D43F48007820B10BA801F040FB00065BD4DFF8EC80012732
:209DE0008AF8007098F80000D8B101F0DCFD00064FD40121364804F053FF00060AD5F6F7AD
:209E00000FFA01F037F8F6F720FA04F024FDFAF7A9FFCBE701F0F9FD00063AD42068002807
:209E2000E7D0112003F0A8F9000632D406A9002003F0B2F900062CD498F8000058B107A9DE
:209E4000052001F04DFA000623D406A9012003F0A3F900061DD4122003F08EF9000618D4B4
:209E60009DF85400D0B16846FBF7ABF8000610D46846FAF710FE00060BD46846FBF797F88A
:209E8000000606D44F468AF80090FAF7F8FE000653D504F0E0FCFAF765FF5DE68DF80070C9
:209EA0006846FCF710F80006F3D4ADF81090CDF80C908DF81290B84638460BE008C0072009
:209EC0000CC0072010C00720FA02000085C00720B80200108DF80070C0B203A9FBF742F827
:209EE0000006D6D49DF80000401CC0B28DF800000A28F1D94F4603A8CDF80C90FBF757F8EC
:209F00000006C6D4ADF80C7003A8FBF761F80006BFD44046ADF80C808DF80080C0B203A917
:209F2000FBF7B7FC0006B4D49DF80000401CC0B28DF800001A28F1D9A4E7276078462F609B
:209F40003060002008E600002DE9F04796B0002180460170052001F05BFAAC4C00067AD4C1
:209F6000FF2002F07FFF0006F9D46946012002F040FE0006F3D4BDF800009027A44DA54E62
:209F8000402802D30320276043E00FA9002001F0A7F90006E3D49DF83C004FF0020A00096C
:209FA00009D0922020607846C5F800A03060922016B0BDE8F08703A9052001F091F9000605
:209FC000CDD46946032002F0D1FE0006C7D420684FF0070928B90522694603A825F074FBEF
:209FE000C8B19DF83C0000077ED56946002002F0BDFE0006B3D403A90B2001F071F900067C
:20A00000ADD40C2203A9684625F05EFB50B105202760286002E02760C5F800907846306090
:20A020009020C5E769460E2001F05AF9000696D403A800F087FA000691D4BDF80000BDF842
:20A040000C10884208D05D200BF0D8F9000686D409202760DDE7ABE06946042002F086FE51
:20A06000000687D403A9102001F03AF9000691D4BDF80000BDF80C104FF00A098842CAD1D7
:20A080006946062001F02CF9000699D4BDF80C00BDF80010401C8142BDD103A90C2001F066
:20A0A0001FF900068CD46946012002F05FFE00067ED40622694603A825F006FB10B106202C
:20A0C0002760A6E703A9112001F00AF900066FD46946022002F04AFE000669D4062203A930
:20A0E000684625F0F1FA00E003E030B1082027608FE701F0A2F900288DD106AD281D1CF0D3
:20A10000D9FD000679D406A81CF009FE000674D4E91D002002F02AFE00066ED40DF12B0155
:20A12000012002F023FE000667D40DF13101022002F01CFE000660D40EA9042002F016FE31
:20A1400000065AD4BDF83800ADF8420010A906A8F6F73DFC11A9052001F0C2F800064CD4BA
:20A16000FAF760FD000648D404F07EFD00063BD49DF83C00000704D406A801F06CF9000631
:20A1800032D4012188F8001001F00DFC00062BD4214D0121204804F083FD00060CD5F6F7C8
:20A1A0003FF800F067FE00061ED4F6F74EF800E023E02068000617D401F027FC000613D48B
:20A1C00095F840000028E4D1112002F0D5FF00060AD410A9012002F0DFFF000604D4122040
:20A1E00002F0CAFF000604D504F035FBFAF7BAFDDEE6FAF744FD000601D52068D8E688F861
:20A2000000A0012004F0E4FCD2E6000008C007200CC0072010C00720B80200102DE9F04305
:20A220008BB007A901201CF055F8594C000645D4684600F0ACFF0006F9D408A9032002F013
:20A2400095FD544DDFF85081000616D40027052208A903A825F038FA80B13D200BF0CEF8F3
:20A2600000062BD4922020603120794628609220C8F800100BB0BDE8F08301279DF81100EC
:20A280004FF0000641074FF0870903D4C4F800902E606DE0400654D506A8FAF73AFE000618
:20A2A00074D49DF818000E2801D0002FEED05A200BF0A4F8000602D504F0CDFA66E001F0D5
:20A2C000BCF8000662D4684600F03CF900065DD40DF1020000F01AF9000657D41E208DF88D
:20A2E0000400684601F02FF900064FD48DF800606846FAF7F3FD000648D4684600F0D9FE5F
:20A30000000643D4BDF80000401E80B201F014FB00063BD4214D0121204804F0C1FC000617
:20A3200006D5F5F77DFF00F0A5FDF5F78EFF2DE001F06BFB000629D495F840000028EAD1B8
:20A340001BE00798C00707D08DF800606846FAF7C5FD00061AD410E06846FAF7C9FD000630
:20A3600014D49DF8000040B10420C4F80090286079468720C8F800107CE72F200BF03EF85E
:20A38000000603D401F036F9000695D4206871E708C007200CC0072010C00720B8020010CE
:20A3A00038B5FAF73FFC104D000617D400248DF800406846FAF7EFFE000606D48DF800401C
:20A3C0006846FAF7E3FD000602D5FAF7CBFC38BD68460094FAF7F0FE000601D5286838BDF2
:20A3E000FAF74DFC38BD000008C007201CB5FAF719FC000602D51D4800681CBD01A8FBF74A
:20A4000057F800062CD46846FAF7DBFD000627D46846FAF740FB000622D46846FAF7C7FD36
:20A4200000061DD46846FAF7DDFD000618D46846FAF70BFB000613D46846FAF7C9FD0006BD
:20A440000ED400248DF8044001A8FBF727F8000606D48DF800406846FAF798FD000602D5BD
:20A46000FAF780FC1CBDFAF70AFC1CBD08C007202DE9FC5F944D954E954C070089464FF0AC
:20A4800086084FF0140A03D048F6AD60874204D9C4F80080C5F800A008E04FF0170BB9F57D
:20A4A000B46F08D3C4F80080C5F800B0784630608620BDE8FC9F01A8FBF786F900060CD4C1
:20A4C000BDF804003F1A4FF4B4604743002FDFDB6846FBF789F9000601D52068E9E7BDF895
:20A4E0000010A9EB0100C019DCD40021B0F5B46F06DB8A2020607846296030608A20D8E7FA
:20A5000021607846296030600020D2E738B5044668461CF0CFFB01066D4801D5006838BD60
:20A520009DF800209DF80110C2EB021201EB8201218000210160644801607846634908608E
:20A54000002038BD38B5044668461CF0E8FB000602D55F48006838BD21466846F6F737FAFE
:20A5600038BD1CB56846FFF7D1FF594C000604D401A8FFF7E7FF000601D520681CBDBDF8A7
:20A580000010BDF80400FFF773FF4F494F4A38B191202060882008607846106091201CBD77
:20A5A0000020206008607846106000201CBD2DE9FE43DFF820818146434E98F80000434F23
:20A5C000434C002510B188F8005055E002A93D200CF001FB000644D49DF80800F0B3012181
:20A5E00088F800106846FFF791FF000639D401A8FFF7A8FF000634D4BDF80400BDF80010B2
:20A60000C0EB001000EB400001EB40186846FBF799FA000625D401A8FBF783FA000620D4CC
:20A62000BDF80400BDF80010C0EB001000EB400001EB40109DF80810C1EB011100EB8101A2
:20A64000414519D8B9F1000F0ED05C200AF0D6FE000606D4012004F0BBFA00E00CE0000626
:20A6600002D52068BDE8FE838720206005203060784638608720F5E7256078463560386030
:20A680000020EFE71CB56846FFF740FF104C00060ED401A8FFF756FF000609D401A8FBF75A
:20A6A00036FA000604D46846FBF742FA000601D520681CBD04490020206008607846034914
:20A6C000086000201CBD00000CC0072010C0072008C007202AC0072010B594B00446FAF7EB
:20A6E000A1FA000603D52548006814B010BD201DFBF750F9000617D404F10800FBF75BF9CF
:20A70000000611D4207A11A9FBF773F900060BD4211D11A8F9F7B7FF000605D4207A11A9E7
:20A72000FBF75AF9000602D5FAF71CFBDDE712A94B200CF085F9000619D49DF84800C007F4
:20A7400003D004F021FA000611D49DF84800800710D512208DF80100207A8DF80200606842
:20A76000CDF80300684601F0D1FE000602D504F072F8D9E7FAF783FAB7E7000008C00720AD
:20A7800010B594B00446FAF74DFA000603D52548006814B010BD201DFBF7FCF8000617D4D6
:20A7A00004F10800FBF707F9000611D4207A11A9FBF71FF900060BD4211D11A8F9F783FF13
:20A7C000000605D4207A11A9FBF706F9000602D5FAF7C8FADDE712A94B200CF031F90006AF
:20A7E00019D49DF84800C00703D004F0DAF9000611D49DF84800800710D513208DF8010041
:20A80000207A8DF802006068CDF80300684601F07DFE000602D504F01EF8D9E7FAF72FFAAC
:20A82000B7E7000008C0072070B596B0002604468DF84C604079944DA0B113A8FAF74AFDA1
:20A8400000067DD49DF84C0008B110280AD986208E4928600320086078468D4908608620BA
:20A8600016B070BDFAF7DEF90006EAD46079002851D011A8FAF7AAFC00064BD4A079214642
:20A88000002811A83ED0F9F71EFF000642D411A8FAF792FC00063DD411A99DF84C00FAF7C5
:20A8A000CAFC00067DD4A0792146002811A82CD0F9F709FF000674D411A99DF84C00FAF74C
:20A8C000AEFC00066DD413A8FAF771FD000668D42046FAF75BFD000663D4207911A9FBF7FA
:20A8E000DCF800065DD4214611A8F9F7CCFE000657D4207911A9FBF7C3F8000651D404F023
:20A900009AF864E0F9F7BFFEBFE7F9F7BCFED1E703F0A1FF45E012A8FAF758FC000640D4DB
:20A9200012A8FAF788FD00063BD412981190A0792146002811A837D0F9F7C5FE000600E086
:20A9400091E02ED411A8FAF737FC000629D42046FAF760FD000624D4A079002811A826D002
:20A96000FAF797FC00061CD4214611A8F9F78BFE000616D411A8FAF783FC000611D4207927
:20A9800011A9FBF78AF800060BD4214611A8F9F77AFE000605D4207911A9FBF771F8000689
:20A9A00013D5FAF7DFF95BE7F9F76DFEC6E7FAF780FC0006F5D4214611A8F9F764FE0006E8
:20A9C000EFD411A8FAF76BFCD7E704F041F800069ED411A8FBF75EFA000644D49DF8440046
:20A9E00060B12C48007848B120681490A079002814A826D001F0F5F8000689D411A94C20DB
:20AA00000CF01EF800062ED49DF84400800738D5A079C8B15FF008008DF8010020798DF822
:20AA200006006179684689B1CDF80260C01DFAF795FC0006CCD411A8FAF7A1FC0006C7D43A
:20AA400013E001F025F9D7E70720E5E71299CDF80210C01DFAF7C6FC000604D411A8FAF7A9
:20AA6000D2FC000601D52868FAE6BDF84400ADF808002068CDF80A00684601F047FD0006D6
:20AA8000A6D4FAF7FCF8EBE608C007200CC0072010C00720FA02000071B581B0FAF7C2F8AF
:20AAA000394C00063CD403208DF800006846FAF76DFA000662D419208DF800006846FAF7B4
:20AAC000D7FE00065AD431490220087001A91920FAF7DFFE000623D4012004F079F800061F
:20AAE0004CD401F0D8FE000648D4BDF8040001F046FE000642D420680025052807D0244E20
:20AB000001F016FF000639D42068D8B913E0FAF729F9000604D4012020F03BF9000601D5DE
:20AB200020687CBD812020601A48056078461A49086081207CBD7078062803D0052801D022
:20AB40000B28DDD120F030FB000617D4012020F020F9000612D4012004F03AF800060DD484
:20AB60008DF800506846FAF711FA000606D48DF800506846FAF77CFE000602D5FAF7F2F8D0
:20AB80007CBDFAF77CF87CBD08C0072000C0072079C207200CC0072010C007202DE9FE4365
:20ABA0004A4C884610B3FBF745F940B1F5F738FB002147A020F09DF9F5F747FB7AE00220D6
:20ABC0008DF8080002A8FAF79AF9000672D40120ADF80400054601A92846FAF75AFE0006F2
:20ABE00068D46D1C1A2DF6D901F0F6FB3F4F0422694638461CF0E1FD00065BD43C4E009876
:20AC00000025B04227D004226946381D00951CF0DFFD00064ED435480422694608301CF0C1
:20AC2000D7FD000646D43148042269460C301CF0CFFD00063ED42D480422694610301CF010
:20AC4000C7FD000636D404226946384600961CF0BFFD00062ED4254804226946143000954C
:20AC60001CF0B6FD000625D420480422694618301CF0AEFD00061DD41C48042269461C305E
:20AC80001CF0A6FD000615D418480422694620301CF09EFD00060DD440460CF091FB0006EF
:20ACA00008D400200BF082FE000603D4F6F793F8000602D52068BDE8FE830E4825600560FD
:20ACC00078460D4908600020F5E7000008C007208EE8A8A1AAA020A8ADA8E6A8A0ABA8A7BF
:20ACE000A0E6A8A8204652414D0A000004000040CEFAADDE0CC0072010C007202DE9F04166
:20AD000088B05348F9F757FD5248F9F754FD05A8FBF7C0F8504C000639D49DF814004F4EF5
:20AD20004F4F00254FF00508A0B106A912200BF087FE00062BD407A8FAF7A4FD000626D40C
:20AD40009DF81800C10705D09DF81C100E290AD0142908D0C4F80080784635603860052076
:20AD600008B0BDE8F081800713D5002001F0DFFF00060CD46946002001F09DFF000606D485
:20AD8000BDF80210022001F0BCFF000603D52068E6E70021F6E7256078463560386000205D
:20ADA000DEE72DE9F04788B000262B4CDFF8B0902A4FB0466D460DF1090A6946022001F0A0
:20ADC0007AFF20B105280FD0932832D12EE0291D2048F9F792FD00062BD451461C48F9F734
:20ADE0008CFD000625D426E005A90120FAF774FB00061ED405A91748F9F77FFD000618D433
:20AE000005A90220FAF768FB000612D405A91048F9F773FD00060CD4052020607946C7F8B3
:20AE20000080C9F8001008B0BDE8F0873868082801D02068F7E7761C642EBEDBC4F80080ED
:20AE40007946C7F800800020C9F80010EBE7000043C007203CC0072008C007200CC0072002
:20AE600010C00720FE48002141708170C17001201BF0BABB1CB506208DF80000F9480178CA
:20AE8000012059B1F649002201AB4A708A708DF80400012168461BF042FB1CBDF24A882167
:20AEA0001160F24908607846F149086088201CBD2DE9FC410546002005218DF80410E949EE
:20AEC0008DF80000E94E0978E94FE74C81B1E4496B46E84A4870012101A81BF020FB0006D9
:20AEE0000FD5F5F79DF9FFF7C5FFF5F7AEF913E08820206001203060784638608820BDE830
:20AF0000FC8125B19DF800006D1EA84206D1D9499DF8000081F840002068F0E792202060FC
:20AF200020203060784638609220E8E72DE9FF5F24208DF8080003A9002000F0D1F9CA4D88
:20AF400000067DD49DF80C00C84EC94F00074FF0920804D42620C5F80080306048E04FF099
:20AF6000000B8DF804B001ABC24A012102A81BF0D6FA00067AD41920FFF79AFF000675D4C3
:20AF8000BC484FF027090178072902D0FFF772FF2AE0D0F80110C0F86E10D0F80510C0F8AE
:20AFA0007210DFF8D0A2D0F80910C0F876100AF1800AD0F80D20CAF80020427C8AF80420E7
:20AFC000D0F81210C0F87A10C18A0446A0F87E100F20FFF76DFF000648D4FFF74BFF000691
:20AFE00044D42078082809D0C5F80080C6F8009078463860922004B0BDE8F09FD4F806103B
:20B00000CAF80C106189AAF81010DFF86882607B217B08F1440800EB0120A8F8460060785F
:20B0200000F00F01000900EB800001EB40008DF80000A07800F00F01000900EB800000E07F
:20B0400014E001EB40008DF80100E07800F00F01000900EB800001EB40008DF8020008F1D2
:20B0600042016846F5F764FC000601D52868C2E7607900F00F01000900EB800001EB400104
:20B08000207900F00F02000900EB800002EB4000C0EB001001EB8001A8F84410704901207F
:20B0A000C870C5F800B07846C6F800B038600020A1E72DE9F0438BB0054639208DF82000B2
:20B0C0006DA04FF000080068674C684E1B27C146CDF824008DF81C7007AB6A46022109A8D2
:20B0E0001BF01DFA90B1306805283AD2B8F1000F37D18DF81C9007AB6A46012108A81BF0EC
:20B100000EFA00062DD44FF00108E3E79DF801009DF80010052300EB012028800622A91C0A
:20B120000DF10200F5F736FB00061AD405230622E91D02A8F5F72EFB000612D405230622AD
:20B1400005F10C010DF10E00F5F724FB000608D40523062205F1110105A8F5F71BFB0006E6
:20B1600003D520680BB0BDE8F083424816222946583024F018FB3A4901208870C4F80090D4
:20B1800078463B49C6F8009008600020EAE72DE9F04389B0044639208DF81C0037A04FF0EA
:20B1A00000080068304D314E1527C146CDF820008DF8187006AB6A46022108A81BF0AFF907
:20B1C00090B1306805286ED2B8F1000F6BD18DF8189006AB6A46012107A81BF0A0F900062C
:20B1E00061D44FF00108E3E79DF8050000F00F01000900EB800001EB40008DF814009DF8A0
:20B20000060000F00F01000900EB800001EB40008DF815009DF8070000F00F01000900EB5E
:20B22000800001EB40008DF81600211D05A8F5F77FFB9DF8090000F00F01000900EB800064
:20B2400001EB40019DF8080000F00F02000900EB800002EB4000C0EB001001EB80000FE06C
:20B2600035000010FA02000008C007200CC0072010C00720B80200100702000007010000D9
:20B28000E0800423052221466846F5F783FA000609D404231A4604F108010DF10A00F5F726
:20B2A00079FA000602D5286809B05CE7DDF80E00E0609DF8120020749DF8130060741422A2
:20B2C0002146F94824F0F6FAF84901204870C5F800907846F649C6F8009008600020E3E7BE
:20B2E0002DE9F0410546F148F24E0C46052D05DC4078A0B9EC48FFF74AFF07E00A2D0ADC56
:20B30000807860B9E8481430FFF7D3FE000606D53068BDE8F081112D01DCC078A0B1E24884
:20B32000E54BDFF88CC3A0F1440100F13C02122D65D2DFE805F00C0F1114181B2022292F73
:20B34000343A444A4E525558FFF7F0FDDEE7407C20704CE0486C07E0B1F8480001E0B1F86E
:20B360004A00208043E0C86C206040E0086D206091F8540006E0808A2DE0D1F85A0020607A
:20B3800091F85E00207132E0D1F85F00206091F86300F7E7486E206091F86800F2E7D1F8E8
:20B3A0006900206091F86D00ECE7D1F86E002060D1F872006060D1F87600A06017E0D1F82A
:20B3C0007A002060B1F87E0010E0106820601079D8E7B0F84200208009E0B0F84400FAE7DC
:20B3E000B0F84600F7E7D0682060108AA0800020306018607846CCF80000002089E7922023
:20B400003060252018607846CCF80000922080E7A64AC3074FF0000100D05170830700D55A
:20B420009170400700D5D170A2480160A248016078469F490860002070471CB501208DF8BC
:20B4400000009EA06B46006801900022022101A81BF065F81CBD30B597B0044608208DF8B2
:20B460004C00974801250078E8B3202249216846F4F7BCFF8DF8005021889248085C8DF827
:20B480000100A1789048415C8DF80210E178415C8DF803102179415C8DF804106179405CB2
:20B4A0008DF80500D4F80700CDF80600D4F80B00CDF80A00D4F80F00CDF80E00D4F8130031
:20B4C000CDF81200B4F81700ADF81600D4F819000690B4F81D00ADF81C00208C000A8DF8D7
:20B4E0001E00208C00E008E08DF81F007748C1896E4828290CD210210BE06E498820086045
:20B500006D48056078466A490860882017B030BD28210170C9B28DF820106DA22131136816
:20B52000CDF821305268CDF8252032228DF82920002242708270C270C9B213AB14AA684672
:20B540001AF0EDFFE2E77FB504465D480125007858B309208DF80000208802A9F5F7A0F9DA
:20B560009DF808105848415C8DF801109DF80910415C8DF802109DF80A10405C8DF8030096
:20B58000608801A9F5F7CEFA20798DF80600474900200246487088708DF80C5003AB0721E2
:20B5A00068461AF0BCFF04B070BD4249882008604148056078463E4908608820F3E71CB5AE
:20B5C000012039218DF804103D498DF80000097831B16B460022012101A81AF0A0FF1CBDC9
:20B5E000344A882111603449086078463049086088201CBD1CB501200A218DF8041030497F
:20B600008DF80000097851B1284900200246487088706B46012101A81AF081FF1CBD254A4B
:20B62000882111602449086078462149086088201CBDFEB50E46002521218DF800108DF882
:20B64000085004230DF101022946F5F761F8194C000627D4144A02AB443A052168461AF0E9
:20B660005EFF00061ED4104F3560443F0020FFF71FFC000616D4206848B10F480C49326816
:20B6800062B325600560784608600020FEBD39780B29EBD1042303223146781DF5F77AF853
:20B6A0000006E3D52068FEBDFC0200103500001010C0072008C007200CC007200801000054
:20B6C000FA020000F6090300C6110300F0CD0720465072696E742D3232000000FFE7922230
:20B6E000226027220260784608609220FEBD2DE9FC41F749F74FDFF8E0830978F74EC9B137
:20B70000A0218DF80010010AF54C8DF801108DF8020000256570207801AB401C8DF8040047
:20B72000F04A032168461AF0FAFE00060BD53068BDE8FC8188203060012079463860882003
:20B74000C8F80010F4E7E748217880F840104554356079463D600020C8F80010E8E72DE94F
:20B76000FE43DB49DB4FDFF870830978DB4EE1B1A1218DF8001004230DF101020021F4F7A9
:20B78000C7FF00060ED4D64C002502AB65702078D44A401C8DF80800052168461AF0BFFEF8
:20B7A00000060BD53068BDE8FE83882030600120794638608820C8F80010F4E7C948217838
:20B7C00080F840104554356079463D600020C8F80010E8E72DE9FF410F46BD49BD4EDFF8C5
:20B7E000F8820978BD4D29B1A2218DF804105AB104210AE0882028600120794630608820AC
:20B80000C8F8001004B084E505218DF805106946F5F746F89DF80000B34C6946205C8DF85E
:20B8200006009DF80100205C8DF807009DF80200205C8DF808003846F5F732F89DF800009B
:20B84000002703AB205C8DF809009DF80100A54A0821205C8DF80A009DF80200205CA04C51
:20B860008DF80B0067702078401C8DF80C0001A81AF055FE000601D52868C3E79948217846
:20B8800080F8401047542F60794637600020C8F80010B7E72DE9FE438D4B8E4D8E4E1B7859
:20B8A0008E4C6BB142F20F73984201D899420FD9862020601320286078463060862072E738
:20B8C00088202060012028607846306088206AE7A2238DF800300AB1062200E007228DF865
:20B8E0000120020A8DF802208DF80300080A7C4F8DF804008DF805104FF0000887F80180A5
:20B90000387802AB401C8DF80800764A062168461AF005FE000601D5206844E771493A7844
:20B9200081F8402001F80280C4F800807846C5F800803060002036E72DE9FC416449654FFB
:20B94000DFF894810978654EC1B1A3218DF80010010A634C8DF801108DF80200002565702B
:20B96000207801AB401C8DF804005E4A032168461AF0D5FD00060AD53068D9E688203060D4
:20B980000120794638608820C8F80010D0E65548217880F840104554356079463D60002059
:20B9A000C8F80010C4E62DE9FC41A4208DF804004748484FDFF820810078484E80B1484CFC
:20B9C00000256B4665702078464A401C8DF80000012101A81AF0A3FD00060AD53068A7E634
:20B9E000882030600120794638608820C8F800109EE63C48217880F84010455435607946C9
:20BA00003D600020C8F8001092E62DE9FC4105208DF804002E482F4EDFF8BC8000782F4C27
:20BA200098B12F4F00256B467D708DF800502D4A012101A81AF073FD00060FD5F4F7F0FB2B
:20BA4000FFF718FAF4F701FC12E0882020600120794630608820C8F8001069E69DF8000010
:20BA600010B13978884205D11E4981F840000D5420685DE6922020602020794630609220F5
:20BA8000C8F8001054E62DE9FF4104461048134D114902780F48012782B12278012A14D015
:20BAA000022A23D0032A3AD0042A3AD086222A6006220260784608608620A3E688222A60B3
:20BAC00007607846086010469CE610200FE00000FA0200000CC0072010C0072008C007200D
:20BAE00035000010B8020010C611030011208DF80000207B8DF801006E460423B21C0021BC
:20BB00006068F4F705FE000607D40523B21D0021A068F4F7FDFD000605D5286872E612208F
:20BB2000E5E71320E3E7FF4900206A46487088708DF80C7003AB0B2110461AF0F0FC61E606
:20BB40002DE9FF410446F848F84DFA490278F84801279AB118228DF800202278012A14D0C8
:20BB6000022A14D0032A2BD0042A2BD086222A600622026078460860862043E688222A607F
:20BB800007607846086010463CE6102000E011208DF80100207B8DF802006E460423F21CCE
:20BBA00000216068F4F7B4FD000607D40523F21D0021A068F4F7ACFD000605D5286821E6B4
:20BBC0001220E5E71320E3E7D64900200246487088708DF80C7003AB0C2168461AF09FFC04
:20BBE00010E63EB5D049D14C0125097869B116218DF80010006805230DF101020021F4F7FC
:20BC000087FD00060AD520683EBD88202060C84805607846C749086088203EBDC149002098
:20BC20000246487088708DF8085002AB062168461AF075FC3EBD3EB5BB49BC4C0125097891
:20BC400081B118218DF8001016218DF80110006805230DF102020021F4F75AFD00060AD53D
:20BC600020683EBD88202060B14805607846B149086088203EBDAB490020024648708870EC
:20BC80008DF8085002AB072168461AF048FC3EBD3EB5A549A54C0125097869B117218DF8AB
:20BCA0000010006805230DF101020021F4F730FD00060AD520683EBD882020609C480560D1
:20BCC00078469C49086088203EBD964900200246487088708DF8085002AB062168461AF056
:20BCE0001EFC3EBD3EB59049904C0125097881B118218DF8001017218DF801100068052382
:20BD00000DF102020021F4F703FD00060AD520683EBD88202060864805607846854908605E
:20BD200088203EBD7F4900200246487088708DF8085002AB072168461AF0F1FB3EBD2DE919
:20BD4000F041044678487A4E7A4F0078774D86B08846E8B3208802A9F4F7A2FD19208DF8A1
:20BD600000009DF808107448415C8DF801109DF80910415C8DF802109DF80A10405C8DF875
:20BD80000300608801A9F4F7CDFE20798DF806006448002405AB4470847008208DF814004B
:20BDA00003AA072168461AF0BAFB000612D404231A46414603A8F4F7EDFC00060AD40423BD
:20BDC000032208F1040104A8F4F7E4FC000600E004E00BD5286806B0BDE8F0818820286093
:20BDE00001203060784638608820F4E72C607846346038600020EEE72DE9FC5F0D464A49F7
:20BE00004A4C4B4E09784B4F00295BD023218DF80010010A8DF801108DF802004FF000093B
:20BE20008DF8049001AB454A032168461AF077FB000643D4DFF804810020FFF739F800069A
:20BE40003CD498F8401029B198F80000092801D01028F1D1FFF70EF800062FD498F84010A7
:20BE6000404671B3027805F10A0A092A05F10F0B4FF005034FF00602294637D0C01CF4F786
:20BE800089FC00061AD42D4805230622691D0930F4F780FC000611D42848052306225146FC
:20BEA0000F30F4F777FC000608D424480523062259461530F4F76EFC000643D52068BDE8C3
:20BEC000FC9F07E08820206001203060784638608820F4E71421284623F01EFD922020602B
:20BEE00027203060784638609220E8E708F10100F4F750FC0006E1D405230622691D08F1D9
:20BF00000700F4F747FC0006D8D40C480523062251460D30F4F73EFC0006CFD405230622A4
:20BF200059460DE035000010FA02000008C007200CC0072010C00720C6110300B8020010B7
:20BF40008F48B7E7C4F800907846C6F8009038600020B4E72DE9FE430F468A498A4DDFF894
:20BF60002C820978DFF8289231B323218DF80010010A8DF80110824A8DF8020000268DF8A5
:20BF8000086002AB133A032168461AF0C8FA000610D47B4C133C0020FEF78AFF000609D420
:20BFA00094F8400010B120780E28F4D1FEF762FF00060AD528680CE4882001212860C8F894
:20BFC00000107946C9F8001003E494F84000E8B3E07800F00F01000900EB800001EB40007B
:20BFE0008DF80400207900F00F01000900EB800001EB40008DF80500607900F00F01000913
:20C0000000EB800001EB40008DF80600394601A8F4F78EFCE07900F00F01000900EB800094
:20C0200001EB4001A07900F00F02000900EB800002EB4000C0EB001001EB80007880207A5F
:20C0400038712E607946C8F8006000E003E00020C9F8001033E43E609220BE8027212860A1
:20C06000C8F800107946C9F8001028E47CB505462A208DF8040000248DF800406B462A46FB
:20C08000012101A81AF04BFA01063F4801D500687CBD9DF800106C5404603C480460784612
:20C0A0003B49086000207CBD2DE9F04186B024208DF8040006208DF8080004A90020FFF77B
:20C0C0000FF9314D000624D49DF81000DFF8C4802E4E2F4F01074FF0000401D5800602D5A4
:20C0E00088F800402BE0264A8DF800406B46133A012101A81AF013FA00060AD401208DF8D6
:20C100000C00014603AB002202A81AF008FA000601D528685FE69DF80000401EC0B28DF8AB
:20C120000000102809D0282807D092202860202030607846386092204DE688F800002C6076
:20C14000784634603860002045E6124910B50C780D490E4A0E4B5CB1102C09D0282C07D0B2
:20C16000882008600820106078461860882010BD046000200860106078461860002010BDED
:20C18000CB020010FA02000008C007200CC0072010C0072035000010F0B54178F74AF84BC6
:20C1A000F84C962509B1142903D902201560186013E005260C2914D004DC052911D0062949
:20C1C00004D10EE00D290CD00E290AD0EE4F0078795C884209D015601E6078462060962065
:20C1E000F0BD0078801E4128F5D2002010601860784620600020F0BD30B5E04AE04BE14CD2
:20C20000012115292FD2DFE801F02E0D0F0F0F1313151517171911111B1D1F0B1717210033
:20C220000D2014E0032012E0022010E041200EE042200CE00E200AE0072008E0152006E0D7
:20C24000002004E0062002E00A2000E00520CE4D6854491C1429D4D90020106018607846B7
:20C260002060002030BD8F20106003201860784620608F2030BD2DE9F04F99B04FF0C047B9
:20C280003846012215A911971BF097FABB4C00065FD4781C012216A911901BF08EFA00060B
:20C2A00057D4BA494FF00109B54D81F800909DF85400B44E4FF09608572804D0C4F80080A5
:20C2C000C5F8009058E09DF858004FF0030A802805D000BFC4F80080C5F800A04CE011A8E6
:20C2E000F9F7FDFB000634D413A8F9F709FC00062FD438461BF078FA0746504611994FF0C8
:20C30000060AB0EB517FE5D121F06041B942E1D2139AB0EB527FDDD122F06040B842D9D26E
:20C320000229D7D30228D5D3DFF864B213991198884231D0022269461BF03FFA000608D450
:20C340009DF80000FF2808D06846FFF725FF000605D5206819B0BDE8F08F8DF8009013996B
:20C36000119888420CD29DF8002002448A4207D90520C4F800802860784630609620E9E708
:20C380009DF800100844119020F06040B842A1D8CCD1CDF844B0C9E74FF00000206028609B
:20C3A000784630604FF00000D4E738B56846F9F7A7FB724C000604D46846F9F786FB000647
:20C3C00001D5206838BD6E4900202060086078466C490860002038BD1CB56C48674C0078AB
:20C3E00060B148F257014FF0C040ADF804100090022201A91BF0ECF900060BD46448009033
:20C400006846F9F762FB000604D46846F9F76EFB000601D520681CBD594900202060086055
:20C4200078465849086000201CBD5848007870472DE9FC4104460D464FF0C0401BF0D4F966
:20C44000064652484D4F4FF00008007860B16846F9F745FB000604D401A8F9F751FB0006E3
:20C4600007D53868BDE8FC81C4F80080C5F800800AE0A6F102062E60DDE90010401A2060DE
:20C4800002D52968084420603D49C7F800807846C1F800803B4908600020E3E71CB501A95B
:20C4A0006846FFF7C5FF000603D4009808B100201CBD01201CBD2DE9FC4781463348304DDB
:20C4C000304E00782D4C96274FF0040880B101A96846FFF7ADFF000602D52068BDE8FC872D
:20C4E000DDE90010411A09EB4910B1EB400F06D227607846C5F8008030609620EEE700203E
:20C5000020602860784630600020E7E72DE9F04F044697B04FF0C0401BF066F981461B481E
:20C52000174FDFF860800078144E002500287DD014A949200AF084FA000678D49DF8500095
:20C54000032873D002280ED1607814286ED2DFE800F0AC0A0A0A0A0A0A0A0AACAC0A0A0AE7
:20C56000AC0AAC0A0A0A60780A281DD012DC012818D002281AD0092812D115E008C0072039
:20C580000CC0072010C0072058C207203C000010020000600B2809D00F2805D0102803D09F
:20C5A000182004E0782002E00F2000E00C20FFF782FF00066DD4607808B1142809D9962087
:20C5C00030600320794638609620C8F8001017B0C1E6DFF884A40C280CD004DC052815D05C
:20C5E000062804D112E00D2804D00E2853D01AF8000018E004F1100023F0B6F8302802D9E1
:20C6000084F8405030209AF80C100AE004F1110023F0AAF8302802D984F8415030209AF849
:20C620000510303808442070684601E03DE030E0F9F766FA00062CD400982178834620F085
:20C640006040A9EB000A51450DD9FF22422101A8F3F7CCFE524601A958461BF0B9F800069D
:20C6600017D4FE4800902278214600981BF0B0F800060ED420780099084420F06041009007
:20C68000494501D1F54800906846F9F72FFA00060BD530689BE7A01C23F066F8302802D946
:20C6A00084F832503020C01CBDE7356079463D600020C8F800108AE72DE9F84F06464FF072
:20C6C000C0401BF091F8DFF898A30746E54C9AF80000DFF89483DFF8949300254FF0050B44
:20C6E00048B16846F9F70CFA00061FD4DAF8043000998B4209D1C4F800B07946C8F8005023
:20C700000520C9F80010BDE8F88F4222314618461BF053F8000609D4DFF840B33078FF28EC
:20C7200006D03046FFF738FD000616D52068EAE7DAF804105046491CCAF8041021F06041CF
:20C74000B94201D1C0F804B042223146DAF804001BF033F80006E1D5E8E73178DAF804208F
:20C760001144CAF80410B94201D1CAF804B025607946C8F800500020C9F80010C3E72DE946
:20C78000F14FDFF8DC920027B64C99F80000B64DB64E92B0B8464FF0050A002873D011A8A1
:20C7A000F9F7AEF9000636D44FF0C0401BF01CF8834663E0022269461AF0FFFF00062AD489
:20C7C0009DF80000FF2814D09DF8011005291DD006291BD00B2919D0D9F8042049461044E9
:20C7E00020F06042C9F804005A4517D0D9F8040016E0D9F80400401C20F06042C9F80400C9
:20C800005A453BD19548C9F8040037E06846FFF753FF000610D5206813B09CE58F48486088
:20C8200020F06041594507D99620206006202860784630609620EFE79DF80100012803D079
:20C84000052801D0062804D19DF80020D9F804108F1A052803D0062801D00B280ED1BDF8CE
:20C860000A101298814209D1C9F80470C4F800807846C5F8008030600020CDE7D9F80400B2
:20C880001199884296D1C4F800A07846C5F8008030600520C0E7F0B57148734E734F0078B1
:20C8A000704C85B00025A8B36D48001DF9F717F900062CD401A81EF0DBFB000627D46946F2
:20C8C00021200AF088F9000621D49DF80000ADF8040069461F200AF07EF9000617D49DF87E
:20C8E0000000ADF80A00694626200AF074F900060DD49DF80000ADF80C001EF055FC00069B
:20C9000005D4002101A81EF0D4F900060AD5206805B0F0BDFFE70520206078463560386054
:20C920000520F5E725607846356038600020EFE72DE9F8434A4E4C4FDFF830813078494C47
:20C94000002560B16846F8F79DFF000660D47078B8B11EF0EDFB000609D5757058E00520C1
:20C96000206079463D60C8F80010BDE8F8832068052851D03A48001DF9F7A7F8000647D4C6
:20C980007570DFF8EC903A48FFF796FE00063FD42068C0B99DF80000172817D0152815D05C
:20C9A000192813D099F801001328ECD2DFE800F00A0B0B0B0B0B0B0B0B0A0A0B0B0B0A0B65
:20C9C0000A0B0B00DFE720680528CED0552008F015FD00061CD499F80100062809D004DC30
:20C9E000022806D0052817D103E00B2801D0112812D1562008F002FD000609D49DF800003A
:20CA0000172801D0182807D11EF076FB000601D52068AAE701207070256079463D60002078
:20CA2000C8F80010A1E770B50D480E4C92B0007800285ED000210FA01EF05BFA000655D458
:20CA4000002111A01EF055FA00064FD4FFF723FF00064BD420E0000058C20720020000609E
:20CA60003C00001008C007200CC0072010C0072079C207208E9888818A80208693908D8020
:20CA80008B80208A8B0A000086E3E0ADA0AB20AEE7A8E9A5AD0A0000FFF74AFF206800287A
:20CAA000D8D01EF081FB000620D401201EF071F900061BD44D2008F0A1FC000616D40120A9
:20CAC00002F086F8000611D4FFF786FC00060DD40E268DF80160AFF264016D46A81C22F0F3
:20CAE0001FFE6846FFF712FD00060BD5206812B070BD0A4900202060086078460849086037
:20CB00000020F4E78DF80160AFF28401A81C22F007FE6846FFF7FAFCE9E700000CC00720D6
:20CB200010C007202DE9FF470220039019F06EFD0024FC48FC4EDFF8F49344708460254666
:20CB400003274FF03208C4608DF804708DF8055003AB02AA022101A8CDF8008019F011FEB8
:20CB6000000603D5306804B0BDE8F0879DF808009DF8091000EB012009EB45016D1C888647
:20CB8000032DE1D3EA48346004607846E94908600020E8E7E54A02EB4000808E0880E24923
:20CBA00000200860E24908607846E24908600020704708B569460220FFF7ECFF0106DA489A
:20CBC00001D5006808BDBDF80030D949D94AB3F57A7F07D2932303600B20086078461060D4
:20CBE000184608BD0023036078460B601060184608BD2DE9FF418846CA4D022103910124B9
:20CC0000E968CA4A8440C84F0C4202EB40061CD104218DF804108DF805003220009003AB8E
:20CC200002AA022101A819F0ACFD000603D5386804B0BDE8F0819DF808009DF8091000EB4C
:20CC400001207087E8680443EC60718FA8F80010B7490020386008607846B64908600020C4
:20CC6000E6E73EB5044641208DF804000C2002903220009002AB2246012101A819F081FDB9
:20CC80000106A94801D500683EBDA6498A6842F080028A60A54922681439CA6362680A64BA
:20CCA000A2684A6400210160A14801607846A149086000203EBD0EB570B101280ED00228B0
:20CCC0001DD099498820086099490D20086078469849086088200EBD102200E00522121D1C
:20CCE000019209228DF808208DF8090032200A46009001AB022102A819F043FD0EBD0A2250
:20CD0000EDE70EB50022029210228DF804208DF805008DF80610080A8DF80700322001AA2B
:20CD2000009002AB0421104619F02BFD0EBD38B504466946FFF75DFF7B4A000601D51068EE
:20CD400038BDBDF8001039B1491E89B2ADF800102046FFF7D6FF38BD05207549106000203F
:20CD60000860784673490860052038BD2DE9FE4F0D466C4980466E4E6E4F6B4C88684FF0BF
:20CD800093094FF0070AB8F1050F5CD2DFE808F02916160330008B46800729D40120FFF709
:20CDA000C6FFB0BB614901201431FFF784FF000646D4DBF8081041F002010FE08B46C007F4
:20CDC00016D1FFF7B4FF20BB58490020FFF773FF000635D4DBF8081041F00101CBF80810B7
:20CDE00006E0000604D46846FFF73BFF000627D44E481438B8F1050F25D2DFE808F0030B2D
:20CE00000F151B00C16B2960016C6960406CA86021E015E081692960808B03E0D0F81E10E7
:20CE20002960408CA88016E0C16A296090F83000287110E029460220FFF7DBFE00060AD545
:20CE40002068BDE8FE8FC4F800907846C6F800A038609320F5E70020206030607846386003
:20CE60000020EEE72F498A6882438A60CA688243CA602D49002008602D49086078462D4973
:20CE80000860002070472DE9F04F264D042289B08046284F0026DFF89890234C28466A7013
:20CEA0004FF0860A02290CD0032907D004290CD005290AD00821C4F800A044E02E70012020
:20CEC00001E02E700020A87005E001220270052918D00021A97013481730F7F76CFC114880
:20CEE0001030F7F768FCAB4628780E4D1E3558B101202880B8F80010A9806880B8F802000C
:20CF0000E88019E00121E5E7B8F800002880AE80B8F802106980EE8088420DD91321C4F883
:20CF200000A010E02CC0072008C00720600300100CC0072010C00720A888E98888420AD9B4
:20CF40001421C4F800A07846C9F800103860862009B0BDE8F08F69460220FFF74AFE000681
:20CF600067D49BF80000D8464FF0810A20B92888BDF8001088426DD82888401E81B202203B
:20CF8000FFF7BFFE00067AD402A90220FFF793FE206838B105280AD09328D9D1D9F8001078
:20CFA0000829D5D198F8001079B120B10DE098F80000E8BB11E0BDF80820AB889A4204D32B
:20CFC000BDF80A002880AA8010E00143DCD1BDF80800A88098F8000040B96888BDF80010BC
:20CFE000884200D90846ADF800006880BDF80000401E81B20220FFF784FE00063FD402A90F
:20D000000220FFF758FE206828B19328A0D1D9F8001008299CD198F8001069B160B9BDF80E
:20D020000820EB889A4207D8BDF80A00688001E010E024E090B217E0014313D0BDF8000009
:20D04000401E80B2ADF8000029888142CED998F8000050B1C4F800A07846C9F8006038601C
:20D06000812075E7BDF80800E8802888401E81B2A8F804100220FFF744FE000601D52068DB
:20D0800066E726607846C9F80060386000205FE72DE9F047B84DDFF8E492DFF8E482687824
:20D0A000B84C002620B1032819D004280FD107E0052020607946C8F80060C9F8001053E5E1
:20D0C000492008F09BF9000649D40320687026607946C8F800600020C9F8001044E5002797
:20D0E000A9490220FFF7E7FD932804D1D8F80000082834D10127A888401C80B2A880A9787E
:20D1000089B987B14C2008F079F9000627D41EF04BF8000623D4812020607946C8F8006070
:20D12000C9F8001020E52168052904D092491E314988814202D26E704A2017E08FB992499A
:20D140008D48091D1030F7F7D8FB000607D48E49894809311730F7F7D0FB000601D52068AC
:20D1600002E5A8780028BAD027B14C20BDE8F04708F044B94B20F9E700B587B000210691F2
:20D180008DF80400322001AA009006AB0121104619F0F7FA07B000BD70B588B003004FF043
:20D1A0000000784D0E4607900ED0012B0ED0022B0ED08820724928600D20086078466F49D6
:20D1C0000860882008B070BD102402E0052400E00A24241D01209840FFF744FE000601D5BF
:20D1E0002868EFE708208DF804008DF80530224631460DF1060022F0D6FA322001AA00900C
:20D2000007ABA11C104619F0BCFADBE77CB50C4605466946FFF7EDFC5A4B000605D401A93E
:20D220002846FFF7B7FC000601D518687CBDBDF80400BDF80010401A208051490020186098
:20D24000086078464D49086000207CBD7FB5044615208DF808000420039032200D46009025
:20D2600003AB01AA012102A819F08BFA0106454802D5006804B070BDBDF804102180BDF828
:20D2800006102980002101603D48016078463B4908600020EEE70EB50222029216228DF890
:20D2A00004208DF8050041F288300A46009002AB022101A819F065FA0EBD00B587B000213C
:20D2C000059140218DF804100168CDF805104168CDF809108068CDF80D00274801AA05AB70
:20D2E000816821F080018160322000900D21104619F047FA4EE770B58CB0064680208DF81B
:20D3000024001E200A9032200D4600900AAB01AA012109A819F035FA1A4C000608D4BDF874
:20D32000040028801C220DF10601304622F03BFA20680CB070BD3EB504460220029081203E
:20D340008DF80400322001AA009002AB0121104619F017FA01060B4801D500683EBDBDF830
:20D3600004102180002101600548016078460349086000203EBD00002CC0072010C0072031
:20D380000CC0072008C007204C0300102DE9F84F054600794C4C4D4FDFF83481862608B106
:20D3A0001E2802D9052026604BE0288848F6AD614FF0140A884203D92660C7F800A041E071
:20D3C00068884FF0170BB0F5B46F03D32660C7F800B037E06846F8F7F7F9000668D42888D3
:20D3E000BDF80010401A4FF4B46100FB01F9B9F1000FE1DB6846F8F7F7F9000658D468889D
:20D40000BDF80010A0EB010111EB0900DED431490120F8F761F800064AD42F490220F8F773
:20D420005BF8000644D468790F380C2807D2DFE800F00F0F0F0F0F060F0F0F0F060F0820C5
:20D440002660386079468620C8F80010BDE8F88F2846F7F7CEFD00062AD4A81CF7F7DAFD99
:20D46000000625D4281DF7F7E6FD000620D4681DF8F7FEF900061BD4002568460095F8F7E6
:20D4800040FA000614D468460095F8F74BFA00060ED40120ADF800006846F8F710FA000692
:20D4A00006D4ADF800506846F8F71AFA000601D52068CBE7032009498DF800000220087042
:20D4C0006846F7F763FDC1E708C007200CC0072010C00720460000104B00001000C0072037
:20D4E0002DE9F04F87B005A8F8F7CCF9FE4C000672D46846F8F7EDF90006F9D4DFF8ECB3DD
:20D500004FF002099BF80000B8B19DF81400A0F10E01072911D2DFE801F004040C0C0C3550
:20D5200004008BF80100102032E000BFADF8009003E0BDF80010032922D09DF814000E2888
:20D5400002D000BF20F01EFD9DF814100127E84DE84E88204FF0640A4FF000081B2970D2A1
:20D56000DFE801F06FF2F1F1F1F1F0F0F0F0F0F0F0F01E1EEFEEEDECEBEAEAEAEA6FE90071
:20D58000401C05E0BDF800000328DBD19BF801008DF8140005A8F8F76BF90006A8D4C5E763
:20D5A000BDF8001008297FD007DC0829D7D2DFE801F04814249B304961745A296AD006DCA9
:20D5C000092978D00A2967D040293AD170E15B2970D06429F9D19BE069E1C449122009F08A
:20D5E0002FFA000684D49BF8001001F008018BF80010ABE1ADF8009084E08BF8008001F05B
:20D600007BFB0006CAD40420A9E100BFADF80070AFE301F0E7FB0006C0D46846F8F76AF96F
:20D620000006BBD4BDF80000042801D2401C9EE3ADF800706846F8F753F90006AED4052019
:20D6400015E0E5E101F0CBFB0006A7D46846F8F751F90006A2D4BDF800000228E6D3ADF837
:20D6600000706846F8F73CF9000697D40620ADF8000047E001F0B9FB00068FD46846F8F75A
:20D6800039F900068AD4BDF800000428CED30720EDE709E05BE00EE01EE0192007F0AEFE8B
:20D6A00000069FD40820E2E701F096FB000699D40920DCE798E001F08CFB000692D49DF82E
:20D6C00014000E280FD1FDF719FB00068AD42068052808D00A20CAE7FDF763FB000691D48F
:20D6E0002068002811D040E201F009FB000689D49DF814000E2873D01DF0FEFC00068BD491
:20D70000ADF800A06846F8F7DAF807B0BDE8F08F1DF00EFD000684D42068052804D09DF8E6
:20D7200014000E2811D055E1C4F800807846C5F80080306091E284E2EDE3E5E260E28AE1A4
:20D74000F4E1E2E0E8E3E8E38FE25A208FE76846F8F7A0FB000688D49DF8000000287DD097
:20D7600065484FF05B09007800283FF443AF6846F7F7E0FB000685D460480078C0B19DF898
:20D7800000001B2814D06846F8F749F8000688D46F46B81CF8F754F8000688D4381DF8F7B8
:20D7A00060F800068AD46846FDF7CDFE000685D469460420FFF7DAFA000687D4BDF800002E
:20D7C000401C80B2FEF7B8F858B192286FD1F2F727FD13208DF800006846F7F7A1FBFCE337
:20D7E000B8E3ADF800906AE243480078B8B30121434801F055FA00068DD4FEF706F9000651
:20D8000089D43F4890F8400000288DD16846F7F791FB00069FD49DF800000E283DD06846AF
:20D82000F7F7FDFF000696D4DBF8021001919BF806108DF80810DBF80710CDF809109BF876
:20D840000B008DF80D000DF102010420FFF78EFA000690D4BDF80200401C01E021E022E027
:20D86000ADF802001120FFF787FC00068FD469460220FFF791FC000689D41220FFF77CFC97
:20D88000000684D40220FFF752FA000685D469460220FFF710FA000684D4FCF7F3FE00064E
:20D8A00085D44020E3E6164981F84080AEE773E2072020F0D4FA8DF800806846F7F70EFBB5
:20D8C000000699D46946122009F0BAF8000693D49DF8000040077DD56846F6F76CFF0006A2
:20D8E0008AD4694601200DE008C00720440000100CC0072010C00720FA0200005000001084
:20D90000B8020010F7F72EFBFBE1BDF8001017297DD00EDC14292AD006DC012916D00229BA
:20D9200018D0032974D17FE315295AD01629F9D13AE01A296DD004DC18296CD01929F1D1C0
:20D940002CE01B2947D06429ECD1B3E3012001F03FF93EE301F0D0F9000687D41420ADF821
:20D9600000006846F7F7ABFF000685D44EE601F024FA000685D46846F7F7BCFF000685D4AA
:20D98000BDF800001028FFF451AEADF800706846F7F7A6FF000694D4192068E601F001FA71
:20D9A00000068ED4162062E601F00DFA000688D46846F7F79FFF000689D4BDF8000010289D
:20D9C000E1D3ADF800706846F7F78AFF000687D41B204CE602E301F0EAF90006BDD4152006
:20D9E00045E601F0EDF90006B7D46846F7F782FF0006B2D4BDF800001028C4D3ADF8007052
:20DA00006846F7F76DFF0006A7D418202FE608E0ADE015E0FFE701F0C7F900069DD4172081
:20DA200025E601F0D3F9000697D46846F7F762FF000692D4BDF800001028A4D31A2016E6AA
:20DA400001F0B8F977E2000687D455E6206805283FF46AAE35E3BDF800101F2950D009DC05
:20DA600001293FF4C6AD022918D003297ED01E297DD119E020292DD021297FF464AF01F0B4
:20DA80008DF9000687D46846F7F734FF000688D4BDF8000018287FF6C9AD06E301F02CF98F
:20DAA000000684D41E205AE701F06FF900068ED46846F7F71FFF000689D4BDF800001828B6
:20DAC000E9D9ADF800706846F7F70AFF000685D42020CCE501F05FF9000685D46846F7F736
:20DAE00009FF000685D4BDF800001828D3D9ADF800706846F7F7F4FE000685D41F20B6E542
:20DB000001F046F9000689D46846F7F7F3FE000684D4BDF800001828BDD9ADF80070684639
:20DB2000F7F7DEFE000684D42120A0E5BDF8001029294FD008DC012993D0022918D0032911
:20DB400094D0282994D119E02A292DD02B2994D101F018F9000695D46846F7F7CBFE0006CD
:20DB600090D4BDF800001E2895D99EE2DDE0DDE001F0C2F8000685D42820F0E601F0F9F8D4
:20DB8000000684D46846F7F7B5FE000689D4BDF800001E2894D9ADF800706846F7F7A0FEBE
:20DBA000000684D42A2062E501F0E9F800068ED46846F7F79FFE000689D4BDF800001E28A5
:20DBC00094D9ADF800706846F7F78AFE000684D429204CE501F0D0F800068ED46846F7F70A
:20DBE00089FE000689D4BDF800001E2894D9ADF800706846F7F774FE000684D42B2036E5EC
:20DC0000BDF8001003299BD004DC012994D0022998D110E037299AD101F0A8F800069AD4E6
:20DC20006846F7F767FE000695D4BDF800002028FFF4FCAC39E201F05FF800068BD43720BD
:20DC40008DE6BDF8001003296FD004DC0129DDD002296BD103E03829DDD1002055E501F0C6
:20DC60004BF8000687D4382001E5BDF800103E2915D006DC0129C9D002290AD0032955D1B5
:20DC80003DE03F293FF4E1AE402925D064294DD10BE001F031F8000689D43E20E7E401F0B2
:20DCA000A7F8000688D43F20E1E41DF041FA000672D4206805283FF437AD402082E068466F
:20DCC000F7F7FDFD000667D4042020607846C5F800803060042018E5FBF79AFD00065BD40D
:20DCE0000327ADF800706846F7F7E9FD000653D427607846C5F800803060032005E500F027
:20DD0000FEFF000648D4DCE1BDF8001008293FF4CBAC0DDC082909D2DFE801F008092FFC9E
:20DD20003F060504B9E4A5E48CE47DE181E054E452297DD006DC09293FD0502945D0512915
:20DD400077D19CE0532975D0542985D16846F7F7D1FD000620D4BDF80000C0B20546FBF7A3
:20DD6000F3FD000618D4182D7ED26D1CE8B2ADF800006846F7F7B4FDC7E48BF8008000F079
:20DD8000BBFF000608D4ADF800706846F7F7A8FD000601D404206AE482E001F023F80006D0
:20DDA0007ED46846F7F7A6FD000679D4BDF800000428FFF43BAC0520D1E501F00AF80006F0
:20DDC0006ED45020ADF8000079E76846F7F7B2F8000665D49DF800000E2833D06846F7F79D
:20DDE0001EFD00065CD4DBF8021001919BF806108DF80810DBF80710CDF809109BF80B00AF
:20DE00008DF80D000DF102010420FEF7AFFF000646D4BDF80200401CADF802001120FFF7A7
:20DE2000ABF900063CD469460220FFF7B5F902E040E000E156E0000632D41220FFF79CF9D1
:20DE400000062DD46946122008F0FAFD000627D49DF8000040070CD56846F6F7ACFC0006E4
:20DE60001ED46946012000E058E0F7F77BF8000616D4FBF70DFD000612D451206FE568461C
:20DE8000F7F738FD00060BD4BDF80000C0B20546FBF7A6FD000603D4102DFFF466AF00E071
:20DEA00079E0ADF800706846F7F71AFD000672D4522010E46846F7F71DFD00066BD4BDF8DF
:20DEC0000000C0B20546FBF7B9FD000663D40A2DE3D3ADF800706846F7F702FD00065AD4CF
:20DEE000532033E46846F7F705FD000653D4BDF80000C0B20546FBF74DFD00064BD41E2DAF
:20DF0000CBD3ADF800706846F7F7EAFC000642D454201BE412E079E020E03DE08DF80080D0
:20DF20006846F6F7DBFF000635D4FCF7ABFB000631D4FCF7E3FE00062DD4B6E0FCF731FF25
:20DF4000000628D4206800283FF488AE00F0D7FE000620D4502007F051FA74E5BDF8001017
:20DF600001293FF4F3AC022902D0632963D105E000F0C2FE00060ED4632093E4544890F84D
:20DF8000400058B30221524800F08AFE000602D4FDF73BFD62E674E0BDF800105C292CD017
:20DFA0000ADC01291BD002297FF4BBAC00F0A4FE000666D45C2075E45D2917D05E297FF453
:20DFC000C2AC4448007800283FF414AB372007F015FA000673D4FFF70DBB50E071E00120AB
:20DFE00000F0F6FD00066AD45D205BE4362007F005FA000663D45E2054E4FFF749F80006C2
:20E000005DD42068052850D0FFF78EBBBDF8001079291ED00BDC012914D00329CFD1012084
:20E020001CF0B7FE00064AD400F069FE0BE57A291AD07B292CD020607846C5F8009030606C
:20E0400088200BE6012000F0C3FD000637D4792028E4572007F0D2F9000630D4FEF71BFC51
:20E0600000062CD47A201DE4FEF762FC0028CBD0052807D0F2F7D4F801201CF08AFEF2F792
:20E08000E4F81CE01DF038F8000618D47B2009E41DF04EF8000612D420680528B4D09DF8E4
:20E0A0001400172803D0182801D0032075E4FEF77CF940E71DF03CF800067FF5C7AC206866
:20E0C000CCE527607846C5F8008030600120C5E5B8020010FA0200001CB5F6F7A3FD244C1E
:20E0E000000609D401A8F7F7CDFB00063AD46846F7F711FC000601D520681CBD0098000646
:20E1000021D46846F6F75DFF00062BD46846F6F7C2FC000626D46846F6F749FF000621D4D7
:20E1200069469DF80400F7F7C1FB00061AD46846F6F78BFC000615D469469DF80400F7F7B2
:20E14000A8FB00060ED400248DF800406846F7F78FFB000606D48DF800406846F6F716FFD0
:20E16000000602D5F6F7FEFD1CBDF6F788FD1CBD08C007202DE9F04F05460079D94CDA4F60
:20E18000DA4E93B04FF0860808B11E2804D90520C4F80080306017E0288848F6AD614FF048
:20E1A000140A884205D900BFC4F80080C6F800A00AE068884FF0170BB0F5B46F0AD300BFA1
:20E1C000C4F80080C6F800B078463860862013B0BDE8F08F0DA8F7F7F7FA00067ED4288816
:20E1E000BDF83410401A4FF4B46100FB01F9B9F1000FD9DB0DA8F7F7F7FA0006EED46888C6
:20E20000BDF83410A0EB010111EB0900D8D4B8494FF0000A012081F800A0B649F7F75CF901
:20E220000006DBD4B4490220F7F756F90006D5D40520FEF717FE0006D0D40DA8F7F72AFE7A
:20E240000006CBD49DF834004FF0010B00287DD0AA4800780028FAD0FDF7B1F90BA90520BD
:20E26000FDF73EF80006B9D40EA90320FEF77EFD0006B3D405220EA90BA821F025FA78B120
:20E280003D2007F0BBF80006A8D4012000F0A0FC922020603120306078463860922096E7B0
:20E2A000FDF7CBF8000699D490480068232809D13A2007F0A3F8000690D49148018821F006
:20E2C000020101800BA90020FDF70AF8000685D49DF82C00400602D5012001E0BFE00020F2
:20E2E00080460DA90420FEF741FD000686D40BA90620FCF7F5FF000693D4BDF83400BDF81F
:20E300002C60401C864201D1012000E000208146B8F1000F13D1B9F1000F10D1761EB6B261
:20E3200009A93046FDF716FE000685D4BDF824002880BDF8260068809DF8280028710DA9FE
:20E340000420FEF713FD00068DD400E06CE0BDF83400401CB04212D0482007F04FF800063C
:20E360007DD4012000F034FC000678D48F2020605E4807210160784638608F2027E704A99B
:20E380003046FDF739FD000669D48DF834A0012710A93846F7F7A0F8000660D407EB8701A8
:20E3A00004A80144491F052210A821F08DF910B18DF834B005E07F1C042FE9D99DF8340026
:20E3C00060B350480680402007F018F800067CD45E2007F013F8000677D4494801260DF1C8
:20E3E0001007018821F0020101804248049901609DF8141001714048DDF8151001609DF8BD
:20E400001910017106EB8600C119491F3046F7F756F8000659D4761C042EF3D958EA0900E8
:20E4200002D0334981F800B02846F6F7E2FD00064BD4A81CF6F7EEFD000646D4281DF6F718
:20E44000FAFD000641D42846F7F7DFF900063CD4A81CF7F7EBF9000637D4281D00E034E080
:20E46000F7F7F5F9000630D4681DF7F701FA00062BD455460DA8CDF834A0F7F742FA00062A
:20E4800023D40DA80D95F7F74DFA00061DD4ADF834B00DA8F7F713FA000616D4ADF83450B0
:20E4A0000DA8F7F71DFA00060FD40DA91C2008F0C7FA000609D49DF8340040B1ADF8345048
:20E4C0000DA8F6F785FD000601D520687FE603200D498DF83400022008700DA8F6F756FD8E
:20E4E00075E6000008C0072010C007200CC0072050000010460000104B000010FA020000DB
:20E5000002C0072030C0072000C007202DE9F84305460E466846F7F7BDFC564C00067DD4D6
:20E520009DF800105448554A4FF0000939B12979862309B11E290BD90521236019E087214F
:20E540002160C0F80090784610600846BDE8F883298848F6AD674FF01408B94203D923609E
:20E56000C0F8008006E06988B1F5B46F06D3172123600160784610608620E7E76F79BC4642
:20E58000BF1F082F69D2DFE807F00404151523272B2F378871888F4202D913212360E8E7AD
:20E5A000BCF1070F04D000223846FDF773F91DE00122F9E7378871888F42D0D8BCF1090FCE
:20E5C00004D000223846FDF705F90FE00122F9E73088FDF78CF809E03068FDF7C0F805E0A1
:20E5E0003088FDF7A9F901E0FDF7DDF9000632D42846F6F7FEFC00062DD4A81CF6F70AFD02
:20E60000000628D4281DF6F716FD000623D4681DF7F72EF900061ED44D4600E01BE0684608
:20E62000CDF80090F7F76DF9000614D468460095F7F778F900060ED40120ADF80000684645
:20E64000F7F73DF9000606D4ADF800506846F7F747F9000604D5206878E70821236088E704
:20E66000032007498DF80000022008706846F6F78DFC6BE708C007200CC0072010C00720B9
:20E6800000C007202DE9F843054688466846F7F701FC4D4C00067CD49DF800004B4E4C4FD8
:20E6A0004FF0030928B129798620A9B1206005202CE0452006F0A2FE000679D4012000F084
:20E6C00087FA000674D48F2020607846C6F8009038608F20BDE8F883298848F6AD629142F8
:20E6E00002D92060142011E06988B1F5B46F02D3206017200AE0697902290CD003290AD07B
:20E70000042908D0052906D0206008203060784638608620DEE74046FEF7B5FB4FF0000885
:20E7200098B1812844D1452006F068FE00063FD4012000F04DFA00063AD4812020607846AD
:20E74000C6F8008038608120C4E72846F6F751FC00062DD4A81CF6F75DFC000628D4281D97
:20E76000F6F769FC000623D4681DF7F781F800061ED445466846CDF80080F7F7C2F800063A
:20E7800016D468460095F7F7CDF8000610D4012000E00DE0ADF800006846F7F790F80006F2
:20E7A00006D4ADF800506846F7F79AF8000601D520688FE707498DF80090022008706846D5
:20E7C000F6F7E4FB86E7000008C007200CC0072010C0072000C0072038B5592006F00EFED8
:20E7E000354C000613D44D2006F008FE00060ED46846F6F7E6FB000609D46846F6F74BF91C
:20E80000000604D46846F6F7D2FB000601D5206838BD2A4900202060086078462849086047
:20E82000002038BD10B5142006F0E8FD000602D52148006810BDBDE810401CF0B5BC1F489B
:20E840000068092801D8D23000E0D2201D490860442006F0D3BD10B5F1F7E2FC1A4C208821
:20E8600000070DD53E2006F0C9FD00061FD41CF09BFC00061BD4208820F00800208016E0AE
:20E880001CF099FD00201CF0EBFC3E2006F0B6FD000603D41CF088FC000603D5208840F099
:20E8A000080020801FF08CFE01201CF0D9FCBDE81040F1F7CABC000008C007200CC00720D0
:20E8C00010C0072054C0072002C0072010B5002006F094FD000602D5B848006810BDBDE8FA
:20E8E00010401CF061BC38B5012000F071F9B34C00060DD46946142008F0A2F8000607D4FB
:20E900009DF80000C00705D01CF019F8000601D5206838BDAA490020206008607846A949A5
:20E920000860002038BD70B5A74C208840F0040020800E2006F062FDA04D000603D41CF06D
:20E9400033FC000601D5286870BD20889C4920F00400208000202860086078469949086096
:20E96000002070BD10B50D2006F048FD000602D59248006810BDBDE810401CF015BC70B53A
:20E980009148924D8D4C0088297800F02000084314D00C2006F032FD000603D41CF004FC44
:20E9A000000601D5206870BD00208549287020600860784683490860002070BD00201CF0ED
:20E9C0004FFC0C2006F01AFD000603D41CF0ECFB000601D501202870F1F722FC01201CF01B
:20E9E0003FFCF1F732FCDDE710B50B2006F006FD000602D57148006810BDBDE810401CF04D
:20EA0000D3BB10B50A2006F0F9FC000602D56B48006810BDBDE810401CF0C6BB10B5092059
:20EA200006F0ECFC000602D56448006810BDBDE810401CF0B9BB10B5532006F0DFFC0006B6
:20EA400002D55E48006810BDBDE810401CF0ACBB10B5542006F0D2FC000602D557480068BB
:20EA600010BDBDE810401CF09FBB10B5082006F0C5FC000602D55148006810BDBDE810402A
:20EA80001CF092BB10B5072006F0B8FC000602D54A48006810BDBDE810401CF085BB10B5DD
:20EAA000062006F0ABFC000602D54448006810BDBDE810401CF078BB10B5052006F09EFC47
:20EAC000000602D53D48006810BDBDE810401CF06BBB10B5042006F091FC000602D53748B0
:20EAE000006810BDBDE810401CF05EBB10B5032006F084FC000602D53048006810BDBDE83A
:20EB000010401CF051BB10B5022006F077FC000602D52A48006810BDBDE810401CF044BBB9
:20EB200010B5012006F06AFC000602D52348006810BDBDE810401CF037BB10B5112006F037
:20EB40005DFC000602D51D48006810BDBDE810401CF02ABB10B5122006F050FC000602D5E9
:20EB60001648006810BDBDE810401CF01DBB10B5132006F043FC000602D51048006810BD92
:20EB8000BDE810401CF010BB10B5512006F036FC000602D50948006810BDBDE810401CF0E7
:20EBA00003BB10B5522006F029FC000602D50348006810BDBDE810401CF0F6BA08C0072048
:20EBC0000CC0072010C0072002C0072058C0072070B5894D0646894C2888800714D5312096
:20EBE00006F00CFC000609D426B1462006F006FC000603D41CF0D8FA000601D5206870BDB3
:20EC0000288820F0020028807D4900202060086078467C490860002070BD10B5362006F073
:20EC2000EDFB764C000607D47748007830B1372006F0E4FB000601D5206810BDBDE81040DF
:20EC40000120C5E710B501461422704820F0ABFD332006F0D3FB000602D56848006810BD5C
:20EC6000BDE810401CF0A0BA10B5362006F0C6FB624C00060ED4372006F0C0FB000609D4E6
:20EC80000120FFF7A5FF000604D43F2006F0B6FB000601D5206810BDBDE810401CF084BA65
:20ECA0002DE9F041A6B006468846202294216846F1F79CFB564D96F840206F46EC89314647
:20ECC000A01A384420F06FFD0A203855781C0021215468461CF00DF9484C000608D4E989F9
:20ECE00068461FF06FFDB8F1010F01D11CF05CFA206826B0BDE8F081152006F07FBB10B560
:20ED00001C2006F07BFB000602D53C48006810BDBDE810401CF048BA1CB50120FFF758FF73
:20ED2000364C000617D46946142007F089FE000611D401A9122007F083FE00060BD49DF846
:20ED40000000C00709D09DF80400400705D51BF0F6FD000601D520681CBD2949002020600C
:20ED6000086078462749086000201CBD2D2006F045BB292006F042BB2A2006F03FBB2B2098
:20ED800006F03CBB2C2006F039BB252006F036BB262006F033BB272006F030BB282006F094
:20EDA0002DBB212006F02ABB222006F027BB232006F024BB242006F021BB1D2006F01EBBFB
:20EDC0001E2006F01BBB1F2006F018BB202006F015BB1B2006F012BB1A2006F00FBB1720EC
:20EDE00006F00CBB162006F009BB182006F006BB342006F003BB000002C0072008C0072097
:20EE00000CC0072010C00720FA0200004C030010F0CD072010B500201CF022FA0F2006F097
:20EE2000EDFA01201CF01CFA1B49002008601B49086078461A490860002010BD10B5102085
:20EE400006F0DCFA000602D51348006810BDBDE810401CF0A9B938B50120FFF7B9FE0E4C01
:20EE600000060DD46946142007F0EAFD000607D49DF80000C00705D01BF061FD000601D593
:20EE8000206838BD0549002020600860784604490860002038BD000008C007200CC0072035
:20EEA00010C0072070B50023202439E0C55C132D28D00DDC132D32D2DFE805F024242424E4
:20EEC00024242424242B262424242424242424001D2D17D004DCA5F11405082D1FD811E030
:20EEE000F52D0FD008DC1E2D0CD01F2D0AD0F32D08D0F42D13D105E0F62D03D0FD2D01D00D
:20EF0000FE2D0CD1C4540AE0012AFBD1002B20D0F8E7C5186E78092E01D1C4546C705B1CBF
:20EF20008B42C3D3032A0DD1FE4AD2898A4202D2114600E0491E421812F8012C202AF9D0DE
:20EF400000224254084410F8011C092901D100F8014C70BD2DE9F04F89B09146012B09D0A8
:20EF6000022B0AD0032B40D0042B06D0002009B0BDE8F08F0225012201E0022536E090460C
:20EF80004FEA116212064FF0000203D5404262EB01010122924606460F463022691C6846A2
:20EFA000F1F724FA0024EB460A2200233046394620F0BAF8064602F130000BF80400641CFA
:20EFC0000F465A4656EA0700EED1681C844200DA6C1CBAF1000F06D0B8F1000F03D02D2121
:20EFE0000BF80410641C002009E003250022C6E7211A114411F8013C09F80030401CA04235
:20F00000F6DB5DB109EB0400411B481C2A4620F00FFC2E21621B641C09F80210002109F84D
:20F0200004102046A3E72DE9FF4180460D4617461C4602A91A2007F003FDBB4E000618D4C7
:20F04000012C1AD05FF002009DF808104FF0000408408DF8080021D0BFB103A99420CDE90C
:20F060000001434602223946032008F0E3F8000605D5306804B0BDE8F0810120E4E702221B
:20F0800040462968FFF70EFF09E0A848007828B11322A7A1404620F086FB00E02C60A9483B
:20F0A000346004607846A84908600020E2E72DE9FF4F0024A3B0074689464FF0010BA2462E
:20F0C0002546A0460DA8F5F77CFF974E00066FD40020ADF80C00309801280AD09B4C484684
:20F0E000B9F1010F79D0022878D0B9F1030F60D1ECE0B9F1090F5CD2DFE809F05B0D052D98
:20F100002026343D26000120ADF80C000DA8F5F7C2FC0006DBD421A8F5F764FF0006D6D464
:20F12000BDF80C00BDF88410084482B2ADF80C2087A10EA820F094F805460CE00DA8F5F722
:20F14000AAFC0006C3D438E04FF0000B0DA8F5F7A2FC0006BBD4B9F1040F2ED0B9F1050FBD
:20F160002BD010E04FF0000B0DA8F5F794FC0006ADD4012407E04FF0000B0DA8F5F78BFC24
:20F180000006A4D4022422A8FBF7DCF90CA8FBF7BDF904A9BDF88800F1F76FFC20208DF8DC
:20F1A000180040F26451012C19D0022C20D028E07DE025990020086053E122A8F5F723FF65
:20F1C000000674D40CA8F5F72FFF00067BD426A8F5F73BFF000676D4DBE72FE03CE0BDF8D8
:20F1E0003000884201D23C3006E0A0F2645003E0BDF8300018B13C38ADF8300001E0ADF84A
:20F2000030100DF11901BDF83000F1F754FC4FF00E09BBF1000F06D09DF898204EA11EA890
:20F2200020F01EF8804603A91B2007F009FC000649D49DF80C00C0075AD160E0628944A139
:20F240000EA820F00DF805466088ADF88800A088ADF83000227B0CE062893DA10EA81FF06F
:20F26000FFFF05466088ADF88800A088ADF83000227C39A11EA81FF0F3FF8046D4F806005C
:20F280000D9003A9BDF88800F1F70AFBBDF830203C20B2FBF0F100FB11209DF80C2000928D
:20F2A000CDE901109DF80D309DF80E2000E00AE02BA104A81FF0D4FF814603A91B2007F029
:20F2C000BFFB000610D5306827B051E6A088ADF88800E088ADF83000227B1FA11EA81FF01F
:20F2E000BFFF8046A068CBE79DF80C00800706D522A224A116A80D9B1FF0B2FF82464C46C4
:20F3000015B109EB0504641CBAF1000F01D05444641CB8F1000F01D04444641CDFF804B0EB
:20F3200034E00000F0CD072008C00720FA0200008D808B8E838E829B8920888D918F858AA9
:20F34000928E90000CC0072010C0072079C20720232530346C7500004B25303275000000DD
:20F36000253032752D253032752D2530327520253032753A2530327500000000848E8A2E23
:20F380002000000025732530386C7500BBF80E00A04239D20A2139545FEA0A0007D002466F
:20F3A00016A9384620F0FFF9BBF80E40641C35B138192A460EA920F0F6F92C44641CB8F191
:20F3C000000F10D0BBF80E00411CA14206D207EB4001A1EB0901A1EB080000E0381942464F
:20F3E0001EA920F0E0F9BBF80E005C4607EB4001A1EB0900401C4A4604A920F0D4F9E18952
:20F40000012000EB410129E000202DB138462A460EA920F0C8F9681C5FEA0A0104D00A4625
:20F42000384416A920F0BFF9B8F1000F0BD0BBF80E004246C119A1EB0901A1EB0800401E8B
:20F440001EA920F0B0F9BBF80E005C46C119A1EB09004A4604A920F0A6F9E18925980160E6
:20F460000020FE49306008607946FD48016000202AE72DE9F04788B00646DDE910858A469B
:20F4800017469946084620F06FF929680446A14200D20C4622465146304620F084F9404600
:20F4A000B8F1050F22D003466A4638464946FFF751FD0246A0182968401C884208D9E9488A
:20F4C0000123C18903EB41012960C0890A21315428686946801A3044044620F064F9B8F15F
:20F4E000010F09D0B8F1020F10D105E03A46DEA168461FF0B5FEDCE7F62004F8010C14F846
:20F50000020C092802D1202004F8020CD84900200860D24908607846D149086008B000204B
:20F52000BDE8F08708B56846F6F7B4FC98BB9DF8000000283DD06846F5F732FD58BB9DF819
:20F540000000012806D003280FD0CA48008802282ED02FE06846F5F728FEE0B99DF80000E3
:20F56000012825D0022825D122E06846F6F78AF988B99DF80000142812D00DDC042817D03D
:20F5800004DC022814D0032814D111E005280FD00E280FD104E00DE0153804280AD807E047
:20F5A0006846F5F7C7FC28B99DF800000E2801D0012008BD002008BDF0B58BB006460F4625
:20F5C0000AA8F6F767FCAA4D000614D49DF828000024E8B1A8A2AAA168461FF041FE421ED9
:20F5E0000DF10101304620F0DEF808A90120FDF7BDFB000602D528680BB0F0BD99480C3E31
:20F600000C23C0890622811908A8F1F7F0F900E03C6092482C6004607846914908600020C9
:20F62000EAE7F0B58DB005460F4601A8F6F732FC8F4C000619D49DF80400002678B3914822
:20F64000007860B36846FCF780FD00060DD40AA90320FDF78BFB000607D40A23052202A9EA
:20F660000AA8F1F7C4F9000602D520680DB0F0BD7C48009AC1892944891A029AC1F8052032
:20F68000039AC1F80920BDF81020A1F80D20C08900992844401A7CA10968016001E0FFE7E2
:20F6A0003E606E482660066078466D4908600020DCE72DE9F04792B004468A461546994668
:20F6C00080201A9EFDF7CEFB694F00066BD40DA8F5F71FFC000666D40EA8F5F73CFC00063C
:20F6E00061D40CA8F6F7D6FB00065CD468A0DFF874810088A4F80100012D02D0022D03D032
:20F7000017E0FFF70FFFA0B15E48007840B1432060710920E071F32121726072F420A07241
:20F72000B9F1010F05D1F5202070B8F80E20611E505446B19DF8300028B1B8F80E002528F3
:20F7400001D30C2502E0B8F80E50083D69460020FDF70CFBDFF8049140B3D9F80000062847
:20F7600009D09DF834000E2805D09DF838100E2919D1082817D160193F220721F0F736FEA9
:20F78000ED1D002E63D09DF8300000285FD03AA23BA168461FF064FD06460FA90120FDF7F3
:20F7A000E5FA00060DD5386812B0B9E66019DDF805100160BDF8091081809DF80B1081714C
:20F7C000DEE7A919B8F80E000D316D46884210D32044801B0C38721E691C1FF0E4FF1E23BB
:20F7E000062269460FA8F1F702F9B8F80E000D3C23E00A212154B8F80E20601C10442146D9
:20F800001FF0D1FFB8F80E1020222046F0F7EEFDB8F80E00012101EB4001CAF80010721E52
:20F82000691C20461FF0BFFF1E23062269460FA8F1F7DDF8B8F80E000C3C2044DDF8121023
:20F840000160DDF816104160DDF81A10816000203860C9F80000784601491BE00CC007205C
:20F8600010C00720F0CD07202530346C7500000008C007202801001020888D8D2000000039
:20F8800025730000FA0200009D8A8B87000000008F8400000860002086E72DE9F04F99B0F5
:20F8A00080460D46164605A90B2007F0C9F8FF4C00066ED4FE48DFF8FCA3DFF8FCB34FF02E
:20F8C0000109092E71D2DFE806F0700510162438424C680004A8F5F7FDFC000659D402A88C
:20F8E000F5F72BFD000654D442E08DF8109002A8F5F76CFCF6E704A8F5F7FCFF000648D4EF
:20F9000002AA9DF8101001200CE000BF8DF8109032E004A8F5F7EEFF00063AD402AA9DF8A9
:20F9200010100220F5F71DFE000632D49DF814000128EBD00328E9D01AE004A8F5F7DAFF96
:20F94000000626D402AA9DF810100320EAE704A8F5F7D0FF00061CD402AA9DF81010042070
:20F96000E0E7C17B8DF81010D0F80B00012602909DF810000028C9D00EA91E20CDE9000141
:20F9800006AB01229DF81010082007F053FC000614D5206819B0BDE8F08F8DF81090D0F81F
:20F9A000020002260290E7E7FFE7862008212060CAF800107946CBF80010EBE702230FA975
:20F9C00006A80E9AF0F7E6FE10B10020286085E0BDF83C000028F8D09DF814000028F4D0C2
:20F9E0000D22B6A140461FF0DEFE042306AABDF83C000021FFF7AEFA0E909DF81400012819
:20FA000002D0022803D004E0022E21D001E0012E1ED0032E15D0042E13D0052E18D0062E9A
:20FA200016D0032830D00428CFD1012ECDD10026A6490E9A9319C8891133834227D82868CA
:20FA40002CE09DF80C20002062F30700029901E002990020BDF83C200026A2FB013706FB19
:20FA6000017102FB001141F28830181842F2107341F100011A44D3171FF0CDFB022310AA03
:20FA8000FFF768FA0646D3E7022ED0D09DE70A2308F80030C98909EB41002860801B811A12
:20FAA00001EB0800C01E06A91FF07DFE28682521821B02EB080000F8031C76B1286832468D
:20FAC000811B01EB080010A91FF06DFE2868F621821B02EB080000F8011C002020607946B6
:20FAE000CAF800000020CBF8001053E72DE9FC416E4E002507460C46012A0AD00D600520AD
:20FB000030606C48056078466B4908600520BDE8FC8101A8F5F749FB000612D49DF80400BD
:20FB20006FF07708012806D002281AD003281AD0042821D11AE069461D2006F081FF00063F
:20FB400001D53068E3E79DF80000C00714D060A001683960416879600089388187F80A805E
:20FB6000CDE75EA0F4E714225FA101E0142264A138461FF018FEC2E72560C0E72DE9F04FD9
:20FB80004A4EA9B0054689464FF00008012A09D0022A3DD0032A7DD000200521C9F8000055
:20FBA000316073E224A8F5F700FB000673D49DF89000012805D0022803D0032801D0042817
:20FBC00022D107A90F2006F03BFF0006EED49DF81C00C00718D026A8F5F77CFB0006E5D40B
:20FBE0009DF8981081B104AA9420CDE900022B460122072007F01EFB0006D7D4022228466E
:20FC00000499FFF74FF934E20020C9F8000031E224A8F5F7CAFA0006C8D49DF89000012893
:20FC20007AD0022878D0032876D0042874D000208DF81C0026A8F5F74DFB0006B6D49DF83F
:20FC400098204AB19DF81C00C00705D0AFF6DC0122A81FF005FB804607A9312006F0F0FE9E
:20FC60000006A3D427A8F5F746FB00069ED4032310AA00212798FFF76DF9824625A8F5F7F6
:20FC80004BFB000692D4022318AA00212598FFF761F901E001E28DE1049025A8F5F74DFBD6
:20FCA000000693D4022308AA002136E008C0072079C207200CC0072010C00720828A8B9E59
:20FCC00097809F208D808B8E83000000F0CD072097858A208F908E848086880097858A2076
:20FCE0008F8E8A938F8A880097858A20828E878290809280208F908E848086880000000049
:20FD000097858A20828E878290809280208F8E8A938F8A880000000018E02598FFF71AF929
:20FD20000746F7481FF020FD049A04460AEB0200C3199DF81CC0691C0933F2480691BCF1A0
:20FD4000000F43D0BCF1010F07D00AE007A92A2006F076FE000684D46CE72799B1F57A7F8F
:20FD600034D0C189994279D28346881A0390284418A91FF018FD03985821801E52462954F9
:20FD8000A0EB0A00401E284410A91FF00CFDBBF80E003A46C7EB4000401C2844824608A9BF
:20FDA0001FF001FDF6210AF8011CB8F1000F79D0BBF80E10A81C0844424622A91FF0F3FCCD
:20FDC000BBF80E1008F1030008446EE08346C0893A46C01B2844824608A91FF0E4FCF62164
:20FDE0000AF8011C5FEA080007D0024622A9681C1FF0D9FC08F1020000E00020824607A9CE
:20FE00004E2006F01DFE0006A5D494B1BBF80E20D846D11BA1EB0A00401EA04203D39DF873
:20FE20001C00012805D09DF81C00C0B1012816D002E002208DF81C00BBF80E00C11BA1EBA9
:20FE40000A00411EA14200D80C46224605EB0A00AB491FF0A8FCBBF80E10FCE08EE006986A
:20FE6000294610441FF09FFCB8F80E102022491C2846F0F7BBFAB8F80E00A04200D80446D4
:20FE800022469F4928461FF08EFCB8F80E10012000EB4101C9F80010B8F80E100A2068546A
:20FEA000DBE0FFE7BBF80E00401C824607A94E2006F0C6FD00067DD494B1BBF80E20D8464A
:20FEC000C7EB4201A1EB0A00A04203D39DF81C00012805D09DF81C0000B301281ED002E0D3
:20FEE00002208DF81C00BBF80E00C7EB4001A1EB0A00A04200D80446224605EB0A008049C6
:20FF00001FF051FCBBF80E20012101EB4202C9F80020BBF80E000A2129549EE006981118C3
:20FF200005EB4200801C1FF03EFCB8F80E200698294610441FF037FCB8F80E102022491CB4
:20FF40002846F0F753FAB8F80E00A04200D8044622466B4928461FF026FCB8F80E0000EBD9
:20FF60004000801CC9F80000B8F80E100A206854B8F80E1005EB410148706EE0A1EB070B8C
:20FF800005EB0B003A4608A920901FF00CFC2098F62100F8011C049A18A9ABEB0200A0F102
:20FFA000020B05EB0B001FF0FEFBABF102005821295400E077E0A0EB0A00401E284452466F
:20FFC00010A91FF0F0FB5FEA080007D0024622A9681C1FF0E8FB08F1020000E000208346F9
:20FFE00007A94E2006F02CFD00065CD4CCB1DFF814810499B8F80E20D01B411AA1EB0A014D
:020000040001F9
:20000000A1EB0B00401FA04203D39DF81C00012807D09DF81C0000283FF421AF0128FBD0B1
:2000200002E002208DF81C00DFF8D8800499B8F80E00C01B411AA1EB0A01A1EB0B00411FCD
:20004000A14200D80C46224605EB0B002C491FF0AAFBB8F80E10C9F8001007A90B2006F097
:20006000EFFC00061FD49DF81C00022801D0042809D10020244930600860794623480160DA
:20008000002029B087E40520306000201E49086079461E4801600520F3E701222846FFF74C
:2000A000FCFB0006EFD53068EBE72DE9F0410024174D154E154F012A09D0022A13D0032A3F
:2000C00013D04FF00508042A13D00C6026E011A10A680260898881802C6078463460386060
:2000E0000020BDE8F081012200E00222BDE8F04144E50322FFF742FD00060FD52868F0E7F9
:20010000BBC20720F0CD07200CC0072010C0072008C0072091928E908D8E0000C5F80080E5
:200120007846346038600520DBE72DE9F0478EB006460C46FE4D0027DFF8F893DFF8F8A37F
:200140004FF00508012A01D00F6038E00BA8F5F727F9000615D40220CDE900040023F7A18B
:2001600030460B9AFFF785F90AA8F5F7F7F8000607D49DF8280010B30CA8F5F700F9000663
:2001800003D528680EB0BDE8F087042302AABDF830000021FEF7DEFE0246EB48C48902E0C9
:2001A000305D202801D0641EFAD1A01A3044401E02A91FF0F8FA2520311901F8010CC5F8C2
:2001C00000807946C9F800700520CAF80010D9E72DE9F047D64D0027DFF85893DFF858A3CD
:2001E0008EB006460C464FF00508012A01D00F6036E00BA8F5F7D4F8000615D40220CDE924
:2002000000040023D1A130460B9AFFF732F90AA8F5F7A4F8000607D49DF8280000B30CA8CA
:20022000F5F7ADF8000601D52868ABE7042302AABDF830000021FEF78DFE0246C248C48937
:2002400002E0305D202801D0641EFAD1A01A3044401E02A91FF0A7FA2520311901F8010C4D
:20026000C5F800807946C9F800700520CAF8001088E72DE9F04705270025DFF8B882DFF865
:20028000B892AB4CAAB082460E46012A01D00D6027E028A8F5F713FC000616D429A99420F6
:2002A000CDE9000102AB01229DF8A0100E2006F0C1FF000609D4032202A82999FEF7F2FD36
:2002C00027A8F5F76DF8000602D520682AB05AE70220CDE90006002302A95046279AFFF785
:2002E000C8F827607946C8F800500520C9F80010ECE72DE9F04F02278D4CABB083460D4651
:20030000012A0AD00026DFF82C92DFF82CA24FF00508022A11D00E6035E027A8F5F795F854
:20032000000626D4CDE9007500238BA15846279AFFF79FF82BB0BDE8F08F28A8F5F7BFFBE2
:20034000000616D429A99420CDE9000102AB01229DF8A0100E2006F06DFF000609D40322C3
:2003600002A82999FEF79EFD27A8F5F75DF8000601D52068DEE7CDE90075002302A95846B1
:20038000279AFFF776F8C4F800807946C9F800600520CAF80010CDE770B5654CAAB00646F5
:2003A0000D46022B19D027A8F5F70FFB000611D428A8F5F7F9FA00060CD429A99420CDE953
:2003C000000102AB01229DF89C100D2006F032FF00060AD520682AB070BD614988788DF814
:2003E0009C00D1F803002890E7E7032202A82999FEF758FD0220CDE90005002302A9304613
:20040000289AFFF736F805204A492060002008607846494908600520DDE72DE9F047002424
:20042000444E454F424DAAB082468846012A06D04FF00509022A0CD0C8F800403AE00D2278
:2004400048A11FF0B0F92C6078463460386000203CE7022B18D027A8F5F7B7FA000611D4D6
:2004600028A8F5F7A1FA00060CD429A99420CDE9000102AB01229DF89C100D2006F0DAFEF6
:20048000000609D5286821E7354881788DF89C10D0F803002890E8E7032202A82999FEF761
:2004A00001FD0221CDE90018002302A95046289AFEF7DFFFC5F800907846346038600520F8
:2004C00004E72DE9F04F1A4D8DB006460C464FF00208012A0AD00027DFF858A0DFF858B077
:2004E0004FF00509022A10D00F6067E00AA8F4F7ACFF000646D4CDE90084002316A13046FB
:200500000A9AFEF7B6FF0DB015E70AA8F4F78CFF000637D4CDE90084002308A130460A9A7B
:20052000FEF7A7FF0BA8F4F75DFF00062AD421E008C007200CC0072010C0072020918A8885
:20054000848A802000000000F0CD0720208D80848180828A80000000829185838E00000022
:2005600079C207208E928C858D80208D808B8E83800000009DF82C0000B30CA8F4F743FF3D
:20058000000601D52868BEE7042302AABDF830000021FEF7DFFC0246FC48C48902E0305D59
:2005A000202801D0641EFAD1A01A3044401E02A91FF0F9F82520311901F8010CC5F80090BC
:2005C0007946CAF800700520CBF800109BE72DE9F04FEF4D8DB006460C464FF00208012AD0
:2005E0000AD00027DFF8ACA3DFF8ACB34FF00509022A10D00F6045E00AA8F4F726FF0006E9
:2006000024D4CDE900840023AFF2B40130460A9AFEF72FFF77E70AA8F4F706FF000615D403
:20062000CDE900840023AFF2DC0130460A9AFEF720FF0BA8F4F7D6FE000607D49DF82C009D
:2006400000B30CA8F4F7DFFE000601D528685AE7042302AABDF830000021FEF77BFC024631
:20066000CA48C48902E0305D202801D0641EFAD1A01A3044401E02A91FF095F825203119E4
:2006800001F8010CC5F800907946CAF800700520CBF8001037E72DE9F74F05468CB00120FC
:2006A0000024834608900E98B94E8846A146A2462746012801D0022841D109A9192006F0E7
:2006C000BFF900067DD4B14C9DF82400E789C10701D002210891400703D57F1C4FF0020B8A
:2006E0007F08012008991AF07CFA0006EAD49DF82400C00602D501201AF0F1FBA348C089CC
:2007000000F00100C0F1010A0AA8F4F75FFD0006D8D402236A4600210A98FEF71BFC044693
:20072000401DB84209D8BBF1020F08D10A2000EB44019648C089814201D94FF001090E98DE
:2007400009226946012804D002284FD003287DD191E0B9F1000F05D090A000682860C8F821
:20076000007011E0BBF1020F15D08CA0224600682860381B054469462846C8F800701FF0FA
:2007800012F8F62005F8010C584608991AF029FA000616D465E083A0894603682B604068FE
:2007A00068607A4920464FF0FF37CB89A0EB040C07EB4C0C634409EB000CDBB21CF801CC85
:2007C00000E083E005F803C02B44401E03F8012CEBD1C889634207EB43031844C0B2F62350
:2007E0002B54284400F8012CC98934E0B9F1000F34D0DFF898B1601C8E469146BBF80E10AE
:20080000401E01EB0503A0EB04070AEB47011EF800205A54BBF80E302B44194401F8019C7C
:20082000ECD1012008991AF0DCF900064ED4BBF80E10F6224B1964420AEB44010B4403F8BB
:20084000022CBBF80E302B44194400E02DE001F8039CBBF80E10C8F8001002E00020C8F8C5
:2008600000004C4900203060086079464A48016000200FB05FE5012108461AF0B2F90006CB
:2008800024D400201AF02BFB00061FD409A90B2006F0D6F8000619D49DF8240001280ED0C3
:2008A00003280CD00020C8F80000052039493060002008607946384801600520D9E70222E9
:2008C00041462846FEF7E9FF0006EED53068D0E72DE9FC412E4D364E07460C46012A12D030
:2008E0000120022A1DD0032A23D0042A28D0002008600521296027490860784626490860D4
:200900000520BDE8FC8101A8F4F79FFB000601D52868F6E70123327821463846FEF783FBF3
:20092000EFE700900A46337801213846FEF7BFFBE7E7012300901A463846FEF7BAFEE0E733
:200940003846FEF76EFEDCE72DE9F04305260025104FDFF844800E4C89B08146012A01D00C
:200960000D6037E007A8FBF7F0FB000609D46846F4F77CFD000604D401A8F4F788FD000675
:2009800018D5206809B0BDE8F0830000F0CD072008C007200CC0072010C0072088928E8329
:2009A0000000000009880992098E09830000000085C00720DDE90023FCA102A81EF050FCF2
:2009C0000246FD48C18901EB09000799401A02A91EF0E9FE266079463D600520C8F80010DA
:2009E000D0E7F8B50125012A0FD0F44EF44FDFF8D4C30024022A10D005200C603060784661
:200A00003C60CCF800000520F8BDEF4A009513780A460821FEF74BFBF8BDDA074FEA8372CB
:200A20000BD0002A03DA01231A46009502E0012300220094FEF73DFEF8BD002A03DABDE86E
:200A4000F840FEF7B9BD0C60346078463C60CCF800000020F8BD2DE9F04F83460120D74E9C
:200A6000D74FDFF86083DFF86093002485B00D46082A72D2DFE802F08104394A68727A7C19
:200A800002A8F4F715FD000645D403A8F4F77CFB000640D49DF80800012801D002281CD1BB
:200AA000CA481EF061FE002860D0DFF80C93DFF81CA3B9F80E10814204D9091A50442022EB
:200AC000EFF794FCB9F80E20C04958460AF802401EF069FEB9F80E002860346079463C602B
:200AE0000020C8F8001005B025E402A8F4F7E0FC000610D403A8F4F747FB00060BD49DF89B
:200B000008000221012808D002280CD004A8F4F79CFA000610D53068E5E7CDE90015002339
:200B2000ABA1039A04E0CDE90015039A0023ABA15846FEF79EFCD6E7012399F800202946E3
:200B40005846FEF770FACEE7009099F800302A4602215846FEF7ABFAC5E70EE00123009079
:200B60001A4629465846FEF7A4FDBCE72C60B4E729465846FEF755FDB5E705202C60306077
:200B800079463C60C8F80010ADE7F0B58B4C0026ABB007460D46012A0AD00E6005202060E1
:200BA0008748066078468749086005202BB0F0BD29A8F4F7F5F9000624D49DF8A400012853
:200BC00001D02E60EAE727A8F4F7B9FA000619D49DF89C10012917D02AAA9420CDE90002F3
:200BE00002AB0122491E0C2006F024FB000609D4032202A82A99FEF755F928A8F4F7C4FA4C
:200C0000000607D52068D1E70F2276A102A81EF051FEF2E70220CDE90005002302A9384661
:200C2000289AFEF726FCB9E72DE9F0470024644E644F624DAAB082468846012A06D04FF086
:200C40000509022A0CD0C8F800403FE00E2269A11EF0A9FD2C60784634603860002012E4E5
:200C600028A8F4F76CFA00061FD420209DF8A0108DF8080002A8012919D027AB9322CDE94E
:200C80000023431C0122491E0C2006F0D3FA00060BD427990322491C02A82791FEF702F9D8
:200CA00029A8F4F771FA000607D5286808E40F224CA1401C1EF077FDF2E70221CDE90018E9
:200CC000002302A95046299AFEF7D3FBC5F800907846346038600520C1E72DE9FE4F02279A
:200CE000364D83460C46012A0AD00026DFF8D090DFF8D0A04FF00508022A10D00E601DE0EA
:200D000002A8F4F7D8F900060ED4CDE9007400233CA15846029AFEF7ACFBBDE8FE8F02A8A9
:200D2000F4F732FA000601D52868F6E7CDE90074002337A15846029AFEF79BFBC5F800802C
:200D40007946C9F800600520CAF80010E5E72DE9F843814610461C4A184D194E194F12785E
:200D600000244FF0010C06287AD2DFE800F082030A69707A0E220A6027A148461EF013FDE2
:200D800057E0294B98789A2852D12848006804284ED0001F80460246191D48461EF003FD92
:200DA000022241464846FEF77DF842E0253038752023253036750000F0CD072008C0072056
:200DC0000CC0072010C0072085C00720BBC20720828D8591858D888500000000829B8F8B9E
:200DE000809280008D808B88978D9B8C882020202020000091928E908D8E208F8B809285A1
:200E0000868000008F8E8B9397858D8E0000000091848097800000008E928A909B9288853A
:200E200020918C858D9B0000ECC2072088C007200C602C607846346038600020BDE8F88362
:200E400001B04846BDE8F0430123FEF7ECB813460A4603214846CDF800C0FEF728F9EDE7F4
:200E600007E001231A464846CDF800C0FEF721FCE4E705200C6028607846346038600520EF
:200E8000DCE72DE9FF5F83460D46924602A8F4F7F9FCFB4E00066FD469469DF80800F4F7D4
:200EA00005FD000668D49DF80800F64FDFF8D88300244FF005091B2871D2DFE800F0B35326
:200EC000AAAAAAAA666666668F8F8F8F0E313F47434B57B3B3B3B3B34F00BAF1010F03D090
:200EE000BAF1020F5BD101E0E8A167E003A8F4F7D1FF000640D49DF80C0070B101A9042049
:200F0000FBF734FF000637D4BDF8040010F10100ADF8040082B2E1A10BE0BDF80000F7E703
:200F2000BAF1010FE0D0BAF1020F7BD1BDF80020DFA158461EF094F9286074E0BDF80020FF
:200F4000E0A1F6E7BDF80020E4A1F2E7BDF80020E8A1EEE7BDF80020ECA1EAE7BDF80020C5
:200F6000F0A1E6E7BDF80020F5A1E2E701A90420FBF7FCFE000603D5306804B0BDE8F09FC7
:200F8000BDF80420F4A1521CD3E75146BAF1010F06D0022911D0BAF1030F43D119E041E09C
:200FA000F5A158461EF05CF928609DF80800072801D0092806D12C6004E0F2A158461EF0BE
:200FC0004FF92860346079463C600020C8F80010D3E707283FD006283DD038E0BAF1010F5C
:200FE00003D0BAF1020F1DD10FE00A2807D00B2807D00C2807D00D28DDD1E5A1DEE7E9A1AF
:20100000DCE7EDA1DAE7F1A1D8E7BDF80020F3A18FE75146BAF1010F0DD0022911D0BAF1A8
:20102000030F10D02C60C6F8009079463C600520C8F80010A1E70328BDD00528BBD0CEA12D
:20104000BCE7EBA1BAE7022805D0032803D0BDF80020EBA16DE7BDF80020EDA169E72DE945
:20106000F843814688466946292005F0E9FC844D00060DD49DF80000824E834FC0074FF0D9
:20108000000414D069463B2005F0DAFC000601D52868D3E6E3489DF80020C1894846EFF7D0
:2010A000A5F92C607846346038600020C6E6C8F80040F6E72DE9F74FAEB00E4693464FF04D
:2010C00000092AA94C2005F0BBFC6D4D000649D49DF8A8006B4FDFF8B081C0074C464FF0A8
:2010E000050A26D02CA8F1F7BDF800063AD49DF8B000F0B12BA99420CDE9000102AB012271
:2011000059460E2006F096F800062BD4032202A82B99FDF7C7FE29A8F4F7ECFB000621D48F
:20112000BDF8A4004FF0020A02280DD003280FD011E03460C5F800A079463C600520C8F8D8
:20114000001031B0BDE8F08F0320ADF8A40002E05046ADF8A4A027AA594680B2F4F781FCA3
:20116000000601D52868ECE79DF8A0004B46279A60F3070352EA030006D134602C60794657
:201180003C60C8F80010DCE7CDE900A602A92E98FEF76FF9D5E72DE9F74FAEB000250F4606
:2011A00016462C462BA8F1F75DF8DFF8D48000065CD427A8F4F79EFB0006F9D4BDF89C0079
:2011C0004FF0020A022802D0032804D005E00320ADF89C0001E0ADF89CA0DFF8A8B04FF050
:2011E0000009102E43D2DFE806F042080D244A494848484848484848484739462E98FFF7BE
:201200002EFF9EE7BDF89C00012805D0022809D0C7F80090484671E183A12E980A680260DD
:20122000496804E083A22E981168016051684160F0E79DF8AC0058B128A9BDF89C00F4F7CC
:201240004BF90006B4D49DF8A400289D60F3070420208DF80800BDF89C00012808D0022817
:2012600007D0032806D0042805D1FEE077E188E1E6E0F2E0EEE092E167E11AE1FCE03AE1E2
:2012800008C007200CC0072010C007208E92978592209193928E978D9B8900009120838047
:2012A00098858D88858C2024202530347500000081858720838098858D889F20242025304F
:2012C000347500008E92978592208F8E2091858A96889F8C20242025303475008F8E9780BB
:2012E000918E828E89208E929785922024202530347500008E92978592208A8091918890B4
:201300008E82202420253034750000008E92978592208A8E8B8897859192822024202530C8
:2013200034750000918B938685818D9B8920848E8A938C858D922024253034750000000057
:201340008E8199858520838098858D888520242025303475000000008082809088898D8E61
:20136000852087808A909B92888520918C858D9B2024202530347500918E8A908099858DBD
:201380008D9B89008E92978592209D8A8B87000088928E838820808A92888288878096884F
:2013A000880000008A8B208F8E208D8E8C85909320918C858D9B0000848E8A938C858D929B
:2013C000208F8E20238A8F8A000000008F8E208D8E8C85909320918C858D9B008E92978538
:2013E00092209D8A8B87202420253034750000008E92978592208F808C9F9288208F84002B
:201400008F8E20848092808C20242025303475008F8E20918C858D808C20242025303475B1
:2014200000000000F0CD07208F908E848086883A000000008F8E8A938F8A883A00000000BA
:20144000F7A00168CDF809108088ADF80D008DF80F90A4E01122F4A109E0F8A00168CDF8D5
:2014600009104068CDF80D0099E01222F5A10DF109001EF098F992E09DF8AC0060B128AA5A
:201480000121BDF89C00F4F7D0F8000667D49DF8A400289D60F307040F22AFF2B8610DF1A0
:2014A0000A001EF080F920208DF808008DF8090075E0082E2BD8F01E2CA9C0B205F0C0FAAE
:2014C00000064CD49DF8B000A8B100BF9DF8AC0060B128AA311FBDF89C00F4F7A6F8000635
:2014E0003DD49DF8A400289D60F3070455EA040011D1082E0FD94846C7F80090C8F800009F
:201500007946CBF80000D4480160002019E601208DF8B000DAE720208DF808008DF809003B
:201520002AA99220CDE900010DF10A030122711F0C2005F07FFE000611D42A990322891C9B
:2015400002A82A91FDF7AEFC29E09DF8AC0070B128A9BDF89C00F4F714FA000602D5D8F855
:201560000000EEE59DF8A400289D60F30704BDF89C0001280ED002280CD003280AD00428AD
:2015800008D0A6F10F02102A12D839462E98FFF791FDD6E5B14AB2A102A81DF061FECDE909
:2015A00000A72A46234602A92E98FDF762FFC8E50522C7F80090C8F800207946A648CBF872
:2015C000009001601046BCE52DE9F04F87B083460E46144602A8F4F78DF9A24F000630D40A
:2015E000DFF88492DFF870A24FF00008012C02D0022C34D114E0BDF8080001280BD0C6F829
:201600000080C7F800807946C9F800800020CAF8001007B096E531465846FFF720FDF8E7E0
:2016200000252C4605A8F0F71DFE000609D49DF8140068B103A9BDF80800F4F752F800061B
:2016400001D53868E5E79DF81000039D60F30704BDF80810022001290CD002290FD0052180
:20166000C6F8008039607946C9F800800520CAF80010CEE72A462346AFF6AC0103E02A4669
:201680002346AFF6A801CDE900065846FDF7F1FEBFE72DE9FF5F83460E46904603A8F0F7B7
:2016A000E1FD704C00066FD400270525DFF8B891DFF8A4A1ADF80870B8F1110F70D2DFE8CB
:2016C00008F06F86090D1D2A3786445364707B868B9BFE005846AFF2B02139E09DF80C00A9
:2016E00028B102A90120F4F747F80006DBD4CDE90056BDF8082000235CA18CE09DF80C0050
:2017000010B102A9012046E0CDE90056BDF80820002358A17FE09DF80C0010B102A9032082
:2017200045E0CDE90056BDF80820002353A172E09DF80C0010B102A9032043E0CDE90056D3
:20174000BDF80820002350A165E05846AFF21C310A6802604968416027607946C9F800702A
:201760000020CAF8001008E49DF80C0028B102A90220F4F701F8000606D4CDE90056BDF8BF
:201780000820002345A146E049E09DF80C000028BAD002A90220F4F705F800063FD4B3E70E
:2017A000AEE09DF80C000028BBD002A90420F3F7E3FF000633D4B4E79DF80C000028BDD0AE
:2017C00002A90420F3F7EEFF000628D4B6E731465846FFF744FC2DE49DF80C0028B102A943
:2017E0000120F3F794FF000672D4CDE90056BDF8082000232CA10EE09DF80C0028B102A913
:201800000220F3F784FF000662D4CDE90056BDF80820002327A15846FDF72BFE0AE457E049
:201820008F908E8480860000828E87829080928E82208F908E848086000000008F8E8A9315
:201840008F8E8A00828E87829080928E82208F8E8A938F8E8A00000010C007201401010008
:201860002025730008C007200CC00720208F908E848086002091928E908D8E0020828E8744
:20188000829080928E8200002091928E908D8E20828E87829080928E82000000208F8E8AE6
:2018A000938F8E8A00000000828D8591858D888900000000829B8F8B80920000FFE79DF8E2
:2018C0000C0060B102A91A20F3F7F0FF000601D5206848E7BDF80800401EADF80800CDE91C
:2018E0000056BDF808200023F5A15846FDF7C1FD25607946C9F800700520CAF8001032E727
:201900003760F5E72DE9F74FB2B00E46174600242EA8F0F7A7FCF04D00067DD430A8F3F70B
:20192000E9FF0006F9D42FA94B2005F089F80006F3D49DF8BC009DF8B81000F00100404245
:20194000DFF89893DFF898A30842A04670D0BDF8C000012804D1012F08D0022F2FD0BF1E7B
:2019600002282FD003282FD0C0B22EE04FF0010B01272BAA39465846F4F754F80006CCD452
:201980009DF8B0102B9861F3070450EA040103D17F1CFFB2052FECD950EA040106D10BF166
:2019A000010101F0FF0BBBF1040FE1D92043CDD031463298FFF753FB35B0BDE8F08F1622EB
:2019C000C8A141E0032000E002208346072F2FD2DFE807F0800441414141410001272BAAD4
:2019E00039465846F4F71EF8000661D49DF8B0102B9861F3070450EA040103D17F1CFFB2B8
:201A0000052FECD9204365D05846BBF1010F0CD002280ED0032800E04AE013D0BBF1040F20
:201A200016D0C6F8008040462AE00F22B3A10BE050E0B6A132980A680260898881808021AA
:201A40008171F0E70F22B3A132981DF0ACFEEAE70F22B4A1F8E77F1EF8B2014603902BAA8B
:201A60005846F3F7DFFF000622D49DF8B0002B9F60F3070457EA04000AD14046C6F80080B3
:201A800028607946C9F800000020CAF8001093E720208DF814002DA99320CDE900010DF1BB
:201AA000150301220D20039905F0C4FB000601D5286881E72D990322491C05A8FDF7F2F9BE
:201AC0000220CDE900063A46234605A93298FDF7D0FC71E70521C6F8008029607946C9F842
:201AE00000800520CAF8001066E72DE9F0478AB006460F46012A0DD0774C0025DFF8DC81D6
:201B0000DFF8DC91022A0AD04FF0050A032A2CD00D604DE0FFF7A3FA0AB0BDE8F08707A852
:201B2000F3F7B0FE00062ED406A9122004F088FF000628D49DF81C000E2801D0142805D1DD
:201B40009DF81800400701D57AA000E07CA001683160416871600089308125607946C8F8F3
:201B600000500020C9F80010D6E70020CDE9020008A8F0F777FB000605D404A90120F3F7EF
:201B8000FDF9000601D52068C6E704980290BDF81400ADF80C009DF816008DF80E00022036
:201BA000CDE90007DDE902234AA13046FDF761FCC4F800A07946C8F800500520C9F80010AA
:201BC000AAE72DE9F04F89B083460E46904602A8F0F748FB404C00066FD403A90120F3F793
:201BE0007BFC000669D407A90420F3F775FC000663D407A903A8F2F7FEFC00065DD405A99C
:201C00000320F3F769FC000657D407A90220F3F763FC000651D407A905A8F2F7ECFC0006A7
:201C20004BD4002202212D4FDFF8B49013464FF0050A1546B8F1070F40D2DFE808F0B5045E
:201C40001A1D222FA5009DF8080068B19DF81820002062F307039DF81040039A059964F3DE
:201C60000700521A60EB03030120CDE9000637A11FE0132237A106E09DF80800B0B13A4879
:201C800010E0142239A158461DF08DFD256079463D600020C9F8001009B08EE69DF8080073
:201CA00020B138480268007960F30703CDE9001608A15846FDF7DDFBEEE76BE074E0000040
:201CC000918B938685818D9B9520848E8A938C858D928E820000000008C007200CC007209B
:201CE00010C0072091938C8C80208D808B8E838E82208F8E2092888F808C00008F908E8415
:201D00008086802020202020202020008F8E8A938F8A8000828E8782908092208F908E845E
:201D200080868800828E8782908092208F8E8A938F8A8800888D8A8091918096889F0000E1
:201D40008D808B88978D8E91929C0000829B9093978A8000918C858D8D9B892088928E83E6
:201D6000208F908E8480860046000010918C858D8D9B892088928E83208F8E8A938F8E8A8A
:201D8000000000004B00001031465846FFF767F9000601D520687FE7C4F800A079463D60FB
:201DA0000520C9F8001077E73560F5E72DE9FF5F002483460D469046ADF80440274602A8D4
:201DC000F3F760FDFE4E00061AD44046B8F1050F04D0062802D0B8F1070F26D19DF8080012
:201DE0000E2801D0142820D103A90C2004F028FE000605D401A90220FBF708FA000601D542
:201E00003068B0E4BDF80400401EADF80400FDF789FB48B19DF80C00012803D0BDF804000F
:201E20001E2801D2012700E0002742460121E548DFF89483DFF894934FF0050A092A6CD2D8
:201E4000DFE802F06B050C252D2F3A4B54000278012329465846FDF7E6F884E49DF8082051
:201E60000C2A0FD2DFE802F0060E060606060E0E0E0E0E06009103782A4605215846FDF7E6
:201E800016F970E4009103782A460421F6E7012300911A4629465846FDF70BFC63E42C6071
:201EA00013E0002FFBD0CAA108200A68CBF800204968CBF8041007E0002FF0D01422C7A151
:201EC00058461DF070FC1420286034607946C8F800400020C9F8001045E4002FDFD0BDF82F
:201EE0000420C4A158461DF0BBF9EDE7FDF71AFB98B19DF808000E280FD014280DD029469A
:201F00005846FDF78EFB00BFC6F800A07946C8F800400520C9F8001025E42C60F4E72DE94E
:201F2000FF4F95B00E4690469A4603A8F3F7E2FCA34D000676D4BDF80C00A34FC0B2DFF855
:201F40008C9200240090B8F1010F08D04FF0050BB8F1020F28D0B8F1030F59D15AE00128D5
:201F600001D034604CE05046BAF1010F07D0022809D003280FD0BAF1040F41D10EE0AFF638
:201F80005831159802E0AFF6543115980A6802604968416034E011229CA101E01222A0A152
:201FA00015981DF000FC2BE04FF0000805AA50460099F3F7D6FA000634D414A8F0F752F985
:201FC00000062FD49DF81810404661F30700DDF814A080465AEA00011AD09DF85000B8B18E
:201FE00094A107A8009A1DF03BF90220CDE900065246434607A91598FDF73BFA000611D4B2
:202000002C6079463C600020C9F8001019B0D4E4346009E00AF1020231461598FDF73DFC9A
:20202000000601D52868F1E7C5F800B079463C600520C9F80010E9E72DE9FF4F85B00F46E0
:20204000914602A8F0F70EF95D4D000676D400224846DFF874B11446164690464FF0020A94
:20206000914607286BD2DFE800F07F04223345536B009DF80800B0B101208146014603AAB1
:202080000898F3F76EFA000663D49DF81000039960F3070409F101007618C0B248EB040838
:2020A00081461028EAD932464346644940E09DF8080050B103A90898F3F79EFA000648D402
:2020C0009DF81000039A60F3070423465C492FE09DF8080050B103A90898F3F777FA0006F8
:2020E00037D49DF81000039A60F307045449234610391DE00E2253A105981DF054FBC5F80F
:20210000009079463148CBF8009001600020C3E59DF8080050B103A90898F3F7DDF90006CB
:2021200017D49DF81000039A60F3070423462AA1CDE900A70598FDF79CF9ADE509E013E0EF
:202140000898042807D039460598FEF788FF000601D52868A0E505202860CBF80090794694
:202160001A480160052097E50521C7F800902960CBF80090F3E72DE9F74F8EB00F46924609
:2021800002A8F0F76FF80E4D000618D40DA8F3F7B1FB000613D4BDF83400DFF82C80C6B2DE
:2021A000DFF828900024192E08D15046BAF1010F57D002285CD0BAF1030F76D04AE097E0DA
:2021C00008C0072085C007200CC0072010C00720828D888C808D88850000000082208F80CC
:2021E0008C9F9288208F84208E9192808B8E919C00000000253034752091828E818E848DF1
:202200009B95208F8E8B858900000000828E87829080928E82208F908E8480863A0000005C
:20222000828E87829080928E82208F8E8A938F8E8A3A000020232530327500009C090100B3
:202240004C05010091938C8C80908D9B892088928E830000BAF1010F2ED0BAF1020F6FD12F
:202260003DE00E22AFF224010E981DF09CFA26E000229DF80800144650B103A90120F3F72B
:202280002BF9000634D49DF81000039A60F3070402202346AFF2C001CDE900070E98FDF728
:2022A000E8F811B0BDE8F08FFFE739460E98FEF7D6FE00061CD43AE0012E08D03C602C6046
:2022C0007946C8F800400020C9F80010E9E7AFF6A8610E980A68026049684160EFE74FF0EF
:2022E000000A03AA31460120F3F7C0F9000601D52868D6E79DF81010504661F30700DDF848
:202300000CB082465BEA00011AD09DF80800B0B13346721EFAA105A81CF0A2FF0220CDE935
:2023200000075A46534605A90E98FDF7A2F8052028607946C8F80040C9F80010B1E7FFE7C0
:202340003C60F4E72DE9F74F8EB00F46924602A8EFF788FFED4D000662D40DA8F3F7CAFA4F
:2023600000065DD4BDF83400DFF8A483C6B2DFF8A4930024192E08D15046BAF1010F0BD049
:20238000022810D0BAF1030F27D0BAF1010F2BD0BAF1020F6BD13AE00E22AFF258110E98D7
:2023A0001DF001FA23E000229DF80800144650B103A90220F3F790F8000631D49DF8100008
:2023C000039A60F3070402202346AFF2F411CDE900070E98FDF74DF863E739460E98FEF7D1
:2023E0003EFE00061CD43AE0012E08D03C602C607946C8F800400020C9F8001051E7AFF6D5
:20240000CC710E980A68026049684160EFE74FF0000A03AA31460220F3F728F9000601D567
:2024200028683EE79DF81010504661F30700DDF80CB082465BEA000119D09DF80800B0B1BB
:202440003346721EAEA105A81CF00AFF0220CDE900075A46534605A90E98FDF70AF80520DB
:2024600028607946C8F80040C9F8001019E73C60F5E72DE9F74F8EB00F46924602A8EFF775
:20248000F1FEA24D00065DD40DA8F3F733FA000658D4BDF83400DFF87882C6B2DFF874921A
:2024A0000024192E08D15046BAF1010F0BD002280DD0BAF1030F24D0BAF1010F28D0BAF196
:2024C000020F66D135E00E22AFF288212DE000229DF80800144650B103A90320F2F7FCFF4B
:2024E00000062FD49DF81000039A60F3070402202346AFF21C31CDE900070E98FCF7B9FFAC
:20250000CFE639460E98FEF7AAFD00061AD438E0012E08D03C602C607946C8F8004000202B
:20252000C9F80010BDE610227BA10E981DF03BF9F1E74FF0000A03AA31460320F3F796F812
:20254000000601D52868ACE69DF81010504661F30700DDF80CB082465BEA000119D09DF8BA
:202560000800B0B13346721E65A105A81CF078FE0220CDE900075A46534605A90E98FCF755
:2025800078FF052028607946C8F80040C9F8001087E63C60F5E72DE9F74F90B00E469346D9
:2025A00003A8EFF75FFE594D000654D40FA8F3F7A1F900064FD4BDF83C00DFF85481C7B2DF
:2025C000DFF8509100244FF0050A192F584605D0012825D0BBF1020F20D133E0012803D03B
:2025E000BBF1020F1AD103E00E22AFF2A83125E000229DF80C00174650B105A90420F2F7C5
:202600006BFF000627D49DF81800059A60F307070220CDE900063B4643A139E034603AE098
:20262000012F09D034602C607946C8F800400020C9F8001013B035E611223CA110981DF01E
:20264000B2F8F0E74FF0000B05AA39460420F3F70DF8000601D52868ECE7059904919DF867
:202660001810584661F30700049983460143D5D09DF80C000028D1D03B467A1E20A107A8F7
:202680001CF0EEFD0220CDE90006049A5B4607A91098FCF7EEFEC5F800A07946C8F80040D3
:2026A0000520C9F80010C5E72DE9F74F00208EB0044680460F4602A8EFF7D4FD134E000691
:2026C00072D40DA8F3F716F900067CD4BDF83400DFF83C9000F0FF0BDFF838A00025BBF1AA
:2026E0001F0F06D1109801282AD002282FD0032847D0109801284BD002287DD15CE00000FF
:2027000020253032752D25303275000008C007200CC0072010C00720828E87829080929B45
:20272000208F908E8480863A00000000828E87829080929B208F8E8A938F8E8A3A00000077
:202740000E22AFF200510E981DF02DF824E09DF8080058B103A90120F2F7BEFE000632D457
:202760009DF81000DDF80C8060F30704022042462346AFF24C01CDE900070E98FCF779FE27
:202780008FE539460E98FEF76AFC00061BD441E0BBF1010F09D03D6035607946C9F8005098
:2027A0000020CAF800107CE50DE0F7490E980A68026049684160EFE703AA59460120F2F7A1
:2027C00074FF000601D530686BE59DF81000DDF80C8060F3070458EA04000DD09DF808009E
:2027E00048B15A46AFF2B45105A81CF039FD9DF8080018B105E0FFE73D600BE00020044688
:2028000080460220CDE900074246234605A90E98FCF72FFE052030607946C9F80050CAF867
:2028200000103EE52DE9F74F90B00E46914603A8EFF718FDD54D000663D40FA8F3F75AF8A6
:2028400000065ED4BDF83C00D14F00F0FF0BDFF844830024BBF11F0F08D34846B9F1010F76
:202860000DD0022812D0B9F1030F29D000200290B9F1010F2BD0B9F1020F68D13AE00E2215
:20288000AFF2406110981CF08EFF24E000229DF80C00144650B105A90220F2F71DFE0006B9
:2028A0002FD49DF81800059A60F3070402202346AFF28C11CDE900061098FCF7DAFDB9E6D5
:2028C00031461098FEF7CBFB00061AD438E0BBF1010F07D034602C6079463C600020C8F824
:2028E0000010A7E6A84910980C310A68026049684160F0E705AA59460220F2F7D6FE000635
:2029000001D5286896E69DF818100298DDF814A061F3070081465AEA000118D09DF80C0005
:20292000A8B15A46AFF2F46107A81CF099FC0220CDE9000652464B4607A91098FCF799FD70
:202940000520286079463C60C8F8001072E63460F6E72DE9F74F00208EB0044680460F46B7
:2029600002A8EFF77FFC894E00065CD40DA8F2F7C1FF000657D4BDF83400DFF8149200F05A
:20298000FF0BDFF810A20025BBF11F0F06D11098012809D002280BD0032823D01098012830
:2029A00027D0022857D137E00E22AFF268712FE09DF8080058B103A90320F2F78DFD000610
:2029C00031D49DF81000DDF80C8060F30704022042462346AFF2B021CDE900070E98FCF7B3
:2029E00048FD5EE439460E98FEF739FB00061AD43FE0BBF1010F08D03D6035607946C9F8A9
:202A000000500020CAF800104BE41022AFF2F8210E981CF0C8FEF0E703AA59460320F2F7B2
:202A200044FE000601D530683BE49DF81000DDF80C8060F3070458EA04000CD09DF808009E
:202A400048B15A46AFF6140105A81CF009FC9DF8080010B104E03D600BE00020044680466B
:202A60000220CDE900074246234605A90E98FCF700FD052030607946C9F80050CAF80010EB
:202A80000FE42DE9F74F8EB00E46924602A8EFF7E9FB3E4D000651D40DA8F2F72BFF000685
:202AA0004CD4BDF83400DFF8E88000F0FF0BDFF8E4900024BBF11F0F05D3BAF1010F0AD01E
:202AC000BAF1020F0BD00027BAF1010F1CD0BAF1020F61D12BE00E22AFF6980123E0002205
:202AE0009DF80800174650B103A90420F2F7F4FC000623D49DF81000039A60F30707022070
:202B00003B46AFF2DC3131E0BBF1010F08D034602C607946C8F800400020C9F800100DE420
:202B20001122AFF2F8310E981CF03DFEF0E703AA59460420F2F7B9FD000601D528684BE42A
:202B40009DF81000DDF80CA060F307075AEA070022D09DF80800B0B15A46AFF6281105A888
:202B60001CF07EFB022052463B4605A9CDE900060E98FCF77EFC052028607946C8F80040AC
:202B8000C9F8001028E407E02814010008C007200CC0072010C007203460ECE72DE9F74F98
:202BA0008EB00E460CA8EFF75DFBFF4D000669D40BA8F2F79FFE000664D4BDF82C00FB4F60
:202BC00000F0FF0A9DF83000DFF8E4834FF005090024D8B15046BAF1100F3FD801460AAA8D
:202BE0000120F2F7DAFC00064CD40AAA51460320DDF828B0F2F7D1FC000643D410980A9A95
:202C0000012805D002280BD0032814D034601DE0BAF1010F02D1E7490E9852E0346054E0B3
:202C20005BEA0200F2D05246E3A102A81CF018FB03205A465AE04BEA020031E00320CDE988
:202C400000060023DEA10E98FCF713FCC5F8009079463C600520C8F8001007E4AAF11000F1
:202C6000C0B2834601460AAA0220F2F796FC000608D40AAA59460420DDF828A0F2F78DFC19
:202C8000000601D528683BE410980A9A01280AD0022810D003281FD00428B7D14AEA02004C
:202CA0000028CBD1B2E7BBF1010FB7D131460E98FEF7D5F909E0BBF1010FAFD1BD490E98C2
:202CC0000C310A680260496841602C6079463C600020C8F8001013E45AEA020096D05A4677
:202CE000B5A102A81CF0BCFA03205246CDE90006002302A90E98FCF7BCFB13E42DE9F04739
:202D00008946B349B14B0024A74DA84FDFF8A08209886FF07B0C0A2A59D2DFE802F05805F8
:202D20000A05121A242C3945D9892A22EDF75EFB68E01022A7A11CF036FD1021C9F800109C
:202D400060E0A9A2C9071268026080F804C048D136E0A7A21668066092888280CA0549D49C
:202D60004FEA01612AE0A4A2126802604A0541D44FEA815122E0A2A211F0280F16680660BB
:202D80005268426080F808C034D14FEA416115E09EA21668066056684660926882600A074D
:202DA00028D44FEAC16109E09CA2166806605268426048220272CA041CD44904002910DB58
:202DC000D989001F084498A1096801601AE00520C9F80040286079463C60C8F80010BDE8A3
:202DE000F087D989801F084491A10A6802608988818007E0D989C01E08448FA10988018042
:202E0000922181702C6079463C600020C8F80010E5E72DE9F0410024634D644E644F012AC0
:202E200004D00523022A0CD00C6017E0162283A11CF0B9FC2C607846346038600020BDE8D3
:202E4000F0816249C01FC98908448249D1F805200260B1F809208280C97A81712B6078466C
:202E6000346038600520EAE72DE9F04705464E4E4E4FDFF83C812020DFF8509100248AB075
:202E80004FF0050A072A77D2DFE802F07604263241596300DFF8C09199F8000078B10F22CF
:202EA0006EA128461CF07FFC99F800206FA101A81CF0D6F9024601A905F1110002E01522B7
:202EC0006CA128461CF06FFC346079463C600020C8F800100AB082E76CA10A2309682960CA
:202EE0002871B9F80E000A3D4119052269480BE069490C230622096829602871B9F80E00BB
:202F00000C3D41196348C01FEDF771FDE2E763A001682960416869608068A86009A904203C
:202F2000F9F724FF00061CD4B9F80E0021492D1F2844BDF82420F0391CF092F9C4E7012022
:202F400000905A480A46052103782846FCF7AFF8C0E70123022228460094FCF7AAFB0006B7
:202F600002D53068B6E707E0C6F800A079463C600520C8F80010ADE70C60F5E72DE9F74F78
:202F80000025094FDFF82480DFF8249090B00E4614464FF0050B1A2A04D90D60C7F800B074
:202FA000794685E08AE0000008C007200CC0072010C0072028140100202025303275000031
:202FC00020828E878290809200000000F0CD0720000000108082928E9285919288908E829E
:202FE000808D8885000000008F8E208F84000000454550524F4D00004652414D0000000079
:203000008F808C9F929C208F840000008F4F208F808C9F9288208F84000000004441544176
:20302000464C4153480000008D8E908C000000008D858D8E908C00008D85920082828584F1
:20304000858D208780828E84918A8E89208D8E8C859000006DC20720540000108F859085B2
:20306000908583889192908096889F002420253032750000808A92888288878096889F20EE
:203080008F808C9F9288208F8400000020908D8C200000005703001078F80000208D8E8C1F
:2030A000859020918C858D9B0000000085C00720C8F800500520C9F8001012E4012C15D097
:2030C0000E2C13D0142C11D0192C0FD0DFF804A45AF824001CF048FB421C5AF8241002A8BC
:2030E0001CF061FBFC48007810B121E00D6003E0A01F072808D835603D607946C8F80050CB
:203100000020C9F8001021E48E208F21022C06D0042C04D0032C07D0052C05D008E08DF8DA
:2031200014008DF8151003E08DF80F008DF810100FA92046F2F7BAFB000601D5386805E494
:20314000BDF83C000023401E82B2ADF83C20CDE900B602A91098FCF78CF9AEE72DE9F043B3
:2031600005270024DFF87483DFF87493DD4D8BB00646012A01D00C6031E0DBA001683160B4
:20318000416871608068B06009A813F0C8FD822810D1EDF745F80AA8F1F7BBFEEDF755F814
:2031A0009DF828001A2805D0192803D028680BB0BDE8F083BDF824009DF82630A0F5FA6011
:2031C00000909DF82720CCA101A81CF049F80246CD4801A9C0893044801A1CF0E4FA2F6049
:2031E0007946C8F800400520C9F80010DFE72DE9F04305260024B94FDFF8E482B94D8BB036
:203200008146012A01D00C601EE00D22BFA11CF0CAFA09A813F04EFD000601D52868C6E70A
:203220009DF8260000909DF825309DF82420BBA101A81CF015F8C2B2B348C18901EB0900B4
:20324000801A01A91CF0AFFA2E6079463C600520C8F80010ABE72DE9F04F0F46002189B001
:2032600005464FF0050A082A06D9121FB2FBFAF30AFB13220121121D9A4EDFF86082DFF8D6
:203280006092AA48DFF880B20024092A75D2DFE802F0A705141E303F4E5B7D000021084608
:2032A000F9F72FFD000678D41522A1A128461CF07AFA8848001F04708AE0012300223946A7
:2032C00028460094FCF7F5F909B0BDE8F08F97490020F9F7F0FC40B105285ED19AA2A1A187
:2032E00028461BF0BDFF38605DE01522AFF27C216BE0AFF268200068286020202871BBF85F
:203300000E000A3D411989480A2305220B300BE095490C2306220968296020212971BBF8F6
:203320000E100C3D2944001DEDF761FBCCE78FA10968296080212971BBF80E10083D2944C1
:203340000088EDF79AFBBFE7C9B1AFF2B0210A682A604A686A608968A9604288854901A827
:203360001BF07EFFBBF80E10081A284401990160029941600399816002E031E00DE03C6036
:203380005448001F0178491C017021E067490020F9F791FC80B1052801D0306894E7012072
:2033A000386020202870C6F800A07946C8F800400520C9F8001087E746486FA1001F0278E5
:2033C00001A81BF04DFF024601A928461CF0EBF934607946C8F800400020C9F8001073E7FF
:2033E0003C60E0E72DE9F04F89B005468946062A03D9D21E02F00302D21CDFF8D8A000246E
:20340000384E364FDFF8D8804848DFF8FCB0AAF1040A072A5DD2DFE802F05C0413323E4F6B
:20342000E30000210120F9F76CFC00060FD4152257A128461CF0B7F901218AF8011017E021
:203440003A490120F9F737FC80B1052801D030683AE755A128461BF003FFC9F80000052066
:20346000306079463C60C8F800102DE7C9F80040346079463C600020C8F8001024E79AF800
:2034800001204FA168461BF0EBFE0246694628461CF089F9ECE74FA10A230A682A604968E9
:2034A000696020212972BBF80E100A3D29440522001DEDF79CFA07E72CA1096829608021CE
:2034C0002971BBF80E10083D29440088EDF7D5FAFAE6A4E058000010FA0200000CC00720D9
:2034E00010C0072008C0072082828584858D80208480928000000000253032752D25303261
:20350000752D253032750000F0CD072082828584858D8E208290858C9F000000253032759E
:203520003A253032753A2530327500004C03001090858A82888788929B2090858388919278
:2035400090809688890000008D859220808A928882888780968889208F808C9F9288208FF1
:20356000840000002573000078F800002084809280000000381301008F85908590858388F4
:203580009192908096889F20253032750000000090858A82888788929B20808A92888288EC
:2035A00087809688890000008D859220808A928882888780968889209D8A8B870000000064
:2035C000808A92888288878096889F20242025750000000020908D209D8A8B872000000045
:2035E000AFF248510A682A604A686A608968A9604288FA4968461BF033FE0246BBF80E001F
:2036000069462844801A1CF0CEF89AF801100120491C8AF80110F249F9F74DFB54E6C9F8F9
:2036200000401CE7F0B591421BD900256F1E4FF00A0C3B46002406E010F806E0BEF1200F7D
:2036400000D13346641C944202D266198E42F3D3002B01DB00F803C025448D42E9D301200A
:20366000F0BD0020F0BD2DE9F05FDFF878A30024DD4EDE4FDFF8788383460D46012A05D00F
:203680004FF00509022A15D00C601FE0D9A2DCA11BF0E6FD401E28600146BAF80E205846D0
:2036A000FFF7C0FF346079463C600020C8F80010BDE8F09FD4A2DAA11BF0D2FD401E286091
:2036C0000146BAF80E205846FFF7ACFFC6F8009079463C600520C8F80010E9E72DE9FF4FB2
:2036E000C14EDFF80893DFF808A381B00F461C464FF00008012A04D0022A66D0032A78D1C1
:2037000075E0C94DDFF8DCB2102C2DD006DC062C1ED00A2C3CD00F2C04D110E0142C4AD002
:20372000162C35D0AB4655F824001CF01DF805465BF8241001981BF0F3FF3D6068E0BA4870
:20374000E96B7038427801981BF08AFD0546F4E709220A60A96901981CF025F80221084688
:2037600017F03FFA05B0B0E569461920F2F79EF800064BD455F82410BDF8002001981BF039
:203780006FFDBBF80E10814200D80846386024E0A54850F824001BF0E7FF0546A24850F8A0
:2037A000241001981BF0BCFFBBF80E2029460198FFF738FFC1E79D4855F823100288019830
:2037C0001BF04EFDBBF80E50B7E7062B11D116220A6097A101981BF0E6FFC6F80080794671
:2037E000C9F800800020CAF80010BBE701E0062B06D0C1F8008005213160C9F800800BE0F0
:203800000121084617F0EDF9000601D53068A9E705203060C9F8008079460520CAF800109B
:20382000A0E72DE9F0430024704E714F6E4D8DB08146012A09D0022A23D0032A2CD04FF0CC
:203840000508042A2FD00C604EE00BA8F6F77AFE01A9BDF82C00EDF710F920208DF80C0033
:2038600009A8F6F753FE0DF10D01BDF82400EDF722F95C480E22C18901EB09000E3801A972
:2038800001E00F2270A11BF08EFF2C6078463460386000200DB08BE44FF00F020BB16EA190
:2038A000F1E771A1EFE774480122002B0078009203460A4601D0062100E007214846FBF71B
:2038C000F6FB00060ED40AA8F1F77BFB000609D40AA8F1F7E0F8000604D40AA8F1F767FBD0
:2038E000000601D52868D5E7C5F800807846346038600520CEE72DE9F04705263A4F00247A
:20390000DFF8E880DFF8E8900D46012A01D00C6006E05A495AA20B685CA11BF0A1FC286039
:203920003E607946C8F800400520C9F80010BDE8F08738B56946182003F082F82A4C00065B
:203940001BD49DF80000574D410702D42978012906D0010702D42978022901D0297871B93A
:2039600000F00300012804D0022801D0032806D1002017F025FC000601D5206838BD002099
:2039800028700521216019490860784618490860052038BD2DE9FE4F0024134EDFF84C80F2
:2039A000DFF84C9082460D46012A06D00527022A12D0032A11D00C60A2E012223AA11BF0E8
:2039C000F2FE1220286034607946C8F800400020C9F80010BDE8FE8F70E07FE038130100CC
:2039E0004C030010F0CD072008C007200CC0072010C0072091818E89209780918E820000AA
:203A000025730A0A000000008F84208220908586888C852082828E8480208480929B0000EA
:203A200025730A0A0A0A0A00C400001030C007209D8A8B87208F8E9792880A2087808F8E5C
:203A40008B8D858D802100008F84208F85908582858B209780919B008D80208B85928D8569
:203A600085208290858C9F008D802087888C8D8585208290858C9F0085C0072054C00720F7
:203A80008E9888818A80209D8A8B870025732025750A200A200A200A200A200A200A200A12
:203AA000200A000000C007209080878D9B85208D8E8C85908020918C858D000002A9042037
:203AC000F9F754F900060FD4CDE90075BDF808200023F7A15046FBF7CCFC7BE702A906207A
:203AE000F7F7FEFB000601D5306873E7BDF80820CDE90075521ED317F0A15046FBF7B9FCE1
:203B000037607946C8F800400520C9F8001061E72DE9FE4FED4BDFF8B0B3ED4DB3F80480D3
:203B2000B3F806A0EB4EEC4F0024A0F10909012A11D06FF0640EA0F1060C022A17D0032A39
:203B400020D0042A3AD005200C60286078463460386005203EE7B8F1000F06D0BAF1000FA8
:203B600003D043214170988817E00C6020E0DBA10A6802604A6842600989018180F80AE0C0
:203B80001A8825E0B8F1000FEFD0BAF1000FECD08F2141708E218170D8886946ECF76DFF32
:203BA000BBF80E1001EB090000990160019941602C6078463460386000200BE7C7A10A68A8
:203BC00002604A6842600989018180F80AE05A88BBF80E00C4A160441BF042FBE8E72DE9E0
:203BE000FF410023CDE90233B94DBA4EBA4F1C46012A10D00223022A10D0032A10D0042A87
:203C000018D005200C602860784634603860052004B0BDE8F0811522B5A103E0BA4A0AE06C
:203C20001622BAA11BF0BFFD2C607846346038600020EDE7BB4A146802949488ADF80C409C
:203C40009279CDE900318DF80E20DDE902239AA1FBF70FFCDCE72DE9F0430023B24F9C4E82
:203C6000DFF87082DFF8709285B005461C46012A0FD00220022A2CD0032A32D00C600520AC
:203C800030607946C8F80040C9F8001005B0BDE8F083388802A9ECF7F0FE8B48C189A5F148
:203CA0000900084402990160039941609F48A0A1028802A81BF0D4FA024602A928461BF0D5
:203CC00072FD34607946C8F800400020C9F80010DCE73C7A7A68CDE9000164F307039649DF
:203CE00008E07C7BD7F80920CDE90001924964F3070318312846FBF7BCFBC7E72DE9F04F97
:203D000087B083460E46924604A9122002F098FE6F4D000604D405A8F1F7B4FD000603D552
:203D2000286807B0BDE8F08F9DF81000694FDFF8A881C0074FF000044FF0050905D09DF8FA
:203D400014000E2803D0142801D034601FE00020CDE902005146BAF1010F20D0022002293F
:203D600020D0032930D0BAF1040FEED16D490A6802928A88ADF80C2089798DF80E10CDE9B0
:203D80000006DDE902234CA15846FBF772FBC5F8009079463C600520C8F80010C1E71922C8
:203DA00066A113E058490A6802928A88ADF80C2089798DF80E10CDE90006DDE902233EA154
:203DC0005846FBF756FBACE71A2263A158461BF0EAFC2C6079463C600020C8F80010A0E742
:203DE0002DE9F04782468CB00020CDE9020004464E480227364DDFF8DC80DFF8DC90008810
:203E00000E460E2A52D2DFE802F051070F1D2234373A45CFD2F1FEEE56A2AFF6B80150463F
:203E20001BF01EFA3060E6E043490A68CAF800204A68CAF804200989AAF8081086218AF81C
:203E40000A10D8E002A90120DFE04FA2BDE004A9F7F7D2FF00062AD4AFF6A4024B4909A877
:203E60001BF0FEF9049802909DF814008DF80C00AFE0152246A1BBE002A90320C5E004A970
:203E8000F7F7BAFF000612D4DDF81A0002909DF81E0096E0284918310A68CAF800204A6825
:203EA000CAF804208968CAF80810A4E0BFE0B6E0918C858D80208F8400000000918C858D87
:203EC00080209D8A8B870000F0CD07204AC0072008C007200CC0072010C007208D8E8C85EF
:203EE0009020918C858D9B002530346C750A000043938C8C80908D9B892088928E83208F2B
:203F0000908E8480860000003CC0072043938C8C80908D9B892088928E83208F8E8A938FF3
:203F20008E8A000043C007204C03001030C0072024253034750000005C1D01008D858E810C
:203F40008D938B9F858C809F2091938C8C80208F908E8480860000008D858E818D938B9F49
:203F6000858C809F2091938C8C80208F8E8A938F8E8A00009080878D9B852088928E83881D
:203F800020918C858D0000008F8400006018010088928E8320828E87829080928E82208F81
:203FA000908E84808600000002A902202DE004A9F7F722FF000632D4DDF8150002909DF8A6
:203FC00019008DF80C00AFF61022F84909A81BF047F9CDE90076DDE9022309A95046FBF7D2
:203FE00048FA0CB0A3E415E00DE0FFE71622F0A150461BF0D8FB2C607946C8F800400020CC
:20400000C9F80010EDE702A90420F1F765FA000605D41AE704A9F7F7EFFE000601D5286811
:20402000DFE7DDF81F0002909DF82300C9E70520346028607946C8F80040C9F80010D0E744
:204040002DE9FC4107460C46164601A8F1F71AFCDD4D000608D4012E27D169469DF80400F0
:20406000F1F724FC000602D52868BDE8FC819DF80400152806D0162808D017280AD018288E
:2040800013D10BE0BDF80020D0A10AE0BDF80020D4A106E0BDF80020DBA102E0BDF80020E9
:2040A000E2A138461BF0DCF820600520EA492860002008607846E94908600520D5E72DE9E9
:2040C000F04FADB0074601202190109000202490269001900E46924629A8F1F7D3FBBA4DB0
:2040E000000670D4DFF878B3DFF86C83DFF86C939BF801003122002415283AD2DFE800F0CD
:20410000390B49FDFCFBFBFAFAF9F8F74B4BF6F5F4F3F2F1F000BAF1010F03D0BAF1020FC2
:2041200006D026E09DF8A400192877D0346056E29BF802006FF0770A012806D002281AD08E
:2041400003281BD0042814D11CE023A91D2002F077FC0006C5D49DF88C00800709D5C148A0
:2041600001683960416879600089388187F80AA080E23460FCE7BB480C30F1E7B949142228
:20418000183102E0B7491422303138461BF00BFB70E20D23D9E10D2804D1BAF1010F0CD0F1
:2041A000AAF1010A5046BAF1010F0DD0022836D0BAF1030FDDD10722FCE3AB480168396093
:2041C0008088B8800BE227E29BF80200DA46012805D0022803D0032801D00428A6D123A98E
:2041E0000F2002F02DFC0006B4D49DF88C0080079CD59AF80F10002998D002AA9420CDE976
:2042000000023B460122072003F014F80006A1D4022238460299FAF745FEE0E1F1E39BF8BE
:204220000200DA46012815D0022813D0032811D004280FD08DF88C409AF80F208AB19DF848
:204240008C0080070DD5AFF6C04127A81BF008F8259007E023A92A2002F0F2FB0006C3D4BB
:20426000EAE725942AA9322002F0EAFB0006BBD4DFF8ECA10323AAF10C0A19AADAF8130040
:2042800000210090FAF766FE0190DAF80F00022303AA0021FAF75EFE0290DAF817000223C6
:2042A00011AA0021FAF756FE82466D48103021901BF05AFA8346DDE90102811801EB0A03EC
:2042C0009DF8A8000933E8B3012803D10098B0F57A7F44D06548C189994265D2881A0DE0EB
:2042E000FEE341E139E1FCE3FCE3E2E2D4E284E246E226E2BFE13EE126E123E100903844FD
:2043000003A91BF050FA00985821801E39540199401A401E0A46384419A91BF044FA53489C
:204320005246C189CAEB4100401C384411A900901BF039FA0098F62100F8011C4B48259A2F
:204340008AB300E00BE0C189B81C084427A91BF02AFA4648C1892598C01C08448CE0434838
:204360005246C189A1EB0A00384411A901901BF01AFA0198F62100F8011C259A32B127A9A8
:20438000781C1BF010FA2598801C00E0002037495B46B1F80EC0ACEB0A01091A4A1E5A45B7
:2043A00066D91946B9E065E07BE061E06018010088928E8320828E87829080928E82208FA7
:2043C0008E8A938F8E8A000008C007208A8E8D92908E8B9C8D809F208B858D92802024253C
:2043E000303275008A8E8D92908E8B9C8D809F208B858D928020242530327520918E8A9056
:204400008099858D8D809F008A8E8D92908E8B9C8D809F208B858D9280202425303275206E
:204420009120838098858D88858C00008A8E8D92902E8B858D928020242530327520918E62
:204440008A908099858D8D809F209120838098858D88858C000000000CC0072010C007206A
:2044600079C20720D0FC000014010100F0CD0720491E52E0C089401CDFF878C45B46BCF86E
:204480000E20CAEB4201091A594500D919460B46012101EB42013160BCF80E200A21B954B0
:2044A0003EE0A1EB0A0000903844524611A926901BF079F92698F62100F8011C029A009899
:2044C00003A9801A801E009038441BF06CF900985821801E39540199401A401E0A46384422
:2044E00019A91BF060F9259A32B127A9781C1BF05AF92598801C00E00020FE49029A5B4655
:20450000B1F80EC0ACEB0A018A1A0199511A091A4A1F5A453FF645AF491F0B46C6F800C04E
:2045200038441A4621991BF03EF923A90B2002F087FA000670D49DF88C0002284FD0042859
:20454000FCD066E30C2300E00B23524631463846FFF7C4F82DB0BDE8F08F02235246314695
:204560003846FBF719FFF5E70223524631463846FBF753FFEEE75146BAF1090FBFF4D1AD81
:20458000DFE80AF00506202E4B4E55647200F0E5D94800901BF0E8F800283FF4C7ADDFF826
:2045A00054A3BAF80E10814205D9091A584411302022EBF71BFFBAF80E20384600991BF053
:2045C000F2F82DE29DF8A40019287FF4AFAD10230A4631463846FFF781F80006AAD4E4E268
:2045E000052809D10220CDE90006DBF80C200023C2493846FAF73DFF9BF801100629EED16C
:204600000221CDE90016BD49DBF80C2000230C313846FAF72EFFC8E2ADE29BF81020CEE2FE
:20462000022000909BF8103032460146D3E223A9282002F005FA0006D0D49DF88C00C007EA
:20464000ABD031463846FAF7B7FF83E723A9272002F0F6F90006C1D49DF88C00C0079CD0F6
:20466000022300220094E9E031463846FAF7D9FF0006B3D4CDE2BAF1010F1BD0BAF1020F3A
:2046800085D19BF80610F9B102A8CDE90020DA4603AB01220E2002F0CDFD00069ED4032279
:2046A00003A80299FAF7FEFB0220CDE90006DAF80A205FE0DBF80220002AC1D00220CDE929
:2046C000000600238E493EE2DA4608280AD10220CDE900068A49DAF80A2000231C393846EC
:2046E000FAF7C7FE9AF8010007280AD10220CDE900068349DAF80A2000230C393846FAF7EA
:20470000B8FE9AF807100029B4D0BAF80800042303AA0021FAF71EFC024602907548C689ED
:2047200002E0B85D202801D0761EFAD1B01A401E384403A91BF037F82520B91901F8010C63
:2047400067E29BF8021001290DD002A8CDE90020491E03AB01220C2002F06CFD000688D4C3
:204760000322029940E065490F22143103A81BF0A1F83CE0002303A93846FAF77AFE48E2EA
:20478000BAF1010F23D0BAF1020F7FF4CAACDFF864A1202203A8BAF80E10EBF727FE9BF893
:2047A0000210012917D002AA3020CDE90002531D491E01220C2002F03DFD0006CFD402998C
:2047C000BAF80E004A1C90420CD2491C0BE04B490E222431E6E149490DF10D0014311AF0E7
:2047E0009FFF04E00146032203A8FAF75BFB0220CDE90006DBF80320BCE7BAF1070FBFF4EE
:2048000090ACDFE80AF005FD06040D2025000EE7AFE4022000909BF80C3032460121DAE1DF
:2048200023A9272002F00CF9000698D49DF88C00C0073FF47BAC02230122009431463846E9
:20484000FAF737FF86E631463846FAF7EAFE81E62BA8F1F71FFB0006B0D49DF8AC000028C8
:20486000D6D0284800780028D2D02449DBF81130DBF80D20243903A81AF0F2FC029025A800
:20488000F7F763FC000699D41A482599029AC0893844401A03A979E40BF102001AF064FF09
:2048A00002903168814200D202910BF10201029A6BE4BAF1010F02D0BAF1020F4ED123A987
:2048C000192002F0BDF80006AFD40A489DF88C10C08901908A0701D502222192090704D5EB
